:020000040800F2
:104000000050002079FC0008E5CD0008E9CD00084B
:10401000EDCD0008F1CD0008F5CD0008000000004E
:10402000000000000000000000000000FDCD0008BE
:10403000F9CD00080000000001CE00089D9900089D
:1040400005CE000809CE00080DCE000811CE0008EC
:1040500015CE000819CE00081DCE000821CE00089C
:1040600025CE000829CE00082DCE00080000000053
:104070000000000000000000000000000000000040
:1040800000000000000000004DCE000851CE0008E6
:1040900061CE000871CE000881CE000891CE0008E4
:1040A00095CE000899CE00089DCE0008A1CE00084C
:1040B000A5CE0008A9CE0008ADCE0008B1CE0008FC
:1040C000B5CE0008B9CE0008BDCE0008C1CE0008AC
:1040D000C5CE0008C9CE0008A1900008D1CE0008C6
:1040E000D5CE0008D9CE0008DDCE000800000000C3
:1040F00000000000000000000000000000000000C0
:0C41000000000000000000005FF800005C
:1041100030BF704720BF704740BF7047BFF36F8FFD
:104120007047BFF34F8F7047BFF35F8F704701DF5A
:104130007047EFF31480704780F31488BFF36F8FDC
:104140007047EFF30980704780F309887047EFF3F9
:104150000880704780F30888704772B6704762B66F
:10416000704771B6704761B6704780F31188704729
:10417000EFF31280704740BA704700BA70470000F2
:104180000E4B10B59B680E4813F4004C0D490E4AB7
:104190000E4B09D04FF0010C0D4C80F800C00D48BB
:1041A0001C6010600C6007E080F800C00A480860DE
:1041B0000A4911600A4A1A6010BD00BF0008014098
:1041C000BC0D0020240E0020E00F0020A00E0020D7
:1041D00015930008859F0008A9930008E59800083A
:1041E0002D98000837B50AF019FA6F4B00254FF4E7
:1041F00080301D700AF032FA0AF096FB012804465E
:1042000027D1102009F0F4FC28460AF077FA284656
:104210000AF088FA4FF480600AF07AFA4FF44030DE
:104220004FF4E0110AF046FA20460AF04FFA39201E
:104230000AF064FB0028FAD0022009F0C1FC022039
:104240000AF04AFA0AF052FA0828FBD1564B01222A
:104250001A70042001210AF007FB03238DF80630B1
:10426000153301A951488DF807304FF48073ADF82C
:10427000043009F0F1FE06200AF03AFB0120014665
:104280000AF0F2FA4FF480414FF000600AF0E8F8CB
:104290004FF440700AF046F800F050FA00F0B4FB1A
:1042A000FFF76EFF00F060F905F0D8FB05F0A8FB02
:1042B00004F018FE00F080F800F072F930B100F060
:1042C0006FF93B4C607000F06BF9A060384C00F067
:1042D000BDF9207804F044FFE07804F09DFE354BF2
:1042E0001B7823B922696079A16805F0F7F8314B92
:1042F0001B780BB105F0F8FE06F0D4FC08F010FBBB
:1043000001F0CCFD05F00CFF06F032FD274B4FF419
:1043100000721A61A2F5A07203F580635A6105F07C
:1043200069FB044603F05EFF06F036FD05F00AFF68
:1043300005F060FB001B0028B8BF4042B0F57A7F53
:1043400025DD1C4C237893B1184B9B6813F4004374
:104350001AD1237005F088FE05F064FDFFF710FF09
:10436000134B1A695879996805F0B8F80CE00F4BAF
:104370009B6813F4004F07D005F074F801232370F5
:10438000FFF7FEFE05F0B0FE05F034FB044600F03A
:104390005DF900F04DF90028C4D006F083FC01F06F
:1043A0007DFD06F0E5FCBDE7C80F002000080140D8
:1043B00004000020BC0D0020134B82B01B7803B317
:1043C000124B4FF400625A61A2F580621A61002319
:1043D00001E0019B01330193019A0D4B9A42F8D9F8
:1043E0000A4B4FF400621A61A2F580625A61002301
:1043F00001E0019B01330193019A054B9A42DFD8FA
:10440000F7E702B0704700BF440E0020000C0140E7
:104410003F0D0300072816D8DFE800F00406080A5D
:104420000C0E101201220CE002220AE0042208E025
:10443000082206E0102204E0202202E0402200E0F0
:104440008022014B5A61704700140140072816D89A
:10445000DFE800F00406080A0C0E101201220CE03E
:1044600002220AE0042208E0082206E0102204E00A
:10447000202202E0402200E08022014B1A617047B6
:104480000014014038B50546002455FA04F2E3B2A1
:1044900012F0010F184602D0FFF7D8FF01E0FFF736
:1044A000B9FF0134082CF0D138BD00BF072805D86A
:1044B000DFE800F0060B10151A1F2429002026E063
:1044C000134BD86800F0010021E0114BD868C0F30D
:1044D00040001CE00E4BD868C0F3800017E00C4B86
:1044E000D868C0F3C00012E0094BD868C0F30010D0
:1044F0000DE0074BD868C0F3401008E0044BD868C3
:10450000C0F3801003E0024BD868C0F3C0107047BE
:1045100000140140052804D8DFE800F0050A0F1454
:10452000191E00201CE00F4B986800F0010017E0F6
:104530000C4B9868C0F3400012E00A4B9868C0F337
:1045400080000DE0074B9868C0F3C00008E0054B01
:104550009868C0F3001003E0024B9868C0F3401065
:10456000704700BF0018014062B6704772B67047CE
:1045700010F0010F03D0094B10221A6102E0074B23
:1045800010225A6110F0020F03D0044B20221A614E
:1045900002E0024B20225A61704700BF000C01402C
:1045A0001C4B9A689B6812F4807F14BF0020802007
:1045B00013F4007F03D1002814BFC0204020154B06
:1045C0009B6813F4806F134B08BF40F020009B687A
:1045D00013F4006F0F4B08BF40F010009B6813F4FA
:1045E000805F0C4B08BF40F008009B6813F4005F2D
:1045F000084B08BF40F004009B6813F4804F054B44
:1046000008BF40F002009B6813F4004F08BF40F061
:104610000100704700100140044B18780138C0B207
:1046200001288CBF00200120704700BF2802002015
:10463000044B1878012801D0002001E002221A70F2
:10464000704700BF2802002000207047082008B5EE
:1046500005F0ECF9592804D9064B1A784AB9013209
:1046600006E0082005F0E2F9542802D8014B0022A8
:104670001A7008BD2802002008B5072805D8DFE811
:1046800000F006080D121720252A002027E0002040
:104690000FE0134B9868C0F3400020E0104B98687F
:1046A000C0F380001BE00E4B9868C0F3C00016E01A
:1046B000042005F0BBF9B0F5006F94BF0020012085
:1046C0000DE0074B9868C0F3401008E0044B986871
:1046D000C0F3801003E0024B9868C0F3C01008BD1F
:1046E0000010014038B500242546E0B2FFF7C4FFB2
:1046F00020B10123A34043EA0505EDB20134082CA3
:10470000F3D1284638BD00BF08B5C0B206F078F82E
:1047100008BD00BF08B5C0B206F062F808BD00BF12
:1047200008B510B109F0A6FE01E009F0ABFE08BD26
:1047300008B5C90805F0E0FE08BD00BF2DE9F34744
:10474000644F6548012101AD09F016FD04200121E7
:1047500003240AF089F81026384642F202632946FB
:10476000ADF804308DF806408DF8076009F074FC50
:1047700040F202634FF0040838467B6129464CF250
:104780000803DFF868A1ADF804308DF806408DF815
:10479000078009F061FC4FF001033846294648279D
:1047A000ADF804308DF807708DF8064009F054FC20
:1047B000082001210AF058F841F6FD4950462946E3
:1047C000ADF804908DF806408DF8076009F044FCC0
:1047D000CAF81090304601210AF046F84FF0FF0960
:1047E0003E482946ADF804908DF806408DF80780C4
:1047F00009F032FC4FF60073384829460AF5006A82
:10480000ADF804308DF807708DF8064009F024FCEF
:10481000202001210AF028F84FF0FF3350462946A6
:104820002F4FADF804308DF806408DF8076009F081
:1048300013FC4FF47F43CAF8103040200121CAF81E
:1048400014900AF011F840F2FF3338462946ADF8CB
:1048500004308DF807808DF8064009F0FDFB4FF617
:10486000004329463846ADF804308DF806408DF8EF
:10487000076009F0F1FB4FF47C4301217B6119488B
:1048800009F07AFC00231A461946124C4FF40055E1
:1048900065612046A468013314F4804F4FF400543E
:1048A0000461806808BF013110F4804F18BF0132E5
:1048B0000A2BEAD10A2903D10A2A01D1012200E0F8
:1048C0000022094B04481A70012109F055FCBDE88B
:1048D000FC8700BF000801400002300000100140CA
:1048E0000018014000043000440E0020000C01407C
:1048F00070B504460D46164608287AD8DFE800F061
:1049000005101316191C1F0A0D003B4B4FF4805263
:104910005A6119E04FF4007213E04FF4807210E016
:104920004FF480620DE04FF400620AE04FF48052D1
:1049300007E04FF4005204E04FF4804201E04FF4EE
:1049400000422E4B5A6110E02D4802210AF0EEF889
:104950000028F9D029462A480AF08CF82848012175
:104960000AF0E4F80028F9D00FE0264802210AF006
:10497000DDF80028F9D0294622480AF07BF82148C2
:1049800001210AF0D3F80028F9D03EB3082C30D822
:10499000DFE804F005101316191E210A0D00164B4E
:1049A0004FF480521A611DE04FF400720DE04FF495
:1049B00080720AE04FF4806207E04FF4006204E086
:1049C0004FF4805201E04FF400520C4B1A610BE09F
:1049D0004FF48042F9E74FF40042F6E714B1082C97
:1049E00007D801E0064800E006480AF045F8C0B2E2
:1049F00000E0002070BD00BF000C01400014014029
:104A000000380040003001402DE9F04F01218BB00B
:104A10004FF4804009F036FF494C012009AF0146B0
:104A200009F022FF03264FF0180B204639464AF2C0
:104A30000003DFF81491ADF824304FF0040A8DF82C
:104A400026608DF827B009F007FB204639464FF461
:104A500080430DF11008ADF824308DF826608DF8F4
:104A600027A009F0F9FA4FF48273002402224FF4D0
:104A7000007C012548464146ADF812304FF008034E
:104A8000ADF81620ADF81AC00392CDF808C0ADF805
:104A90001C30ADF81040ADF81440ADF81850ADF82A
:104AA0001E40ADF8204009F071FF4846294609F044
:104AB000A9FF29464FF4805009F0D6FE09F5504968
:104AC0002846214609F058FB484639464FF0A003D6
:104AD000ADF824308DF827B08DF8266009F0BCFAC7
:104AE000484639464FF04003ADF824308DF8266033
:104AF0008DF827A009F0B0FA039ADDF808C04FF44A
:104B000082734146ADF812300E484FF02803ADF8DD
:104B10001620ADF81AC0ADF82040ADF81040ADF841
:104B20001440ADF81850ADF81C30ADF81E4009F037
:104B30002DFF0448294609F065FF0BB0BDE8F08F52
:104B4000000C01400030014000380040014B187853
:104B5000704700BF2C0200202DE9F8450546144699
:104B60000F4600295FD000285DD081425BD0022A29
:104B700094BF0026012601D8510101E0D11E490150
:104B800041F00601C9B2304607F032FB022C8246E2
:104B900001D8610101E0E11E490141F00C01C9B2F7
:104BA000304607F025FB804628460DF00BF90546F8
:104BB00038460DF007F9014628460DF00FFA074672
:104BC00050460DF0FFF839460DF008FA0DF018FBCD
:104BD000054640460DF0F6F839460DF0FFF90DF0A8
:104BE0000FFB1249002814BF80464FF001083846D9
:104BF000002D08BF01250DF0DBFA18B14146204613
:104C000007F0E4FD022C01D8610101E0E11E490139
:104C100041F00601C9B230462A4607F0B1FB044B09
:104C2000E41801232371BDE8F88500BF0000A0410E
:104C30002C02002010B5114B0446C3181B79DBB1C0
:104C4000022801D8410101E0C11E49010C4B41F08D
:104C5000060153F82420022C94BF00200120C9B281
:104C600007F028FC074BE0B253F8241007F0AEFD24
:104C7000024BE4180023237110BD00BF2C0200205A
:104C8000A40D00208C09002013B59C4CA0780528A9
:104C900000F2C4836378A32B00F009835BD8842BD4
:104CA00000F0D38028D8062B00F0428110D8022BC8
:104CB00000F0CB8006D8002B00F0AB80012B40F039
:104CC000A183ADE0042B00F0FB8000F21D81EEE03B
:104CD000802B00F09E8009D80C2B00F06B810D2BEF
:104CE00000F08581072B40F08D8341E1822B00F09D
:104CF0009B8100F2E58093E0932B00F0788114D83B
:104D0000872B00F09A8106D8852B00F0D080862B67
:104D100040F07883F8E08C2B00F0BE818D2B00F002
:104D2000C7818A2B40F06E8390E19A2B00F0388285
:104D300008D8952B00F0D181C0F03C81992B40F030
:104D40006183F9E1A12B00F0A88200F2AB82A02BD5
:104D500040F058839CE2B22B00F00C8327D8AA2B9A
:104D600000F0DF8211D8A62B00F0C18206D8A42B58
:104D700000F0A182A52B40F04583AAE2A82B00F009
:104D8000C7825E4B00F2C982BEE2AE2B00F0E08229
:104D900006D8AC2B00F0CD82584B00F2D582C4E28D
:104DA000B02B00F0DE82554B00F2E082D5E2C22B40
:104DB00000F0278215D8B72B00F0198308D8B52B3F
:104DC00000F0F38200F2FB82B32B40F01B83D5E2AC
:104DD000C02B00F0CD8000F20D82B82B40F0128382
:104DE0000BE3CC2B00F0308209D8C72B00F0A08059
:104DF000C82B00F01882C32B40F0048309E2D52BA6
:104E000000F03582D62B00F03982D42B40F0FA82A4
:104E100023E2022801D841010AE0C11E490107E04E
:104E2000022801D8410101E0C11E490141F00201FF
:104E3000324BC9B25A68DB78022894BF00200120A7
:104E400043EA022207F09CFAEBE2022801D8410172
:104E500001E0C11E4901294C41F00801E378626874
:104E6000022894BF00200120C9B243EA022207F0C1
:104E700021FBA078022801D8410101E0C11E4901AF
:104E80001E4C022894BF00200120E378626841F0A4
:104E9000060143EA0222002AB8BF5242C9B207F013
:104EA00009FB174AA378D31801221A71B9E2022824
:104EB00001D8410101E0C11E490141F00A01FFE0B2
:104EC000022801D8410101E0C11E49010B4C41F00B
:104ED0000601E3786268C9B243EA0222022894BF5D
:104EE0000020012007F0E6FAE2786068A37842EA41
:104EF0000020034A03499A1815E000BF6407002008
:104F00002C020020A40D0020984CE378616843EA4D
:104F1000012107F05BFCE2786068A37842EA002098
:104F2000934A94499A1841F823000023137178E2B8
:104F300005F012FA8D4B60B9DA78A72A05D899786E
:104F40008D4B03EB41135A7207E08C4B04221A700D
:104F500003E09B788A4A0121D154844B864A987891
:104F6000D978884B02EB40121B5C5172022B68E12E
:104F700005F0F2F97D4B60B9DA78A72A05D899785F
:104F80007D4B03EB41139A7207E07C4B04221A70AD
:104F900003E09B787A4A0121D154744B764A987881
:104FA000D978784B02EB40121B5C9172002B40F0D9
:104FB000388219E2022801D8410101E0C11E4901ED
:104FC00041F01401C9B2022894BF0020012001AAB7
:104FD00007F060F9654A9DF805305168D27852EAC9
:104FE000012114BF43F0020323F0020391E00228E1
:104FF00001D8410101E0C11E490141F01401C9B2CB
:10500000022894BF0020012001AA07F043F9574A63
:105010009DF805305168D27852EA012114BF43F05F
:10502000010323F0010374E0022801D8410101E0EB
:10503000C11E490141F0040142E0022801D84101AA
:1050400001E0C11E490141F00E0139E0022801D8FA
:10505000410101E0C11E490141F01401022894BF41
:1050600000200120C9B201AA07F014F93F4B98783B
:10507000DB78022801D8410101E0C11E490141F05D
:105080001401C9B2022894BF0020012001AA8DF8A2
:10509000063007F0E5FAC4E1344B374ADB7802EB1F
:1050A0004012C3F10801C9B2D37205F079FDB8E12D
:1050B000022801D8410101E0C11E490141F01A0155
:1050C0002A4BC9B25A68DB78022894BF002001201D
:1050D00043EA022207F0EEF9A3E1022801D84101D8
:1050E00001E0C11E490141F01401C9B2022894BF78
:1050F0000020012001AA07F0CDF81C4A9DF80530D8
:105100005168D27852EA012114BF43F0040323F01E
:1051100004038DF80530154B9878022801D8410119
:1051200001E0C11E490141F01401C9B2022894BF37
:105130000020012001AAACE7022801D8410101E0CA
:10514000C11E490141F01801022894BF002001202E
:1051500001AAC9B207F09EF8044A9DF8053090787C
:10516000D278022810D8410110E000BF6407002067
:105170002C0200208C090020A40E002080090020B1
:10518000D00F0020D80F0020C11E490141F01801A6
:1051900002F00F0223F00F03C9B242EA030321E039
:1051A000022801D8410101E0C11E490141F0180166
:1051B000022894BF0020012001AAC9B207F06AF8B2
:1051C000914A9DF805309078D278022801D84101A3
:1051D00001E0C11E490141F0180103F00F03C9B2FB
:1051E00043EA0213022894BF0020012001AA8DF88F
:1051F00005304EE7844B854ADB7802EB40100372A2
:105200000FE1E3786268400143EA02227F4BC2501B
:1052100007E17D4B7D495A68DB7801EB401043EA9A
:1052200002234360FDE0784B784AD978784B794C7B
:105230001B5C02EB40124FF0010C04F800C0032B82
:10524000D17740F0EE80CFE06268E3786F4943EABF
:10525000022301EB4010C381E3E06B4B6B495A68BA
:10526000DB7801EB401043EA02234361D9E0664B4F
:10527000664ADB7802EB40108377D2E0624B6349E9
:105280005A68DB7801EB401043EA02238383C8E0CD
:105290005D4BD97805F076FCC3E05B4BD97805F01F
:1052A00067FCBEE0584BD97805F026FBB9E0E17801
:1052B00005F016FBB5E004F07DFF534B20B9D9781B
:1052C000987805F0F5FAACE0D978987805F0C0FA4E
:1052D000A7E004F06FFF4C4B20B9D978987805F01F
:1052E000DBFA9EE0D978987805F09AFA99E004F014
:1052F00061FFE178A37818B9184605F0C1FA90E08B
:10530000184605F099FA8CE0D97805F0ADFA88E0F6
:105310003D4BD97805F09CF983E0D97805F08CF9FC
:105320007FE0E17805F07CF97BE0D97805F06CF955
:1053300077E0354CE17805F05BF9A178364BE278FF
:1053400003EBC1035A716CE0D97805F0EDF868E021
:1053500094F9031005F0DCF863E0D97805F0A2FBBE
:105360005FE0294BD97805F091FB5AE0D97805F038
:1053700081FB56E0E17805F071FB52E0234B03EB33
:10538000401308335A78A72A02D89B78A72B07D94D
:105390001D4B5968DB7843EA012101293ED101E028
:1053A000194BD97805F042FB3BE0174B17495A6877
:1053B000DB7801EB401043EA0223836131E01249BC
:1053C000154B4C68CA7842EA042243F8302022B9CF
:1053D00003EBC003597905F00BF90B4B0C4A987895
:1053E000125C012A1DD1D978FFF7A2F919E00A4A07
:1053F000E37802EBC000037113E0034BD97805F0AA
:1054000063FA0EE003220AE064070020A40E0020E5
:10541000D80F0020D00F0020E40D00200422014B03
:105420001A701CBD8009002013B5814B987805289F
:1054300000F2D9825B787F4CD62B00F2D182DFE874
:1054400013F0D700DE00EE00FB00040106010A01A4
:105450000F011401540170015E0128013D01CF02CA
:10546000CF02CF02CF02CF02CF02CF02CF02CF02B4
:10547000CF02CF02CF02CF02CF02CF02CF02CF02A4
:10548000CF02CF02CF02CF02CF02CF02CF02CF0294
:10549000CF02CF02CF02CF02CF02CF02CF02CF0284
:1054A000CF02CF02CF02CF02CF02CF02CF02CF0274
:1054B000CF02CF02CF02CF02CF02CF02CF02CF0264
:1054C000CF02CF02CF02CF02CF02CF02CF02CF0254
:1054D000CF02CF02CF02CF02CF02CF02CF02CF0244
:1054E000CF02CF02CF02CF02CF02CF02CF02CF0234
:1054F000CF02CF02CF02CF02CF02CF02CF02CF0224
:10550000CF02CF02CF02CF02CF02CF02CF02CF0213
:10551000CF02CF02CF02CF02CF02CF02CF02CF0203
:10552000CF02CF02CF02CF02CF02CF02CF02CF02F3
:10553000CF02CF02CF02CF02CF02CF02CF02CF02E3
:10554000CF02D700DE0085010401EE00FB0006015A
:105550008E01CF02CF029701CF02AA01AF01CF0285
:10556000CF02CF02CF02CF023D012801C101CF02FD
:10557000CF02CF02D601EB015E0170011401CF0210
:10558000CF025C025F02620265026802750283025A
:1055900090029302960299029C029F02A402A70223
:1055A000AB02AE02B102B402B702BA02BD02C2023D
:1055B000C602CC02CF02CF02CF02CF02CF02CF026F
:1055C000CF020F01FF01040208020D020F02CF02F9
:1055D0000A011102CF02CF02CF021602CF021B0234
:1055E0001D023402CF02CF02CF024D0252025702F7
:1055F000022801D841010AE0C11E490107E0022842
:1056000001D8410101E0C11E490141F00201C9B2C6
:10561000022894BF0020012006F0EAFDCFE0022816
:1056200001D8410101E0C11E490141F00801BFE07C
:105630006407002080090020022801D8410101E010
:10564000C11E490141F00A01B2E0994B00E0994BBB
:1056500053F82030BFE1984B03EB4010437ABAE196
:10566000954B03EB4010837AB5E1022894BF0020EC
:10567000012006F08FFC914B9B78022B88BF033BE7
:105680005B00012212FA03F303420CBF0022012245
:1056900028E0022801D8410101E0C11E490141F082
:1056A000140101AAC9B2022894BF0020012006F00B
:1056B000F1FD9DF80520C2F3400213E0022801D855
:1056C000410101E0C11E490141F0140101AAC9B222
:1056D000022894BF0020012006F0DCFD9DF8052083
:1056E00002F00102764B5A6080E10228744C01D826
:1056F000013000E00230C0B2FEF7BEFF22E17C21A3
:10570000022894BF0020012001AA06F0C3FD6B4BC4
:105710009DF806209B78022B88BF033B5B0002218B
:1057200010E07C21022894BF0020012001AA06F08D
:10573000B1FD624B9DF806209B78022B88BF033B8E
:105740005B00012111FA03F313429EE7022801D8FE
:10575000410101E0C11E490141F0040128E0022895
:1057600001D8410101E0C11E490141F00E011FE0D5
:10577000022801D8410101E0C11E490141F0140194
:1057800001AAC9B2022894BF0020012006F082FDC0
:105790009DF80620A6E704F0EBFCC0F10800D1E07C
:1057A000022801D8410101E0C11E490141F01A015E
:1057B000C9B2022894BF0020012006F053FD404BDF
:1057C000586013E1022801D8410101E0C11E4901DE
:1057D00041F0140101AAC9B2022894BF002001209F
:1057E00006F058FD9DF80520C2F380027AE70228F2
:1057F00001D8410101E0C11E490141F0180101AA8F
:10580000C9B2022894BF0020012006F043FD9DF894
:10581000052002F00F0265E7022801D8410101E0EE
:10582000C11E490141F0180101AAC9B2022894BF62
:105830000020012006F02EFD9DF80520120951E7F9
:105840001D4B03EB4010037AC5E01B4B4001C358CE
:10585000C1E0194B03EB40104368BCE0194BF7E67D
:10586000194BF5E6144B03EB4010C37FB3E0124B2A
:1058700003EB4010C389AEE0144BE9E6144B002261
:105880001B5C626013B10E4B01325A60114B104A1F
:105890001B5C0021115423B1094B5A6842F00202EB
:1058A0005A600C4B00221A54A0E00B4B84E000BF5E
:1058B000A40D00208C090020A40E00206407002005
:1058C00080090020C00D0020680F00202C0E002051
:1058D000900E00201C0E0020980E00204C4B03EB75
:1058E0004010436977E04A4B03EB4010837F72E03E
:1058F000474B03EB4010838B6DE004F041FC21E04B
:1059000004F046FC1EE004F04BFC1BE004F052FCEB
:1059100018E004F04FFC3F4C3F4B18B9987804F066
:105920005DFC0FE0987804F081FC0BE004F042FC91
:10593000384C394B18B9987804F05AFC02E0987842
:1059400004F088FC606051E004F034FC314C324BD0
:1059500018B9987804F056FCF4E7987804F070FCD5
:10596000F0E704F059FCEDE704F07EFCEAE704F010
:1059700085FCE7E704F08CFCE4E704F093FCE1E746
:10598000264B03EBC000437925E004F09FFCD9E7E8
:1059900004F0A6FC40B2D5E704F0B6FCD2E704F070
:1059A000BBFCCFE704F0C0FCCCE704F0C5FCC9E7C2
:1059B00004F0D2FCC6E71A4B1B5C0CE0144B03EB63
:1059C0004010836907E0154B53F8303003E0134B68
:1059D00003EBC0000379636008E004F0F5FBB1E776
:1059E0000323237002E00B4B04221A700D4B1B782B
:1059F0006BB1084B0C495A680C4B0A601AB91A680B
:105A000042F0080202E01A6822F008021A601CBD87
:105A1000A40E00208009002064070020E40D00206F
:105A2000DC0D00207A090020680900206C070020A6
:105A300008B5754B9878052801D90422E0E05B7819
:105A40009A2B20D8992B74D2822B63D00BD8062B9B
:105A500044D003D8042B3BD0052B0AE0072B4AD0B7
:105A60000C3B012B0CE08C2B56D005D8832B2FD070
:105A7000862B40F0C4802DE08D2B58D0933B022B19
:105A800000F2BD8044E0C72B28D00ED8C12B5DD0DA
:105A900005D8B52B4FD0C02B40F0B1802BE0C22BE6
:105AA00065D0C32B40F0AB8067E0D22B7DD005D80A
:105AB000C82B6AD0CC2B40F0A2806BE0D52B00F035
:105AC0008680D62B00F08E80D42B40F0988072E038
:105AD000062100E00C2106F029FC93E04B4A43012B
:105AE0000833D31803EB401102EB401001F14102DF
:105AF000101A597838E0454A43010833D31803EBAC
:105B0000401102EB401001F14202101A99782BE08B
:105B10001421E0E70421DEE73C4B821C03EB40113B
:105B20000B3103EB401001EB4213181A58E01A2115
:105B3000D1E71821CFE74301344A03F11801511886
:105B40000230D31801EB4010C01A3EE02F4B820008
:105B5000013200F1020C03EBC20101EB4C1103EB2B
:105B60004010081A13F8321003F072F84AE027497F
:105B7000831C01EB4011580127E0244A831C02EBEF
:105B80004010011D01EB43131EE0204A4301991808
:105B90001F3120E01D4B821C03EB40110E3103EB43
:105BA000401001EB4213181A25E0184B4101103147
:105BB0005918821C04E0154B821C03EB4011143170
:105BC00003EB401001EB4213181A042214E00F4AB1
:105BD000430199181E310230D31801EB4010C01A4E
:105BE000012209E0094A430199181C310230D318F7
:105BF00001EB4010C01A022202F0ACFF02E00322C7
:105C0000034B1A7008BD00BF64070020A40E0020DB
:105C10008009002038B59B4DA878052801D90422B9
:105C20002CE16B78952B21D8932B80F0A8800D2B3D
:105C30000BD80C2B80F0A380052B5FD001D8042B50
:105C40000AE0062B7DD0072B23E0862B56D006D802
:105C5000822B00F09680832B40F00F8130E08C2B5C
:105C600000F093808D2B40F00881A5E0C32B00F05D
:105C7000C88011D8B52B00F0A38004D8993B012B24
:105C800000F2FB809AE0C12B00F0A58000F2B38007
:105C9000C02B40F0F28063E0CC2B00F0BF8005D831
:105CA000C72B4ED0C82B40F0E880B2E0D52B00F0D7
:105CB000CC80D62B00F0D480D42B40F0DE80B8E02E
:105CC000062106F057FD6F4B9C78022C01D861012C
:105CD00001E0E11E490141F00601C9B2022C94BF66
:105CE0000020012006F0BEFA664B674A9B78D31865
:105CF000664A42F8240000221A71C1E00C2106F025
:105D000039FD604B9C78022C01D8610101E0E11E55
:105D1000490141F00C01C9B2022C94BF00200120BE
:105D200006F0A0FA574B5A4A9B78574942F824008C
:105D300018465B1852F8201000221A7106F046FD32
:105D40009EE0544B440108341C1904EB401203EB51
:105D5000401002F14103181A02F0E4FE60708FE077
:105D60004C4B440108341C1904EB401203EB401067
:105D700002F14203181A02F0D5FEA07080E014214F
:105D800000E0042106F0F6FC7AE0424C831C04EBB0
:105D900040110B3101EB431304EB4010181A0122A0
:105DA00002F09CFEA87804EB4014E17AC1F10801EE
:105DB000C9B204F0F5FE63E01A21E3E71821E1E738
:105DC0004301344A03F1180151180230D31801EB92
:105DD0004010C01A37E02F4C85000135821C04EBBF
:105DE000C50303EB421304EB4010181A02F09AFEAD
:105DF00004F8350044E02749831C01EB40115801A9
:105E000021E0244A831C02EB4010011D01EB4313E7
:105E100018E0204A430199181F311AE01D4B821CDB
:105E200003EB40110E3103EB401001EB4213181A43
:105E30001FE0184B821C03EB4011143103EB4010A0
:105E400001EB4213181A042214E0124A4301991874
:105E50001E310230D31801EB4010C01A012209E0B4
:105E60000C4A430199181C310230D31801EB401041
:105E7000C01A022202F032FE02E00322064B1A7020
:105E800038BD00BF640700202C020020A40D0020B4
:105E90008C090020A40E0020800900204A49F8B592
:105EA00000230B6049494A4A0B604A4993750B60CD
:105EB000D360136113755375474A4FF0FF3142F8B1
:105EC0002310464A0025D55401332F2BF4D1FD264B
:105ED0002C46022C94BF0027012701D8610100E065
:105EE000710141F00601C9B2384606F081F961013D
:105EF000022C88BF71013A4B41F00C01E850C9B245
:105F0000384606F075F9374B01340136E850043550
:105F1000062CF6B2DDD1344D0024E97AE0B2C1F1AD
:105F20000801C9B2013404F03BFE2035062CF4D13F
:105F300000232E4A002199500433B3F5806FF8D125
:105F40002B4B9B7EABB14FF4C3640DE0384631461A
:105F50000422013502F0C2FD04370436062DF5D1C6
:105F60001834B4F5FF6F04D0224E274636190025A9
:105F7000ECE71F4BDB7E5BB94FF4A7641E4920465C
:105F800009190422043402F0A9FDB4F5C36FF5D158
:105F9000174B1B79012B03D0112B01D0212B01D1E1
:105FA000012200E000220A4B83F8D420104B5B7DD5
:105FB00023B1FEF731FB08B1012200E00022044BBF
:105FC00083F8D520F8BD00BF6809002088090020AB
:105FD0002C0200206C07002044020020F40F002057
:105FE000A40D00208C090020A40E0020A40900208C
:105FF00004000020700100206C04002008B50B4B49
:106000005A7892B9997881B95A68DB7843EA0222C2
:1060100040F2D2439A4208D140F2FF7002F018FEDB
:1060200002F0DAFE0120FEF77BFB08BD64070020CA
:1060300010B5964A9378022B00F05F81032B00F095
:106040006581002B40F06E8253784D2B00F0B780B5
:1060500023D8452B70D00ED8422B56D005D8402BD4
:1060600045D0412B40F05C8246E0432B53D0442B7B
:1060700040F0568256E0482B7CD005D8462B61D0A4
:10608000472B40F04D826AE04B2B00F0858000F2F8
:106090008F80492B40F0448272E0542B00F0E9805D
:1060A00011D8512B00F0B68006D84F2B00F08D8010
:1060B000502B40F03582A6E0522B00F0BD80532BD0
:1060C00040F02E82C2E0832B00F0FA8006D8552BD8
:1060D00000F0E280572B40F02382EAE0852B00F0AD
:1060E000FF80C0F0F580FF2B40F01A8201E1674B82
:1060F00040F2FF70D97805E0644B654ADB780020F8
:106100001946137002F0A4FD0FE2D378604A1946D5
:1061100001205370F6E75D4B5D4ADB780420194699
:106120001371EFE7594B5A495A68DB781C2043EA50
:10613000022341F81C3F0EE0D378554A194605204A
:106140005371DFE7514B52495A68DB780C2043EA20
:10615000022341F80C3F042202F0FCFCE5E14B4B2A
:106160004B4C5A68DB78214643EA022341F8083F4A
:10617000082075E0D3784649262001F8263F83E0C1
:10618000424A434BD27812B1424901224A60DA7541
:106190003F4B1720D97DB5E73C4B3D4CDB780320C6
:1061A0001946E37002F054FDE07802F035FFBCE1DF
:1061B000364B374ADB78022019469370A2E7D37832
:1061C000334A1946152053759CE7304B304CDB7829
:1061D00019201946637602F03BFD607E10F0010045
:1061E00002D00020012100E0014606F051F9284BC1
:1061F000597E11F0020102D00120014600E0012089
:1062000006F046F991E1214B214ADB781620194628
:10621000937577E71E4B1B7D13F0010F05D0D378E4
:1062200013F0010F01D102F0D7FD184B184ADB78AB
:1062300014201946137565E7144B15495A68DB7825
:10624000202043EA022341F8203F84E70F4B104C03
:106250005A68DB78214643EA022341F8103F1020B8
:10626000042202F077FC22696079A16803F036F914
:106270005BE15168D37843EA0122012A00F252819E
:1062800003491A2001F81A3F012265E7640700203C
:1062900004000020800900208E4B5A68DB7843EA16
:1062A0000222012A00F23E818B491B2001F81B3F8C
:1062B000EAE7884B8849DB78272001F8273FE3E7A6
:1062C000D378516843EA0122844BC3F8D8202CE1EB
:1062D000804B5A68DB7843EA0222814B1A6024E142
:1062E0007C4B5A68DB7843EA02227C4BC3F8DC2003
:1062F0001BE1784BDA787B4B16E1D3785168527802
:1063000043EA0121784B43F822100EE153782E2BFB
:1063100000F20681DFE813F02F003C004900040181
:106320000401040104010401040156005E0066003A
:106330006E0076007E0004010401040104010401E2
:1063400004010401040104010401040104018600A4
:1063500089008C008F009200950098009B009E00A1
:10636000A100A400AD00B600BE00C600CE00D6005D
:10637000EC00F400FC00574B5A68DB7843EA022239
:106380005A4B1A6003F036FB544BC3F8E000CCE0E4
:10639000504B5A68DB7843EA0222544B5A6003F0B0
:1063A00029FB4E4BC3F8E400BFE04A4B5A68DB7848
:1063B00043EA02224D4B9A6003F01CFB474BC3F8A3
:1063C000E800B2E0434B5A68DB7843EA0222474BCD
:1063D000DA60AAE03F4B5A68DB7843EA0222434B7B
:1063E0001A61A2E03B4B5A68DB7843EA02223F4B3A
:1063F0005A619AE0374B5A68DB7843EA02223B4BFA
:106400009A6192E0334B5A68DB7843EA0222374BB9
:10641000DA618AE02F4B5A68DB7843EA0222334B79
:106420001A6282E02B4B00201CE02A4B002022E065
:10643000284B012016E0274B01201CE0254B0220B1
:1064400010E0244B022016E0224B03200AE0214BEF
:10645000032010E01F4B042004E01E4B04200AE040
:106460001C4B05205968DB7843EA012106F048F906
:106470005BE0184B05205968DB7843EA012106F000
:1064800003F952E0134B5A68DB7843EA0222174BB8
:106490005A624AE00F4B5A68DB7843EA0222134BF8
:1064A0009A6242E00B4B5A68DB7843EA02220F4BB8
:1064B000DA623AE0074B5A68DB7843EA02220B4B78
:1064C0001A6332E0034B5A68DB7843EA0222074B37
:1064D0005A632AE064070020040000202C020020F8
:1064E0007C09002079090020A4090020800F0020E9
:1064F0000E4B5A68DB7843EA02220D4B9A6314E094
:106500000A4B5A68DB7843EA0222094BDA630CE053
:10651000064B5A68DB7843EA0222054B1A6404E012
:10652000032200E00422034B1A7010BD6407002010
:10653000800F00208009002010B5774B9A78022A3E
:1065400000F0BB80032A00F0BF80002A40F04281A7
:106550005B78502B71D022D8462B55D00ED8422BC9
:1065600048D005D8402B3CD0412B40F0A4803FE0E0
:10657000442B44D0694C6A4B44D83EE04B2B50D05E
:1065800006D8482B46D042D3492B40F0948045E0B2
:106590004D2B4CD048D34F2B40F08D804AE0812BBF
:1065A00061D010D8542B50D006D8522B4AD05B4C17
:1065B0005B4B00F2C98043E0572B4CD0802B4ED070
:1065C000552B78D144E0852B5DD004D8832B54D053
:1065D000524C56D84FE0FE2B64D066D8F02B6AD1CF
:1065E00060E040F2FF7002F09DFA4C4B5860F4E01E
:1065F0004B4B58E04A4B5A7863E01B7987E0484B95
:10660000DA695EE05B7982E0454BDA6859E0444B39
:106610009A6856E0424B93F8262052E0404BDA7DD0
:1066200045E03F4BDA784CE03D4B9A7849E03C4BF3
:106630005A7D46E03A4B5A7E43E0394B9A7D40E022
:106640001B7D64E0364B1A6A3BE0354B9A7E38E09E
:10665000334BDA7E35E0324B93F8272031E0314B73
:1066600093F8D5202DE02F4B93F8D520042A14BFA2
:106670000022012225E02B4B63E02A4BD3F8D820DF
:106680001FE0294B3FE0274A284BD2F8DC104B4350
:1066900003F540533933214923F000404860C2F8E4
:1066A000DC309AE0224B1A780BE0224B1A78003A41
:1066B00018BF012205E003228DE05A781E4B53F8E3
:1066C0002220164B5A6088E05B78144C2E2B7ED823
:1066D000DFE803F0181B1F7D7D7D7D7D7D36393C15
:1066E0003F42457D7D7D7D7D7D7D7D7D7D7D7D48C0
:1066F0004A4C50525456585A5C5E6065686B6E71D5
:1067000074777A000D4B1B6801E00C4B5B6863608B
:1067100063E00A4B9B68FAE76407002080090020C9
:10672000040000202C0200207C0900206D4EC64190
:10673000C80F002079090020A4090020800F002044
:106740002F4BDB68E3E72E4B1B69E0E72C4B5B69C3
:10675000DDE72B4B9B69DAE7294BDB69D7E7284B51
:106760001B6AD4E7002002E0002014E0012005F0BD
:10677000C1FD12E001200EE00220F8E702200AE04D
:106780000320F4E7032006E00420F0E7042002E001
:106790000520ECE7052005F093FD60601DE0184B37
:1067A0005B6AB4E7164B9B6AB1E7154BDB6AAEE751
:1067B000134B1B6BABE7124B5B6BA8E7104B9B6B50
:1067C000A5E70F4BDB6BA2E70D4B1B6C9FE7032389
:1067D000237002E004220B4B1A700B4B1B786BB139
:1067E000084B0A495A680A4B0A601AB91A6842F0FB
:1067F000080202E01A6822F008021A6010BD00BF09
:10680000800F0020800900207A09002068090020FC
:106810006C07002010B51C4CA078052830D8637890
:10682000012B23D003D3022B184C26D121E004F0F6
:10683000EBFEA178164A0023994208D0144C907FB1
:1068400004EB411468B194F81EC0844509D1114885
:106850004FF0010C00F803C00F480CF1FF3C03F8A7
:1068600000C001332032062BE6D10CE004F0D4FE48
:1068700009E004F0D9FE606005E00323237002E024
:10688000024B04221A7010BD64070020800900200A
:10689000A40E0020300200201C0E002037B5584BFB
:1068A0001A7DA2B957494868CA7842EA0022B2F173
:1068B000FF3F04BF544A12680A214A43C3F8EC2040
:1068C00003F098F84E4B01221A75C3F8F0004D4BB7
:1068D0005B78042B00F29280DFE803F00335465921
:1068E000130003F087F8464BD3F8F010D3F8EC20F0
:1068F000411A0029B8BF494291427CD900221A7539
:106900007CE0404B3E4C987804F08EFE30B93F4A14
:106910002075136823F0100313606FE0D4F8EC3097
:10692000002B67D003F066F8D4F8F020D4F8EC30F0
:10693000821A002AB8BF52429A425BD9334B0021D7
:106940001A68217552E02F4CA078022894BF0020CD
:10695000012005F01FFBA378022B88BF033B5B00DF
:1069600001259D40054026E0264C7C21A07801AA07
:10697000022894BF0020012005F08CFCA3789DF82C
:106980000620022B88BF033B5B00022511E01D4C53
:106990007C21A07801AA022894BF0020012005F0E4
:1069A00079FCA3789DF80620022B88BF033B5B008F
:1069B00001259D401540124C06D0144B00211A6849
:1069C000217522F0100213E0D4F8EC3093B103F0FB
:1069D00011F8D4F8F020D4F8EC30821A002AB8BFAD
:1069E00052429A4206D9094B25751A6842F01002A4
:1069F0001A6003E0024BDA68013ADA603EBD00BF7C
:106A00002C02002064070020680900206C07002089
:106A100008B5184B9A7812B1022A26D106E05868B8
:106A2000DB7843EA0020FDF7A3FD21E05878072832
:106A30000AD85A68DB7853EA022202D1FDF7EAFC51
:106A400016E0FDF703FD13E0FF280CD15868DB7852
:106A500043EA0020B0F1FF3F0ABF074BC0B21878ED
:106A6000FDF710FD04E0032200E00422034B1A703E
:106A700008BD00BF640700206809002080090020CD
:106A800010B51F4B9A78012A1CD003D3022A1D4C43
:106A900021D11BE05878082802D8FDF7EDFD0EE063
:106AA0000A2803D1174B00225A6016E00B2802D1A6
:106AB000FDF7CAFD03E0FF280FD1FDF713FE114BD0
:106AC00058600AE0587802F0B1FFF8E75878FDF70F
:106AD000EDFC606001E0042323700B4B1B786BB16D
:106AE000084B0A495A680A4B0A601AB91A6842F0F8
:106AF000080202E01A6822F008021A6010BD00BF06
:106B000064070020800900207A090020680900201D
:106B10006C07002010B5224B5A78812A3FD19A7811
:106B2000922A3CD19A79A32A39D15A79B42A36D1FA
:106B30001A79C52A33D1DB78D62B30D1194B4FF4D3
:106B400000725A61A2F5A07203F580631A6103F026
:106B50008BFA02F04FFF044602F04CFF001B0028A6
:106B6000B8BF4042B0F57A7FF6DBFDF7FFFC07F0D7
:106B7000A7FB002008F0D4F800210B4806F056FFD0
:106B8000094806F0B3FE094806F06EFB06F09EFFCA
:106B90004FF0804008F048FE0020FDF7C1FD10BD19
:106BA0006407002000080140080002400024014062
:106BB0002DE9F047A84CA94DE0786268237864215C
:106BC00040EA0220222B86B029706B70686001F0C9
:106BD000128057D80F2B00F0898426D8072B00F09D
:106BE000388410D8032B00F05F8106D8012B00F009
:106BF000A980022B41F06F82F5E0052B00F0218483
:106C000000F223848FE10B2B00F0338406D8092B8C
:106C100000F0278400F2298400F01FBC0D2B00F047
:106C20005D8400F25F8400F03DBC192B00F0088603
:106C300013D8152B00F0048507D8132B00F05A84C5
:106C4000142B41F0488200F0CDBC172B00F0D68504
:106C5000834B00F2E78500F0C9BD1E2B00F02D86A6
:106C600009D81B2B00F01F86C0F008861C2B41F0B2
:106C7000328200F01CBE202B00F0D78600F2658720
:106C800000F079BE812B01F07A802ED8412B01F0E3
:106C90004A8015D8252B00F0F48707D8232B00F065
:106CA000B687242B41F0178200F0BDBF272B01F0DF
:106CB0001F80C0F0F187402B41F00D8201F030B809
:106CC000452B01F03C8006D8432B01F0328001F2C5
:106CD000338001F02BB8472B01F03780C1F03280B0
:106CE000802B41F0F88101F045B8882B01F0D88065
:106CF00012D8842B01F07D8007D8822B01F05780B9
:106D0000832B41F0E88101F057B8862B01F08B808E
:106D100001F2E68001F082B88C2B01F02B8106D8BD
:106D20008A2B01F00E8101F2208101F007B9F22BCC
:106D300001F0C081FF2B01F0C0818D2B41F0CB8190
:106D400001F063B9A378052B48D8464EFD250024F1
:106D5000414B9B789C4208D0424A02EB43139B7FF5
:106D6000002B33D0B27F9A4230D13F4A4FF001011D
:106D700011553E4A0023A354022C3D4A94BF0027DC
:106D800001278CBF2946E1B2A3543846022205F000
:106D900001FA022C01D8610100E0690141F006010D
:106DA000C9B2384640F2FF7205F084FB022C01D8CC
:106DB000610100E06901284B41F008015A68DB7865
:106DC000C9B2384643EA022205F074FB01340135AA
:106DD0002036062CEDB2BBD101F080B91F4B042246
:106DE0001A7001F07BB91C4B9B78052B57D81D4EB0
:106DF000FD250024184B9B789C4208D0194A02EBD1
:106E000043139B7F002B42D0B27F9A423FD1164A58
:106E10004FF001011155154A0023A354022C144AC6
:106E200094BF002701278CBF2946E1B2A3543846FE
:106E3000022205F0AFF9022C01D8610100E06901DE
:106E400041F00601C9B2384640F2FF7205F032FB4C
:106E5000022C0FD861010EE0640700208009002099
:106E60002C020020A40E0020300200201C0E002066
:106E7000900E00206901954B41F008015A68DB78BB
:106E8000C9B243EA02223846524205F013FB0134EC
:106E900001352036062CEDB2ACD101F01FB98C4B78
:106EA00004221A7001F01AB9A378052B37D8894E3D
:106EB000FD250024854B9B789C4207D0854A02EB38
:106EC00043139B7F1BB3B27F9A4220D1824A002397
:106ED000A354824AE7B2A354384604F09DFB022C27
:106EE00094BF4FF000084FF001088CBF2946394687
:106EF0004046022205F04EF9022C01D8790100E04B
:106F0000690141F00801C9B2404605F0E7FA0134D1
:106F100001352036062CEDB2CCD101F0DFB80423C8
:106F20002B7001F0DBB8694B9878052803D95B78A2
:106F3000022B40F08182654B5B78032B00F2778255
:106F4000DFE813F004006700F4003F02FDF772FE73
:106F50005E4B624A9878002313545F4A0228135408
:106F600001D8410101E0C11E4901584C022894BFDB
:106F700000200120E3786268C9B243EA022205F0EA
:106F8000FFF9A078022801D8014601E0C11EC9B26C
:106F9000022894BF00200120002205F0FBF84B4B93
:106FA0004C4E9B7806EB43139B7F002B01F09680A1
:106FB000FD250024454B474A9B789C4202EB431237
:106FC0001FD0937FB27F9A421BD12046FDF732FE3D
:106FD000022C94BF0027012701D8610100E069015C
:106FE0003A4BC9B25A68DB78384643EA022205F0C8
:106FF000C7F9022C8CBF2946E1B23846002205F0C1
:10700000C9F8013401352036062CEDB2D2D101F099
:1070100065B8FDF70FFE2D4B304A987800231354C6
:107020002D4A0228135401D8410101E0C11E490133
:1070300041F00201022894BF00200120C9B205F0EE
:10704000D7F8224BDA785C689B7842EA042404196A
:10705000022B01D8590101E0D91E4901022B94BF2E
:1070600000200120C9B2224605F08AF9174B987812
:10707000022801D8014601E0C11EC9B2002202283F
:1070800094BF0020012005F085F8104B114E9B782D
:107090000F4A06EB43139B7F5460002B01F01E80C8
:1070A000FD250024094B9878844237D0094BB27FE4
:1070B00003EB40139B7F9A4230D1FDF7BBFD022CBE
:1070C00094BF002701270BD861010AE06407002064
:1070D00080090020A40E00201C0E0020900E00202D
:1070E000690141F00201C9B2384605F081F88C4BC4
:1070F000022C5A68DB7843EA022301D8610100E0E0
:107100006901C218C9B2384605F03AF9022C8CBFA1
:107110002946E1B23846002205F03CF80134013539
:107120002036062CEDB2BDD100F0D8BF10F0C0055E
:1071300039D1052832D87A4EF378726843EA0223AF
:10714000142B2BDC062202FB0303764A52F8234061
:10715000FDF770FDB078744B02281D54734B1D541D
:1071600001D8410101E0C11E4901022894BF00205D
:107170000120C9B2224605F003F9694B987802282C
:1071800001D8014601E0C11EC9B2022894BF002007
:107190000120002204F0FEFF00F0A0BF644B042297
:1071A0001A7000F09BBF402D40F0C4805C4B5F68BC
:1071B000DB7843EA0727142F00F3AD8000231C4639
:1071C00000930193029350FA03F10DF1180C11F0A2
:1071D000010F0CEB040204D00134032C02F80C3C28
:1071E00002D00133062BEED1002621E003AB9D5DDA
:1071F0002846FDF71FFD022D01D8690101E0E91EB7
:10720000490141F00201022D94BF00200120C9B2C2
:1072100004F0EEFF062303FB0755424B6A4653F882
:107220002530C31A002BB8BF5B4242F82630013626
:10723000A642DBDB012C0ADD022C10D1009B019958
:107240008B4207DD18469DF80D20FDF785FCFD25D6
:1072500000242DE008469DF80C201946F5E7032C84
:10726000F5D1009E019D029CAE420DDDA64207DDD8
:10727000304629469DF80D20FDF76EFC30460CE0A7
:1072800031469DF80C200DE0A5429DF80C2008DD4C
:1072900028463146FDF760FC284621469DF80E2021
:1072A000D3E731462046FDF757FC20462946CAE77A
:1072B0001B4A937853FA04F111F0010F4FF00001CB
:1072C00022D05068D278022C42EA00204FF0060209
:1072D00002FB0040154A94BF00260126D154114AF2
:1072E00052F820201048C15401D8610100E0690122
:1072F000C9B2304605F044F8022C8CBF2946E1B2F1
:107300003046002204F046FF01340135062CEDB270
:10731000CED100F0E3BE064B04221A7000F0DEBEB0
:1073200064070020700700201C0E0020900E002033
:1073300080090020802D40F0D1869F4B5A68DB7871
:1073400043EA0223142B37DC7D3500249A4EB378B0
:10735000234113F0010F28D0F3787268204643EAE6
:107360000222062303FB0242944B53F82270FDF7DE
:1073700061FCB37892494FF00002CA549149022C43
:10738000CA5494BF0026012601D8610100E06901BA
:10739000C9B23A46304604F0F3FF022C8CBF2946AE
:1073A000E1B23046002204F0F5FE01340135062C2E
:1073B000EDB2CBD100F092BE834B04221A7000F0E4
:1073C0008DBE10F0800F40F089867B4DEB786A68A7
:1073D00043EA0222062303FB0202784B53F82240C1
:1073E000FDF728FCA878764A00231354754A022832
:1073F000135401D8410101E0C11E4901022894BF84
:1074000000200120C9B2224604F0BAFF6A4B9878E6
:10741000022801D8014601E0C11EC9B2022894BF6A
:1074200000200120002204F0B5FE00F057BE664B9C
:1074300003221A7000F052BE634B04221A7000F04F
:107440004DBEFDF721FC00F049BEFDF7EDFF00F059
:1074500045BEFEF7EDFA00F041BEFEF7DBFB00F0A3
:107460003DBEFEF7E5FD00F039BEFFF765F800F020
:1074700035BEA378022B11D16378372B0AD8534934
:1074800003F5A77001EB83018000042201F062FB89
:1074900000F024BE03232B7000F020BE04232B70C9
:1074A00000F01CBE444B9A78022A12D15B78372B2D
:1074B0000AD8464903F5A77001EB83018000023228
:1074C00001F00CFB00F00ABE3F4B03221A7000F0E3
:1074D00005BE3D4B04221A7000F000BEFFF79AF97A
:1074E00000F0FCBDFFF794FA00F0F8BDFFF7C8FA12
:1074F00000F0F4BD6278364B092A53D8DFE802F079
:10750000050D151D26313941494C2B4A1968506823
:10751000D27842EA0022521843E0274A196850689C
:10752000D27842EA00228A1A3BE0234A196850685E
:10753000D27842EA00224A4333E01F4A1968506871
:10754000D27842EA002291FBF2F22AE01A48196846
:107550004468C27842EA042291FBF2F002FB101266
:107560001FE0154A19685068D27842EA00220A40A2
:1075700017E0114A19685068D27842EA00220A439B
:107580000FE00D4A19685068D27842EA00224A405A
:1075900007E01A68D24304E0074A5168D27842EA09
:1075A00001221A600A4A0B4B1268AAB91A6842F003
:1075B00008021A6000F092BD6407002070070020E6
:1075C000900E00201C0E002080090020A40900203D
:1075D000680900206C0700201A6822F008021A606F
:1075E00000F07CBDA04BA14A5968DB78126843EAE1
:1075F00001239A4206DD9E4B1A6842F0040222F0F3
:1076000003020CE09A4B05D11A6822F0060242F000
:10761000010204E01A6822F0070242F002021A6036
:10762000924A934B12682AB91A6842F008021A600B
:1076300000F054BD1A6822F008021A6000F04EBD36
:1076400063780C2B00F24A85DFE813F00D001C0074
:107650002B003A004900580067007600850094002E
:10766000A300B200C100824B1B6813F0080F00F0AA
:1076700035857D4B5A68DB7843EA02227D4BDA6020
:1076800000F02CBD7A4B1B6813F0080F40F02685E4
:10769000754B5A68DB7843EA0222764BDA6000F0D9
:1076A0001DBD734B1B6813F0010F00F017856E4B67
:1076B0005A68DB7843EA02226E4BDA6000F00EBDB6
:1076C0006B4B1B6813F0010F40F00885664B5A683E
:1076D000DB7843EA0222674BDA6000F0FFBC644BC0
:1076E0001B6813F0040F00F0F9845F4B5A68DB78D5
:1076F00043EA02225F4BDA6000F0F0BC5C4B1B688F
:1077000013F0050F00F0EA84574B5A68DB7843EA20
:107710000222584BDA6000F0E1BC554B1B6813F0B5
:10772000020F00F0DB84504B5A68DB7843EA0222F8
:10773000504BDA6000F0D2BC4D4B1B6813F0030FC6
:1077400000F0CC84484B5A68DB7843EA0222494B6C
:10775000DA6000F0C3BC464B1B6813F0100F00F05A
:10776000BD84414B5A68DB7843EA0222414BDA6020
:1077700000F0B4BC3E4B1B6813F0200F00F0AE8449
:10778000394B5A68DB7843EA02223A4BDA6000F060
:10779000A5BC374B1B6813F0400F00F09F84324BA1
:1077A0005A68DB7843EA0222324BDA6000F096BC7A
:1077B0002F4B1B6813F0800F00F090842A4B5A68FF
:1077C000DB7843EA02222B4BDA6000F087BC284BBF
:1077D0001B6813F4807F00F08184234B5A68DB78A8
:1077E00043EA0222234BDA6000F078BC1E4A51685B
:1077F000D27842EA0122DA6000F070BC1D4B1A69AF
:10780000072A00F26B841849DC684868C97841EAA5
:107810000020511C03EB8202C2F8F440D8601961C9
:1078200000F05CBC1A69134B002A00F05784013A3F
:1078300003EB8201D1F8F4101A61D96000F04EBC5C
:1078400063782E2B04D80C4A0121D15400F046BC99
:10785000FF2B04D1074B01225A7500F03FBC0323D4
:107860002B7000F03BBC00BF6407002068090020BB
:107870006C0700202C020020F40F00208F4B5B7857
:107880002E2B04D88E4A0021D15400F027BCFF2BA8
:1078900004D18C4B00225A7500F020BC8A4B032285
:1078A0001A7000F01BBCFEF7F9FF00F017BC854B07
:1078B000002283F8D52000F011BC6378142B57D830
:1078C000A278052A20D8062101FB03237F4A804C99
:1078D000917E44F82300002900F00084774A537811
:1078E000002B00F0FB83917803F1FF3C062201F5A9
:1078F000C37002FB031302FB0C0204EB8301900034
:10790000042201F027F9E9E3FF2A2DD1B3B94FF49E
:10791000C3640EE0384631460422013501F01AF9FD
:1079200004370436062DF5D11834B4F5FF6F00F096
:10793000D583684E274636190025EBE700245F4BB8
:1079400006215B78624A581E01FB004001FB03419F
:1079500000F5C37002EB810180000422013401F0C4
:10796000F9F8062CEBD1B9E3574B04221A70B5E3B2
:1079700003232B70B2E36378142B52D84F4A9278CA
:10798000052A1AD8062101FB0323514951F8232067
:10799000514B4D491B784A60002B00F09F834F49A3
:1079A0004F4B0A6022B91A6842F008021A6095E348
:1079B0001A6822F008021A6090E3FF2A2DD1B3B9A9
:1079C0004FF4C3640EE0384631460422013501F01D
:1079D00085F804370436062DF5D11834B4F5FF6F59
:1079E00000F07C833B4E274636190025EBE7002448
:1079F000324B06215B78364A581E01FB004001FBE2
:107A0000034100F5C37002EB8101800004220134C0
:107A100001F064F8062CEBD160E32B4B04221A70C2
:107A20005CE3294B03221A7058E36578142D00F2A9
:107A30008880224B9C7814F0800F38D0FD250024DC
:107A40001E4B987850FA04F212F0010F14D0022C59
:107A50005E7801D8610100E0690141F00201C9B21C
:107A6000022894BF0020012004F0C2FB062303FB80
:107A70000646174B43F82600144B9B7E8BB10F4BE9
:107A80005B7873B10621581E01FB004001FB0341E6
:107A90000F4A00F5C37002EB81018000042201F05F
:107AA00059F801340135062CEDB2C9D116E3052C85
:107AB00043D8022C16D8610116E000BF64070020ED
:107AC000F40F00202C020020800900200400002078
:107AD00070070020700100207A090020680900204A
:107AE0006C070020E11E490141F00201C9B2022CDD
:107AF00094BF0020012004F07BFB062303FB054418
:107B00009349944A897E42F82400002900F0E682D5
:107B100091484178002900F0E182807801F1FF3E30
:107B200000F5C37C03FB010103FB0EC302EB8101E3
:107B30009800042201F00EF8D0E2884B04221A705B
:107B4000CCE2864B03221A70C8E26278844B0A2A80
:107B500043D8DFE802F0060B11161C242A30363A0F
:107B60003D0080491A6809688A1803E07D4A19684F
:107B700012688A1A1A6030E07A4A196812684A4311
:107B8000F8E7784A1968126891FBF2F2F2E7754A51
:107B90001968126891FBF2F002FB1012EAE77149D2
:107BA0001A68096801EA0202E4E76E491A6809687E
:107BB00041EA0202DEE76B491A68096881EA0202BB
:107BC000D8E7684B1A68D243D4E71A68654BD1E707
:107BD000644A1868116810601960614A624B126843
:107BE00022B91A6842F008021A6077E21A6822F095
:107BF00008021A6072E25A4B02F07F4219681B7841
:107C000042EA11226260E370FDF73EF866E2544BEF
:107C100002F07F4219681B7842EA11226260E37029
:107C2000FEF706FA5AE24C4B5B78052B00F25682BF
:107C3000DFE803F003090F151B214B4B1A6802F014
:107C40000F021A604AE2484B1A6822F010021A60CA
:107C500044E2454B1A6822F020021A603EE2424B91
:107C60001A6822F040021A6038E23F4B1A6822F08C
:107C700080021A6032E23C4B1A6822F480721A6069
:107C80002CE263782E2B04D8384A02EB83039861E8
:107C900024E203232B7021E2344BDFF8C4C0D3F875
:107CA0001491334993F83021D3F818A1CCF80090FF
:107CB000DFF8B0C0D3F81C71D3F82081D3F8246169
:107CC000D3F82851D3F82C41CCF800A0885CDFF819
:107CD00098C0DF60CCF800801E75C3F8F050C3F880
:107CE000EC4008B101238B54204B00229A75F5E13A
:107CF000A378052B10D8184A5278142A08D80621E0
:107D000001FB0233164A1349126841F82320E5E1CA
:107D1000124B03221A70E1E1104B04221A70DDE1CC
:107D200002F000FADAE102F0FFF9D7E102F0FEF921
:107D3000D4E102F0FDF9D1E102F0FCF9CEE102F06C
:107D4000FBF9CBE102F0FAF9C8E102F0F9F9C5E17B
:107D50000400002070070020640700208009002034
:107D600068090020880900206C0700202C020020F0
:107D7000F40F0020924B002283F8D520AEE1637807
:107D800013B1012B10D104E08D4B012283F8D520D3
:107D9000A4E1B0F5006F04D2894AD06082F8D530F2
:107DA0009CE104232B7099E103232B7096E1844B13
:107DB000022283F8D52091E1814B002199755975F4
:107DC0007F4A4FF0FF3402F1180040F821407D480F
:107DD0000023435401312F29F2D17B4913750B60E5
:107DE0007A4982F8D5300B607949D3600B60136112
:107DF00074E1784B1B7D13F0020F0CD1B0F5006FCE
:107E000006D26F4B0422C3F8340183F8D52065E114
:107E100004232B7062E108232B705FE1684B002282
:107E200083F8D5205AE16B4B01219A786A4BB0F563
:107E3000006F1970694B1A7028D2664B1C7D0C407C
:107E400024D103A901F00CF8644B9DF80C709DF847
:107E50000D609DF80E509DF812C09DF811009DF820
:107E600010109DF80F201C725F709E70DD7083F8FB
:107E700004C058719971DA710123584A985C117ADB
:107E800001334118082B1172F7D127E10123534A1E
:107E9000002199540133082BF9D1137813721DE195
:107EA00063788BB94B4A012091784D4A14684A4A4D
:107EB00010704A4A11700133E21812F8011C474A47
:107EC000082B9954F7D109E1012B40F007811822C2
:107ED0002A71013AEA716FF02102AA716B71FDE01B
:107EE000404B5B78032B00F2F980DFE803F00210CF
:107EF0001D22334A3C4BD2F8341192F8D5C0107D84
:107F00000A0A197183F807C098715A71E6E02C4A81
:107F1000354BD16892F8D5C0107D0A0A197183F8E3
:107F200007C098715A71D9E0284B1A682E4B5A60D5
:107F3000D4E0274B1A682C4B5A60CFE0FEF75EF86E
:107F4000CCE06278294B02B101221A70254B284AF5
:107F5000D8781B4B107093F83811264A0023117003
:107F6000254A1370254A1370B8E0154B012283F897
:107F70003921B3E0667816B1012E43D111E0042215
:107F800040F2FB7005A900F0A9FDE378626843EABE
:107F90000222059B9A4202D101236B609EE06E6033
:107FA0009CE0A3782A2B06D140F2FB7014490422EE
:107FB00000F0D0FD92E00C4B03221A708EE000BF5F
:107FC0002C020020F40F00206C070020680900201C
:107FD00088090020040000206C090020700900209E
:107FE000000000206407002080090020D80D002038
:107FF000280E0020D70F002023100020220E002082
:108000006707002003232B7068E0364B5B78032B57
:108010004CD8DFE803F00C023C47324B32495A6837
:10802000DB78D1F83C1143EA022C00232BE02E4BE5
:10803000D3F83C21092A0CD82A49501C4C68C9782D
:1080400003EB820241EA0421C2F84011C3F83C016B
:1080500044E0264B09221A7040E052F82340581C95
:1080600064450FD102EB8002013904E052F8040CA0
:10807000013342F8080C04328B42F7D31A4BC3F891
:108080003C112BE003468B42194AE6D326E0164A00
:108090000023C2F83C31164A0021D1500433282B6A
:1080A000F9D11BE0114B0A225A6017E00F4B032253
:1080B0001A7013E0FEF72EFD10E00A4B5A68DB78C9
:1080C00043EA022240F2D2439A4207D1064B0122F0
:1080D00083F8682102E0054B02221A7006B0BDE861
:1080E000F08700BF640700202C02002080090020D8
:1080F0006C03002073B5204B024640781F4D18706A
:10810000907800265870D078EC46987010790C461C
:1081100098715079587192F806E095E8030083F859
:1081200004E0D2798CE80300DA70154B1E70FEF77C
:108130003FFD144B1B7873B9637023702B78A370C9
:108140006B78E370EB792371AB7963716B79A37111
:108150002B79E37108E0012B06D10B4B9B195B785F
:10816000A3550136082EF8D1044B6A4692E8030065
:1081700083E803007CBD00BF640700208009002065
:108180007A0900206C09002070090020F7B5114D14
:10819000114C6F684FF0000C07F07F4747EA132738
:1081A0006F600E4F6E4687F800C028706970AA7025
:1081B00094E80300EB7086E80300FEF7F9FC96E80C
:1081C00003006368227884E80300054918460A70B2
:1081D000FEBD00BF64070020800900207A0900204E
:1081E0002C0200202DE9F04F984B9BB01B781BB957
:1081F000974B93F869316BB1964B1B78062B09D0DE
:108200000A2B07D00F2B05D01F2B03D0904B002239
:1082100083F838218E4A92F83831591EC9B20129A3
:1082200046D892F86A018C498C4ACC681278012BA6
:108230000CBF4FF0070C4FF0080C00230E948DF884
:1082400034C08DF835008DF83630CAB9844B8E684D
:108250001D7819795C7893F807C098795B798DF867
:108260003C608DF83D508DF83E408DF83FC08DF854
:1082700040008DF841308DF842108DF843200AE01F
:10828000012A08D1774A0133995C1AA8C218082B31
:1082900002F82D1CF6D1744B1B78002B40F0C280E5
:1082A0000DA801F039F8002840F0BC8000F00FBCA8
:1082B000032B25D192F8D440002C40F08680674BE8
:1082C0001B7893B9644D664CA8786E7822786378F1
:1082D0008619B618E279F618A379B6186279F618F5
:1082E0002379B618F618F6B219E0012B40F09A80FF
:1082F0005C4BE05C013400F0ABFE092CF8D191E05E
:10830000042B27D1544D564CAB786E7818469E19E5
:1083100001360023012222706360F6B2637000F020
:1083200097FE687800F094FE207800F091FE607867
:1083300000F08EFEE07900F08BFEA07900F088FE60
:10834000607900F085FE207900F082FE304600F072
:108350007FFE67E0072B3CD192F8D430002B34D15C
:108360003E4A127822BB3C4A3D4B557896781C78A1
:1083700093F801C0AF19D879E719997967445A7908
:10838000C7191B79CF19D719DF198DF858708DF8D7
:1083900050608DF851508DF852408DF853C08DF8D3
:1083A00054008DF855108DF856208DF8573008E0A0
:1083B000012A06D12B4A995C14AAD1540133092B06
:1083C000F8D1294B1B786BB328E0254804F06CFBEF
:1083D00028E0082B26D1204B002259789878224B90
:1083E00045181C781E4B4FF0010C01355A608DF872
:1083F00052C08DF8532016468DF854208DF8552024
:108400008DF856208DF857208DF858505A7083F803
:1084100000C08DF850008DF851101CB114A809212E
:1084200001F0EEFC114B1B78002B00F09980104AF4
:108430000D4B12780F4C013A062A00F28C80DFE8CF
:1084400002F01B1B418A8A8A650000BF790900205F
:108450002C02002064070020040000206C0900208A
:108460008009002070090020BC0D0020231000208E
:10847000D70F0020220E0020AB4A94F800C0D0682D
:10848000926819788DF82C206FF07F028DF82D20DE
:108490000A3200238DF82E207D328DF832C08DF8FF
:1084A00024208DF826300A908DF82F308DF830304A
:1084B0008DF831308DF8253000294CD109A800F015
:1084C0002BFF48E0984D2278AB786E7818469E19BD
:1084D0000A36B61800F0BCFD687800F0B9FD8020BF
:1084E00000F0B6FD8A2000F0B3FD002000F0B0FDE2
:1084F000002000F0ADFD002000F0AAFDF6B22078CB
:1085000000F0A6FD304600F0A3FD24E08648227866
:10851000417880786FF07F0500EB010C1C780CF13E
:108520000A0C002394448DF846500A358DF84750C4
:108530008DF84A308DF84CC08DF844008DF8451008
:108540008DF848308DF849308DF84B201CB111A8BA
:10855000092101F055FC754A00231370744A137009
:10856000744B754893F868110022027083F86921F2
:1085700083F8382111B10120FCF7D2F86D4B93F844
:10858000392152B193F8D4200021D2F1010238BF31
:10859000002283F8391183F8D420684B1B78002B14
:1085A00046D10DA800F096FE002841D09DF8343049
:1085B000062B3DD9624B5C4A9DF83C709DF83D60AE
:1085C0009DF83E509DF83F409DF840E09DF841C029
:1085D0009DF84280116983F803801F705E709D7062
:1085E0009C7183F805E083F804C00E9B514A9DF806
:1085F00035008B4282F86A0102D1012382F8693189
:1086000001F0F8F99DF834304FF00002072B4D4B84
:10861000484C18604C4B1A7001D1012300E0022332
:1086200084F83831434B93F8D5305A1ED2B2E8E083
:10863000404C94F8D450002D40F08C800DF1670030
:1086400000F0D4FC002800F0858000F0EBFC08B1BD
:1086500084F86B51374B9DF8670093F86B114A1CF7
:10866000D2B2C918092A81F86C0183F86B2140F055
:10867000F1802D4993F86C2148784FF0000C90421E
:1086800083F86BC107D091F82730002B00F0E2800F
:108690009A4240F0DF80244B93F82730934203D175
:1086A000244B012283F8692100231A46214C04F54A
:1086B000B671C95C01335218082BD2B2F6D194F8C6
:1086C000743193422DD11E4B94F8711194F872219C
:1086D00094F8735194F86D6194F86EE194F86FC159
:1086E00094F87001DD7059711A711E7083F801E001
:1086F00083F802C0987101F07DF9144D94F8D530DB
:108700002860591E12480022C9B2027003200129B4
:1087100084F8380184F86B2177D9052B75D00132A4
:1087200091E0042373E000BF040000202310002028
:10873000220E00202C0200206C090020BC0D00201D
:1087400064070020C40F0020BD0D0020CC0F0020C6
:10875000D60F00209B4C94F8D43083B19A4804F093
:10876000E9F960B101F046F9984994F8D53008600C
:1087700097495A1E00200870D2B203213FE0914B66
:1087800093F8D440002C45D1924B1B78002B41D05C
:1087900017A801F01FFB00283CD02346224617A94A
:1087A000C95C01335218082BD2B2F8D19DF864107D
:1087B000844C91422BD1844B9DF861109DF862202E
:1087C0009DF85D609DF85EE09DF85FC09DF86000DB
:1087D0009DF8635059711A711E70DD7083F801E0C5
:1087E00083F802C0987101F005F9784994F8D53002
:1087F000086077495A1E00200870D2B2072184F819
:108800003811012A01D9052B1CD100221BE084F864
:1088100038311FE06B4C94F8D530013BDBB2012BB3
:1088200018D8E368B3F5006F10D2FBF7F5FE68B116
:10883000E368654918460133E36000F011FB092342
:1088400084F838310122644B1A7003E05D4B00223A
:1088500083F8D5205B4C94F8D530042B05D15A4EC3
:10886000327812F0800F00F00581564B93F83831C2
:108870003BB1042B05D0082B03D0062B01D0FEF70B
:1088800097F9504C94F83831092B40F0CA8001F028
:10889000B1F8D4F8E030514AC31A002B1268B8BFBF
:1088A0005B4293420AD94E4B1A78012A01D1013218
:1088B0001A7001F09FF8434BC3F8E00001F09AF8FA
:1088C000404BD3F8E420454B821A002A5B68B8BFBE
:1088D00052429A420AD9424B5A78012A01D10132B6
:1088E0005A7001F087F8374BC3F8E40001F082F8C2
:1088F000344BD3F8E820394B821A002A9B68B8BF62
:1089000052429A420AD9364B9A78012A01D1013251
:108910009A7001F06FF82B4BC3F8E800294A537D99
:10892000002B7ED0937D002B7BD19C462D4BD2F823
:10893000F0001B68D2F8EC1007932B4B04901B68D7
:10894000D2F814810693294BD2F818711B68D2F81B
:108950001C41059392F83031D2F820610293107DCA
:10896000D368D2F82451D2F828B1D2F82C2103913F
:1089700001926246DFF86890194619F802A0BAF130
:10898000020F18D11A4951F82210B1F1FF3F0ED051
:108990000546D0B202900398DDF810B00190059E14
:1089A000069FDDF81C804FF0010C002004E0002140
:1089B00009F802101946234601322F2A1AD01C4604
:1089C0000B46D7E72C02002064070020CC0F0020C4
:1089D000D60F0020BC0D00207A090020800F002057
:1089E000F40F002068090020880900206C0700208F
:1089F00044020020374AD160C2F81C310199029B21
:108A000082F816C0C2F81481C2F81871C2F8206149
:108A10001075C2F82451C2F828B1C2F82C1182F89E
:108A200030312C4B93F83821092A06D193F8D51010
:108A3000022902D1033183F8D510264BD3F83C111B
:108A4000002944D0092A42D193F8D520012A3ED1E9
:108A5000D868002308E054F823400133A04203D132
:108A6000052382F8D53032E01A4A8B4202F5A07411
:108A7000F1D32CE094F838314BB3042B27D0082BDA
:108A800025D0062B23D0F3787168D4F83401124D29
:108A900043EA0123B0F5006F6A706B6012D2314671
:108AA00000F00EF93146D4F8340100F031F930B15C
:108AB000D4F834310133C4F83431652300E007239E
:108AC0002B7004E007232B70002384F8D5301BB0F3
:108AD000BDE8F08F2C0200208009002070B504460C
:108AE00000200E46154603210246FBF701FF002039
:108AF000C4F307210246FBF7FBFE0020E1B2024669
:108B0000FBF7F6FE002407E0944214BF0022012286
:108B1000FBF7EEFE3055013400206A1EAC420146E0
:108B2000F2D370BD10B50446002003210246FBF7C6
:108B3000DFFE0020C4F307210246FBF7D9FE002028
:108B4000E1B20246FBF7D4FE002001460122FBF70A
:108B5000CFFE10BD2DE9F04104460F461646002019
:108B600006210122FBF7C4FE002005210246FBF787
:108B7000BFFE002001220146FBF7BAFE10F0020FF3
:108B8000F2D0002002210246FBF7B2FE0020C4F31F
:108B900007210246FBF7ACFE0020E1B20246FBF7DC
:108BA000A7FE002543E0013414F03F08795D01D1B0
:108BB000012204E0721E954214BF0022012200200F
:108BC000FBF796FEB8F1000F30D1731E9D422DD2F7
:108BD000002005210246FBF78BFE00200122014602
:108BE000FBF786FE10F00100F2D106210122FBF70F
:108BF0007FFE002005210246FBF77AFE00200122BD
:108C00000146FBF775FE10F0020FF2D000200221A2
:108C10000246FBF76DFE0020C4F307210246FBF776
:108C200067FE0020E1B20246FBF762FE0135B54265
:108C3000B9D3002005210246FBF75AFE002001228D
:108C40000146FBF755FE10F0010FF2D1BDE8F081AF
:108C500038B5012204460D4600200621FBF748FEE8
:108C6000002005210246FBF743FE002001220146B9
:108C7000FBF73EFE10F0020FF2D000200221024668
:108C8000FBF736FE0020C4F307210246FBF730FE57
:108C90000020E1B20246FBF72BFE2946002001220C
:108CA000FBF726FE002005210246FBF721FE0020EF
:108CB00001220146FBF71CFE10F0010FF2D138BD76
:108CC00038B50725454305F500650C462846097863
:108CD0000135FFF7BDFF284661780135FFF7B8FF82
:108CE0002846A1780135FFF7B3FF2846E178013522
:108CF000FFF7AEFF284621790135FFF7A9FF284687
:108D00006179FFF7A5FF681CA179FFF7A1FF38BDC6
:108D10002DE9F3470725454300200C460246032171
:108D2000FBF7E6FD05F500650020C5F307210246C7
:108D3000FBF7DEFD0020E9B20246FBF7D9FD00207B
:108D400001460246FBF7D4FD82460020014602465A
:108D5000FBF7CEFD8046002001460246FBF7C8FD2A
:108D60000746002001460246FBF7C2FD814600206F
:108D700001460246FBF7BCFD0646002001460246BE
:108D8000FBF7B6FD0546002001220146FBF7B0FDCA
:108D9000237853451DD1637843451AD1A378BB424C
:108DA00017D1E37821798DF804608DF805508DF89E
:108DB0000600627943EA012343EA0243A079019A5B
:108DC00043EA006049EA0229814514BF00200120DE
:108DD00000E00020BDE8FC8738B54FF400640020B7
:108DE00006210122FBF784FD002005210246FBF746
:108DF0007FFD002001220146FBF77AFD10F0020FF3
:108E0000F2D0002002210246FBF772FD0020C4F3DD
:108E100007210246FBF76CFD0020E1B20246FBF79A
:108E200067FD002500203F2D14BF002201220146CE
:108E30000135FBF75DFD402DF4D1002005210246F0
:108E4000FBF756FD002001220146FBF751FD10F013
:108E5000010FF2D14034B4F5804FC0D138BD00BF0E
:108E600038B50725454300200C4602460321FBF791
:108E70003FFD05F500650020C5F307210246FBF71D
:108E800037FD0020E9B20246FBF732FD0020014623
:108E90000246FBF72DFD2070002001460246FBF73D
:108EA00027FD6070002001460246FBF721FDA070FF
:108EB000002001460246FBF71BFDE0700020014642
:108EC0000246FBF715FD2071002001460246FBF724
:108ED0000FFD6071002001460122FBF709FDA07122
:108EE00038BD00BF37B5002005210246FBF700FD65
:108EF000002001220146FBF7FBFC10F07104F2D1C7
:108F000000F078FD054605E0FFF70CFE422814BF8F
:108F10000024012400F06EFD431B002BB8BF5B4210
:108F2000B3F5FA6F40F2FF7002DA002CECD000E0EB
:108F30001CB1294B1B78002B3CD040F2FF70002164
:108F4000FFF786FEFFF748FF002024494022FFF785
:108F500001FE40254FF480742046B4222049FFF7DB
:108F6000F9FDB434284620221E49FFF7F3FD2035D1
:108F7000B4F5A76FF0D100230193E03401AD204692
:108F8000042204342946FFF7E5FDB4F5FF6FF5D15F
:108F900000230193A4F530742046042204342946AA
:108FA000FFF7D8FDB4F5C36FF6D140F2FF70422150
:108FB000FFF74EFE002009494022FFF78FFD4024B5
:108FC00009492046091920222034FFF787FDB4F50E
:108FD000807FF5D13EBD00BF440E0020040000207C
:108FE0004022010870220108640E0020094B196814
:108FF0005A68914201D100200BE01A68D118097A11
:10900000013201701A601A68202A01D100221A6008
:1090100001207047A4030020014B9862704700BFF5
:10902000A4030020034B1A78104612B100221A70D4
:10903000012070472C10002008B5FBF797FA034B6E
:1090400000221A605A60FBF78FFA08BDA4030020C3
:1090500038B50B4B8446DC6A1A6B0134202C08BFF0
:10906000002494420AD0DD6A0648ED1885F834C021
:1090700040F227710122DC6206F06EFC38BD00BFB1
:10908000A40300200044004038B50546002401E058
:10909000FFF7DEFF2B5D01341846002BF8D138BDF9
:1090A0002A4910B50B8813F0200F1CD0284BDB6821
:1090B00013F0020F01D08B8815E0264B5A68186810
:1090C0000132202A08BF0022824205D05C688888CD
:1090D000E118C0B208725A601F4B0A221A601D4B79
:1090E0009A6A1E4B1A601948038813F0800F1BD030
:1090F0001A4B1A68C2B9174BDC6A196B8C420FD035
:10910000134902240C61196BCC1894F834C0013156
:10911000A0F804C01963196B202905D11A6303E074
:1091200040F2277106F018FC0848038813F0400F3E
:109130000BD040F2266106F007FD064B1A6BDB6A86
:109140009A4202D1024B02225A6110BD00440040F3
:1091500000080140A4030020281000202410002053
:1091600030B5054687B0564806F03EFD4FF4003056
:10917000012105F087FB0420012105F075FB042087
:10918000002105F08DFB0820002104F0F5FF06AC5E
:109190004FF0040324F8083D03234A4821468DF884
:1091A000123015338DF8133004F056FF482345482C
:1091B0008DF8133021464FF00803ADF8103004F05D
:1091C0004BFF684606F092FB0B2D25D8DFE805F033
:1091D0002406090C0F1215181B1E20224FF4615390
:1091E0001CE04FF4964319E04FF4E14316E04FF4CE
:1091F000164313E04FF4614310E04FF496330DE053
:109200004FF4E1330AE04FF4613307E02E4B05E001
:109210002E4B03E02E4B01E04FF416530093009BBE
:1092200006A95B0841F8183D2548694606F094FCFC
:1092300026230024012505A88DF8143007238DF876
:1092400015308DF816408DF8175005F075F81C484C
:1092500040F2FF3106F054FC28212246184806F05F
:109260007BFB2A46164840F2277106F075FB2A461A
:10927000134840F2266106F06FFB2A46104840F280
:10928000255106F069FB22460D4840F2244106F0C4
:1092900063FB22460A4840F6460106F05DFB224683
:1092A000074840F66A1106F057FB60212246044841
:1092B00006F052FB2946024806F040FB07B030BDDD
:1092C000004400400008014090D0030020A10700A6
:1092D00040420F0030B50C4B0C4C844622681B6892
:1092E0009A4201D100200EE02368094A5D1C02EB7E
:1092F00003130FCB8CE80F0025602368082B01D1E6
:1093000000232360012030BDBC100020301000205D
:109310003C100020704700BFF0B5437887B0064688
:10932000426833B104238DF80C300023029201937C
:1093300003E0019202938DF80C30B37803B102235D
:109340008DF80D30327800238DF80E20F21801A828
:10935000117AC2180133082BD172F7D104F0BEF88C
:10936000042818D10D4D0E4B2C681B680134082CB5
:1093700008BF00249C4201D100200DE096E80F00B8
:109380002F68084E06EB071C8CE80F0001200146F1
:109390002C6004F095F8012007B0F0BD34100020D7
:1093A00038100020C01000207FB52B4B2B4A1968C5
:1093B0001268914204D10120002104F081F848E0B4
:1093C0001968274A02EB0111487850B11B6802EB7B
:1093D0000312536804228DF80C200022019202939C
:1093E00007E01B68029002EB031253688DF80C0033
:1093F0000193194B1A681A4B03EB02139B781BB1AC
:1094000002238DF80D3001E08DF80D30124B002253
:109410001968134B0901CB5C8DF80E300E4B0DF122
:10942000180C18680CEB020102EB001C0C4801320E
:109430006044007A082A01F8090CEFD11A68013259
:109440001A601A68082A01D100221A6001A804F0E3
:1094500045F807B000BD00BF3810002034100020D0
:10946000C010002073B50220002104F029F810205C
:10947000002104F025F801AC0021012004F020F8BF
:1094800000250726142320468DF804308DF805604A
:109490008DF806508DF8075004F04EFF1523204636
:1094A0008DF804308DF805608DF806508DF8075062
:1094B00004F042FF204613238DF804308DF8056038
:1094C0008DF806508DF8075004F036FF04F002FACC
:1094D00029464FF0007005F0D5F97CBD2DE9F0412B
:1094E00001388AB00C46154607285BD8DFE800F043
:1094F0004C4034281C5A10040C238DF81C300323D4
:109500008DF81D3000238DF81B304FF0020354E01E
:109510000C238DF81C3003238DF81D3000238DF8AB
:109520001B304FF004023AE00C238DF81C3003236B
:109530008DF81D3000238DF81B304FF010022EE007
:109540000C238DF81C3003238DF81D3000238DF87B
:109550001B304FF0140330E00C238DF81C30032334
:109560008DF81D3000238DF81B304FF0280216E0D7
:109570000C238DF81C3003238DF81D3000238DF84B
:109580001B304FF0640318E00C238DF81C300323CC
:109590008DF81D3000238DF81B304FF0C802ADF858
:1095A0001E200CE00C238DF81C3003238DF81D3099
:1095B00000238DF81B304FF00803ADF81E3004F087
:1095C00089F901214FF0007005F05CF90120014696
:1095D00005F04AF90820012105F046F9082000218C
:1095E00005F05EF901214FF4EA1004F0C5FD0AAE62
:1095F0004FF4007226F8042D032331468A488DF873
:10960000263015338DF8273004F026FD042331462B
:1096100085488DF827304FF4807300260127ADF878
:10962000243004F019FD05A88DF81A608DF8146037
:109630008DF815708DF816608DF817608DF818701C
:109640008DF8197003F03AFEB4F5006F01A815DA31
:109650004FF0FF326301ADF80830ADF810608DF8BF
:1096600012708DF804608DF805608DF80670ADF805
:109670000A60ADF80C20ADF80E2013E04FF0FF3378
:109680008DF80670ADF810608DF812608DF80460EA
:109690008DF80560ADF80860ADF80A60ADF80C30E3
:1096A000ADF80E3003F07CFEDDB1B5F5006F18DAD1
:1096B000002201236901ADF80A208DF805204FF042
:1096C000FF3201A8ADF808108DF812308DF8043083
:1096D0008DF80630ADF80C20ADF80E20ADF8103046
:1096E00016E000230122ADF80A308DF812308DF813
:1096F0000530ADF808304FF0FF3301A8ADF8102069
:109700008DF804208DF80620ADF80C30ADF80E3041
:1097100003F046FEE30043F004030DF104080027C4
:10972000012602226413ADF80A3040464FF0FF33A1
:109730008DF80420ADF808408DF805708DF80660AE
:10974000ADF80C30ADF80E30ADF810708DF8126039
:1097500003F026FEBD421ADDEB0043F004036D1357
:109760000322ADF80A304FF0FF3340468DF8042055
:109770008DF80570ADF808508DF812608DF8066010
:10978000ADF80C30ADF80E30ADF8106017E00323E3
:109790008DF804304FF004024FF0FF334046ADF82F
:1097A0000870ADF810608DF812708DF805708DF8A6
:1097B0000660ADF80A20ADF80C30ADF80E3008AFF9
:1097C00003F0EEFD012407260025142338468DF80A
:1097D00020308DF821608DF822508DF8234004F060
:1097E000ABFD152338468DF820308DF821608DF8BB
:1097F00022508DF8234004F09FFD132338468DF846
:1098000020308DF821608DF822508DF8234004F02F
:1098100093FD0220214603F053FE2146102003F061
:109820004FFE0AB0BDE8F081000C014030B52A4D72
:109830002A4B2C681B680134082C08BF00249C426A
:1098400087B044D0012001A903F024FF9DF80C202B
:10985000234B042A09D12A68012103EB021251701B
:109860002A6803EB0213029A08E02A68002103EB3E
:10987000021251702A6803EB0213019A5A609DF894
:109880000D30154A022B164B04D1126803EB02135C
:10989000012203E0126803EB021300229A700E4BC0
:1098A0009DF80E101A680E4B1201D15400230A4A7B
:1098B00006A9C81811680A4D03EB011110F8090C2C
:1098C00001334919082B0872F1D1146002E001201C
:1098D00003F0C4FE07B030BDBC10002030100020E3
:1098E0003C10002030B52A4D2A4B2C681B680134EF
:1098F000082C08BF00249C4287B044D0002001A956
:1099000003F0C8FE9DF80C20234B042A09D12A68D5
:10991000012103EB021251702A6803EB0213029A31
:1099200008E02A68002103EB021251702A6803EB59
:109930000213019A5A609DF80D30154A022B164BFE
:1099400004D1126803EB0213012203E0126803EB57
:10995000021300229A700E4B9DF80E101A680E4BDF
:109960001201D15400230A4A06A9C81811680A4DE9
:1099700003EB011110F8090C01334919082B087287
:10998000F1D1146002E0002003F068FE07B030BDA2
:10999000BC100020301000203C100020104B1A7822
:1099A0007AB159680F4A0131596011680E4B013183
:1099B00011601A6812B11A68013A1A600022084B45
:1099C00000E001221A70094B1A683AB11A68013A8C
:1099D0001A601B6813B9064B01221A70704700BF4A
:1099E000F80300207C09002024100020281000200B
:1099F0002C100020014B5868704700BFF80300206E
:109A000008B5042005F060F948F6A04005F06CF9AF
:109A1000012005F06FF904480321002204F05AFDEB
:109A2000012005F07DF908BD9AC30200042807D083
:109A3000082809D008B100200DE0074B188801E084
:109A4000054B588880B206E0034B988840F26B13B0
:109A500080B25843001370470004002070B592B0E4
:109A600011AE0024032531464FF002034148ADF802
:109A700044308DF846508DF8474004F0EDFA4FF031
:109A8000110331463C48ADF844308DF846508DF80E
:109A9000474004F0E1FA0120014604F0D7FE01211D
:109AA0004FF4007004F0E0FE344803F01FFF344B25
:109AB00032480193334B01A9029380230693DB18AC
:109AC000079303F540730893A3F57873099303F59F
:109AD000FF530A930394049505940B9403F076FFC7
:109AE0002648012103F0A2FF01264FF460232648F7
:109AF0000CA90E930C948DF834608DF835600F949A
:109B00008DF8405003F00EFA1F480A2132462B46CA
:109B100003F08AFA1C480E2102222B4603F084FA35
:109B20002B462A461848092103F07EFA2246164899
:109B30004FF4FC6103F03AFA1348314603F02CFA73
:109B40001148314603F01EFA0F4803F039FA0E4867
:109B500003F03CFA0028FAD10B4803F03BFA0A481C
:109B600003F03EFA0028FAD10748012103F03CFA3D
:109B700012B070BD000C014000100140080002400E
:109B80004C2401400004002000240140014B03222A
:109B90001A60704708040020044A054B927A0AB103
:109BA000052200E001221A60704700BF4C1100201E
:109BB00008040020704700BF014B00225A60704724
:109BC0000804002008B5074B1A6892B242F0080258
:109BD0001A601A6892B242F004021A60FFF7D6FFC8
:109BE00008BD00BF405C004010B5064C4FF6FB734B
:109BF000226802EA03032360FFF7CEFF4FF4064317
:109C0000236010BD405C0040072818BF1F4B10B5F3
:109C10001E4C18BF18702378052B33D8DFE803F0EB
:109C200003060A0E1621FFF7DFFF2BE0FFF7DCFF2C
:109C3000042328E002236370013324E06378013BAE
:109C4000DBB263706378FBB9042218E0104B1A682A
:109C500092B242F010021A6005232370DB18637081
:109C600012E06378013BDBB26370637863B9084A42
:109C70004FF6EF73116801EA030313600622034BEA
:109C80001A7001E00623237010BD00BFB011002040
:109C9000405C0040034B9B7A13B1034B05221A60D2
:109CA000704700BF4C11002008040020014B042223
:109CB0001A60704708040020034B1A7A202A01D149
:109CC00000221A72704700BF08040020704700BFCE
:109CD000212808B508D1124B1B681B7803F07F03BD
:109CE000212B1AD10F4B0EE0202816D10C4B0E4A17
:109CF0001B681B7810720D4A03F07F03212B0CBFE9
:109D0000134600234BB1064A4FF0000112680020B1
:109D1000518293619847002000E0022008BD00BFF7
:109D2000AC110020659D000808040020819D0008FA
:109D3000074B1B681B7803F07F03212B05D10228FA
:109D400001D0222801D1002000E00220704700BF8E
:109D5000AC11002019B9012801D8084600E0022002
:109D6000704700BF28B9044B4FF008021B681A82E5
:109D700000E00248704700BFAC1100204400002002
:109D800028B9044B4FF008021B681A8200E0024811
:109D9000704700BFAC110020440000200B4B10B5F1
:109DA000DA6882B11B68052B01D000220BE000238A
:109DB00003E00749595CC15401330449CC68A3420C
:109DC000F7D30023CB60104610BD00BF080400206D
:109DD000B4110020084BDB68082B01D800200AE0F2
:109DE0000023064A9A5CC2540133092BF9D1024B75
:109DF0000022DA600120704708040020B41100201E
:109E000010B5074C0B468AB2C021636006F0C8FC4F
:109E10000120A18806F0D2FE012006F09DFD10BDB4
:109E20000804002007B5142200238DF8042001A89F
:109E300001228DF806308DF807208DF8053004F0EA
:109E40007BFA0EBD07B5142200238DF8042001A86B
:109E500001228DF806308DF807208DF8053004F0CA
:109E60006BFA0EBD08B5064B1B68DB78042B01D9D5
:109E7000002004E0034901EBC30106F039F808BDF6
:109E8000AC1100204C00002008B5024906F030F863
:109E900008BD00BF6C00002008B5024906F028F894
:109EA00008BD00BF74000020334B10B51B686FF075
:109EB0003F0200245A72DC729C72204606F0C4FCF9
:109EC00020464FF4007106F0DDFC1021204606F01C
:109ED000EFFC4021204606F045FE8021204606F09A
:109EE00031FE204606F06EFD244B204693F86410A8
:109EF00006F086FE204606F03DFD0120214606F0D4
:109F0000C1FC0120C02106F01DFE0120202106F029
:109F1000CFFC0120214606F0E3FC02204FF4C06193
:109F200006F0B0FC02204FF4807106F00BFE022018
:109F3000214606F0D5FC0220202106F0B9FC0320C2
:109F4000214606F09FFC03204FF4887106F00AFEBC
:109F50000320402106F054FE03204FF4405106F048
:109F6000BFFC2146032006F0A3FC204605F0CEFFEF
:109F7000034B01221A6010BDAC11002044000020E8
:109F80000804002008B5174B174A196889B21180D8
:109F900016491288098801EA020212F4806F05D07E
:109FA0004FF6FF321A60124BDB6B98470E4B1A8844
:109FB0000E4B1B8803EA020212F4007F08D0094905
:109FC0000C4A4FF6FF500860117C0131C9B2117480
:109FD000054A1288134013F4004F01D006F01CFB11
:109FE00008BD00BF445C004042110020F411002075
:109FF000440000200804002010B5032006F030FEC5
:10A00000064C034602464FF488710548E36006F0AB
:10A01000DFFB032006F0AEFC10BD00BF08040020EB
:10A02000B411002008B528B105484FF4806104F050
:10A0300079F804E002484FF4806104F075F808BD37
:10A040000008014038B5064D01232B60054B002464
:10A0500020461C60FFF7E6FF03232B60204638BD37
:10A06000405C0040445C004008B5FFF7EBFF08BDD2
:10A0700008B50120FFF7D6FF064B012119600649FC
:10A080004FF4E0520A8005490020186008601A6009
:10A0900008BD00BF405C0040F4110020445C00405B
:10A0A000084B10B51B6800249C72FFF7E1FF064ABD
:10A0B0004FF406431460043A1360044A1460044ADF
:10A0C000138010BDAC110020445C00400804002047
:10A0D000F4110020002008B504F03CFB4FF4000010
:10A0E000012104F0CFFB08BD07B5FFF7F3FFFFF731
:10A0F000A9FE06F033FA0420012104F0B5FB032386
:10A100008DF806300D338DF8073004484FF4806326
:10A1100001A9ADF8043003F09FFF0EBD0008014017
:10A12000704700BF704700BF704700BF704700BF57
:10A13000704700BF704700BF704700BF704700BF47
:10A14000704700BF10B5FFF755FC074C2368C31AD2
:10A15000B3F5FA7F07D9054BDA6882F40062DA605A
:10A16000FFF748FC206010BDF8110020000C0140F2
:10A17000024B03EBC003D879704700BF1C040020DA
:10A18000024B03EBC0035879704700BF1C0400204A
:10A19000024B03EBC0039879704700BF1C040020FA
:10A1A000034B0B2202FB003393F83000704700BFD3
:10A1B0001C040020034B0B2202FB003393F83100F8
:10A1C000704700BF1C040020034B0B2202FB00332E
:10A1D00093F83300704700BF1C040020034B0B2290
:10A1E00002FB003393F83200704700BF1C040020CC
:10A1F000034B0B2202FB003393F83400704700BF7F
:10A200001C040020034B0B2202FB003393F83500A3
:10A21000704700BF1C040020034B0B2202FB0033DD
:10A2200093F83600704700BF1C040020034B0B223C
:10A2300002FB003393F83800704700BF1C04002075
:10A24000034B0B2202FB003393F83900704700BF29
:10A250001C040020034B0B2202FB003393F83A004E
:10A26000704700BF1C040020034B052202FB003393
:10A2700093F87400704700BF1C040020034B0522B4
:10A2800002FB003393F87500704700BF1C040020E8
:10A29000034B052202FB003393F87600704700BFA2
:10A2A0001C040020034B052202FB003393F87700C7
:10A2B000704700BF1C040020034B052202FB003343
:10A2C00093F87800704700BF1C040020034B032262
:10A2D00002FB003393F89400704700BF1C04002079
:10A2E000034B032202FB003393F99500704700BF34
:10A2F0001C040020034B032202FB003393F896005A
:10A30000704700BF1C040020024B03EBC00393F80E
:10A31000A80070471C040020024B03EBC00393F815
:10A32000A90070471C040020024B03EBC00393F804
:10A33000AA0070471C040020024B03EBC00393F8F3
:10A34000AB0070471C040020024B03EBC00393F8E2
:10A35000AC0070471C040020024B03EBC00393F8D1
:10A36000AD0070471C040020024B03EBC00393F8C0
:10A37000AE0070471C040020024B03EBC00393F8AF
:10A38000AF0070471C040020062821D8DFE800F049
:10A3900004080C1014181C000E4BD3F8D83016E02B
:10A3A0000C4BD3F8DC3012E00A4BD3F8E0300EE06F
:10A3B000084BD3F8E4300AE0064BD3F8E83006E067
:10A3C000044BD3F8EC3002E0024B93F837300B60CB
:10A3D000704700BF1C040020F8B5104B0D461E5CF2
:10A3E000C1F3074100223046FAF782FA0C4C07020B
:10A3F000C5F3072100223046C4F8D870FAF778FA7E
:10A4000007433F023046E9B20122C4F8D870FAF798
:10A410006FFA07433F09C4F8D870F8BD4823010814
:10A420001C040020334B032202FB003310B594338D
:10A4300093F901203F2A01DD3F225A702D4B032260
:10A4400002FB0033943393F9012012F13F0FBCBF9C
:10A450006FF03E025A70274B032202FB0033943305
:10A460009A781F2A01D91F229A70224B032202FBDD
:10A4700000324FF44021C3F8F01092F89420012AE2
:10A4800004BF4FF45022C3F8F0201A4B03EBC00274
:10A4900092F8AF204AB9033202FB003292F89520BD
:10A4A000D3F8F01002F07F020CE0032101FB003131
:10A4B00091F895C002F003020CF07C0CD3F8F01078
:10A4C0004CEA02020B4C41EA0222C3F8F0200323BB
:10A4D00003FB004393F89620D4F8F03042EA0303DC
:10A4E0001946C4F8F030FFF777FFD4F8F030C4F81D
:10A4F000E83010BD1C04002008B5044B032202FB09
:10A50000003383F89610FFF78DFF08BD1C04002070
:10A5100008B5044B032202FB003383F89510FFF7C4
:10A5200081FF08BD1C04002008B5044B032202FB78
:10A53000003383F89410FFF775FF08BD1C0400205A
:10A540002A4B052210B502FB003393F87420012A30
:10A5500002D9012283F87420244B052202FB003328
:10A5600074335A78032A01D903225A701F4B0522EB
:10A5700002FB003374339A780F2A01D90F229A70A4
:10A580001A4B052202FB00337433DA78032A01D90F
:10A590000322DA70154B052202FB003374331A795B
:10A5A0000F2A01D90F221A71104C052303FB004317
:10A5B00003F1740292F804C093F874104CF4202351
:10A5C00092F801C043EAC133917843EA4C33D27820
:10A5D00043EA012343EA42131946C4F8F030FFF777
:10A5E000FBFED4F8F030C4F8E43010BD1C040020A9
:10A5F00008B5044B052202FB003383F87810FFF7FF
:10A600009FFF08BD1C04002008B5044B052202FB77
:10A61000003383F87710FFF793FF08BD1C04002078
:10A6200008B5044B052202FB003383F87610FFF7D0
:10A6300087FF08BD1C04002008B5044B052202FB5F
:10A64000003383F87510FFF77BFF08BD1C04002062
:10A6500008B5044B052202FB003383F87410FFF7A2
:10A660006FFF08BD1C0400205C4B0B2210B502FBE1
:10A67000003393F83020032A02D9032283F83020D4
:10A68000564B0B2202FB003330339A78032A01D950
:10A6900003229A70514B0B2202FB003330331A799C
:10A6A0000F2A01D90F221A714C4B0B2202FB0033E7
:10A6B00030335A79072A01D907225A71474B0B22A6
:10A6C00002FB003330339A790F2A01D90F229A7195
:10A6D000424B0B2202FB003338335A780F2A01D940
:10A6E0000F225A703D4B0B2202FB003338339A780D
:10A6F0000F2A01D90F229A70384B0B2202FB00322D
:10A7000092F83010C90341F40024C3F8F04092F8E5
:10A7100031201AB141F40421C3F8F0102F4B0B2162
:10A7200001FB003191F8331029B1D3F8F01041F456
:10A730000051C3F8F010294B92B90B3202FB0032E2
:10A74000303292F804C091784FEACC1CD3F8F04034
:10A750004CEAC12C51794CEA040242EA011222E08F
:10A760000B2202FB003292F838202AB1D3F8F020F5
:10A7700042F48052C3F8F020184B0B2101FB00314A
:10A78000383191F801E0D3F8F020897842EACE120E
:10A7900001F0070C42EA0C1211F0080FC3F8F02088
:10A7A00003D042F40062C3F8F0200C4B0B2202FBF2
:10A7B00000323032D17931B99179D3F8F02041EAC1
:10A7C0000202C3F8F020054CD4F8F010FFF704FEA5
:10A7D000D4F8F030C4F8E03010BD00BF1C040020F5
:10A7E00008B5064B0B2202FB00333033DA791AB17D
:10A7F0000022DA71FFF738FF08BD00BF1C040020FB
:10A8000008B5064B0B2202FB00333033DA791AB954
:10A810000132DA71FFF728FF08BD00BF1C040020D9
:10A8200008B5044B0B2202FB003383F83A10FFF704
:10A830001BFF08BD1C04002008B5044B0B2202FBC3
:10A84000003383F83910FFF70FFF08BD1C04002008
:10A8500008B5044B0B2202FB003383F83810FFF7D6
:10A8600003FF08BD1C04002008B5044B0B2202FBAB
:10A87000003383F83610FFF7F7FE08BD1C040020F4
:10A8800008B5044B0B2202FB003383F83510FFF7A9
:10A89000EBFE08BD1C04002008B5044B0B2202FB94
:10A8A000003383F83410FFF7DFFE08BD1C040020DE
:10A8B00008B5044B0B2202FB003383F83210FFF77C
:10A8C000D3FE08BD1C04002008B5044B0B2202FB7C
:10A8D000003383F83310FFF7C7FE08BD1C040020C7
:10A8E00008B5044B0B2202FB003383F83110FFF74D
:10A8F000BBFE08BD1C04002008B5044B0B2202FB64
:10A90000003383F83010FFF7AFFE08BD1C040020B1
:10A9100010B52D4A4FF46021C2F8F01002EBC001CF
:10A9200091F8AF10034619B14FF47021C2F8F0103E
:10A93000254A02EBC30191F8A90091F8A8C0D2F80A
:10A94000F040000340EA8C302043C2F8F00091F858
:10A95000AA10012904BF40F48060C2F8F0001A4A2E
:10A9600002EBC30090F8ABC0D2F8F01041EA0C2122
:10A97000C2F8F01090F8AC00012804BF41F080014B
:10A98000C2F8F010104A02EBC30191F8AD10012992
:10A9900005D1D2F8F01041F04001C2F8F0100A4C95
:10A9A000184604EBC30393F8AE20D4F8F03043EA22
:10A9B00002131946C4F8F030FFF70EFDD4F8F0305A
:10A9C000C4F8EC3010BD00BF1C04002008B5044BD7
:10A9D00003EBC00383F8AE10FFF79AFF08BD00BF7A
:10A9E0001C04002070B5104B064603EBC00393F81F
:10A9F000AE50032D02D00321FFF7E8FF3046FFF7EA
:10AA000087FF094BD3F8D84014F4002F1CBF6FEA1E
:10AA100004346FEA1434032D03D030462946FFF77F
:10AA2000D5FF204670BD00BF1C04002008B5044BB4
:10AA300003EBC00383F8AD10FFF76AFF08BD00BF4A
:10AA40001C04002008B5044B03EBC00383F8AC10D2
:10AA5000FFF75EFF08BD00BF1C04002008B5044BD3
:10AA600003EBC00383F8AB10FFF752FF08BD00BF34
:10AA70001C04002008B5044B03EBC00383F8AA10A4
:10AA8000FFF746FF08BD00BF1C04002008B5044BBB
:10AA900003EBC00383F8A910FFF73AFF08BD00BF1E
:10AAA0001C04002008B5044B03EBC00383F8A81076
:10AAB000FFF72EFF08BD00BF1C040020064B10B599
:10AAC00003EBC003044683F8AF10FFF721FF2046D5
:10AAD000FFF7A8FC10BD00BF1C04002010B5194AE8
:10AAE0000021C2F8F01002EBC0014979034619B108
:10AAF0004FF40071C2F8F010124A02EBC3018979D9
:10AB000029B1D2F8F01041F48071C2F8F0100D4A6A
:10AB100002EBC302D1790F2901D90F21D171094C60
:10AB2000184604EBC303DA79D4F8F03042EA0303A1
:10AB30001946C4F8F030FFF74FFCD4F8F030C4F8F1
:10AB4000DC3010BD1C04002070B5084D9DF810E0ED
:10AB50009DF8146005EBC00426716270A37084F840
:10AB600003E005F83010FFF7B9FF70BD1C040020AA
:10AB700008B5034B03EBC0039971FFF7AFFF08BDA6
:10AB80001C04002008B5054B03EBC003597109B143
:10AB90000422DA71FFF7A2FF08BD00BF1C040020E9
:10ABA00008B5054B042903EBC003D97101D000227D
:10ABB0005A71FFF793FF08BD1C0400202DE9F047F0
:10ABC000374D0446401990F8F4000E461746984653
:10ABD000DDF82090DDF824A004281FD8DFE800F07D
:10ABE00003090F151B002046FFF73EFD65190123E1
:10ABF00016E02046FFF78CFE6519022310E0204680
:10AC0000FFF79EFC651903230AE02046FFF70AFCC4
:10AC10006519042304E02046FFF760FF651900234F
:10AC200085F8F4301E4B03EBC40494F8AE20012ADF
:10AC30000FD002D3022A28D114E01EB1D3F8D830A5
:10AC40009B0C33700FB3164BD3F8D8309B0A3B7074
:10AC50001BE0B8F1000F18D0D3F8D8309B0AC8F821
:10AC6000003012E0B8F1000F05D0D3F8D830DB0B7C
:10AC70005B01C8F80030B9F1000F06D0084BD3F8DB
:10AC8000D830C3F3842389F80030BAF1000F04D020
:10AC9000034BD3F8D8308AF80030BDE8F08700BF06
:10ACA0001C04002000202F4A2DE9F84F84468646D8
:10ACB0002D4B2E4C03F1940B03F1A80A4FF0010920
:10ACC0000BF80C900AEB0E01251803EB0E08032479
:10ACD00000230527E3444FF002068BF802708BF83F
:10ACE000017081F80590CB714C708B70CB700B713B
:10ACF0008E711E490CF1030C0AF80E400B542B7197
:10AD00006B70AB70EB70C01988F8073088F80530AD
:10AD100088F8063016719771947216705370D3705C
:10AD200093705471D371137253720B32BCF1120FC2
:10AD30000EF1080EBCD11D46ECB22046FFF700FC18
:10AD40002046FFF76FFB2046FFF7E2FD2046FFF7A6
:10AD5000C5FE01352046FFF787FC062DECD1BDE886
:10AD6000F88F00BF4C0400201C0400209004002039
:10AD700038B5074D0024074B0022E254E0B2A97A0F
:10AD80000134F9F7D5FC2035062CF4D138BD00BFCD
:10AD9000A40E0020D80F0020F0B5834B85B01A78A0
:10ADA0004AB96FF00042012119709A615A609A60A5
:10ADB000DA601A615A617C4B1C7F5CB9E0B2F9F72A
:10ADC0005BFC794B03F1200210550134082CF5D1BE
:10ADD00001221A7727240025E8B2F9F74DFC734ABF
:10ADE000535D83421BD0724B05F1080103EB8103D5
:10ADF0005B685055022B05D0032B0AD0012B0ED1D6
:10AE000068B106E058B96B4A115D012907D11355A5
:10AE100005E0684B1A5D012A01D101321A5501354E
:10AE20000134082DD8D1644DEB69B3B1634B1C7864
:10AE30009CB9FEF7DFFD624AEB691268821A002AAC
:10AE4000B8BF52429A4208D92046013401F064FB4F
:10AE5000062CF9D1594B01221A70574D2B6AB3B108
:10AE6000584B1C789CB9FEF7C5FD574A2B6A1268EF
:10AE7000821A002AB8BF52429A4208D920460134A9
:10AE800001F04AFB062CF9D14E4B01221A70464CB8
:10AE90004E4A94F82800830002EBC302127B62B191
:10AEA0004B4A4C4D4C4C0021D3182D1824180A46FF
:10AEB00000950194FFF782FE97E3FEF79BFDE36A9E
:10AEC000C31A002BB8BF5B420A2B40F38E8394F861
:10AED0002800022801D8410101E0C11E490141F0CA
:10AEE0000A01C9B2022894BF0020012001F0BAF97A
:10AEF0002D4D044695F8280001F046FB95F82830C2
:10AF00004FF00C0C022B98BF194694BF002201226F
:10AF100088BFD91E242050430CFB01012F4809187B
:10AF2000097A59B1022B94BF1946D91E24204243F5
:10AF30000C2000FB012129480D580BE0022B94BF87
:10AF40001946D91E242042430C2000FB012123482E
:10AF500009184D68224AD25C032A00F21181DFE809
:10AF600002F0029E1E75002C00F00A81174A0E4E58
:10AF700002EB4311C97F1A4D31B11846F9F7D8FBDE
:10AF800096F82830032208E002EB43121846517A63
:10AF9000F9F7CEFB96F828300222EA54F0E07CBBA9
:10AFA000022B1FD859011FE018050020380500208A
:10AFB000800F0020F40F002004000020D60F002096
:10AFC000CC0F0020BD0D0020C40F0020A40E0020D7
:10AFD0002C0E0020DC0D0020980E0020480E0020D2
:10AFE000D80F0020D91E490141F00801C9B2022B37
:10AFF00094BF0020012001F035F90646002861D0F9
:10B00000534E544B96F8280003EB4013D97F002988
:10B0100000F0AE80002D84EAE472B8BF6D42A2EB6E
:10B02000E472AA4202D0002C40F09B804A4B53F8B5
:10B0300030108A4280F09C8003EBC0031979F9F745
:10B0400077FB434B012193F828308FE0002D84EAF1
:10B05000E471B8BF6D42A1EBE471A94202D0002CAB
:10B0600040F086803C4A3A4E52F833003B4D8142D4
:10B0700009D202EBC30218461179F9F759FB96F889
:10B080002830012209E0334A184602EB4313597A6B
:10B09000F9F74EFB96F828300222EA5468E0002CBB
:10B0A00032D1022B01D8590101E0D91E490141F0EA
:10B0B0000801C9B2022B94BF0020012001F0D2F890
:10B0C000064608BBFEF796FC214D224A95F828302B
:10B0D0004FF00A0E02EB4311B1F81CC099004F1952
:10B0E0007F680EFB0CFCC71B002FB8BF7F42674573
:10B0F00046DD02EBC1021846917AF9F719FB95F883
:10B100002830164AD6543BE0114E124A96F82830A1
:10B1100002EB4312D17F59B3002D84EAE472B8BF29
:10B120006D42A2EBE472AA4200D0CCB90A4951F8B0
:10B1300033108A421CD3074A184602EB4313597A4C
:10B14000F9F7F6FA024B022193F828300EE000BF1F
:10B1500018050020A40E0020E40D0020D80F0020C8
:10B160001846F9F7E5FA96F828300321A44AD15495
:10B17000A44D95F82860FEF73DFC05EB8605686058
:10B18000A04DA14F95F82830A04E1846F618FF188C
:10B190009F4B002103EB80030A46019600979D4ECA
:10B1A000FFF70CFD95F8280006EB40139B69002B78
:10B1B00038D0F9F7AFF9002834D095F8280084EAA0
:10B1C000E47206EB40139B69A2EBE4729A4229D920
:10B1D00001F0A2F995F828308F4906EB4312927FCF
:10B1E0000120C854A2B10025864B8A4A93F8281042
:10B1F000B37F02EB4112927F20369A4205D1284656
:10B2000001F08AF9E8B200F007FA0135062DEBD11A
:10B210007C4B824A93F828300F33D15C012901D14D
:10B220000131D154774D95F82830022B25D80020D4
:10B2300000F0B0FE95F8303010F0010F03F0F80385
:10B2400085F830301CBF43F0010385F8303010F032
:10B25000040F8DF80C0006D06A4B93F8302042F0B2
:10B26000020283F8302010F0100F06D0654B93F8DF
:10B27000302042F0040283F83020624D95F82830E7
:10B28000033BDBB2022B25D8012000F083FE95F8AA
:10B29000303010F0010F03F0C70385F830301CBFC9
:10B2A00043F0080385F8303010F0040F8DF80D00DE
:10B2B00006D0544B93F8302042F0100283F830202F
:10B2C00010F0100F06D04F4B93F8302042F02002C0
:10B2D00083F83020524A137853B14A4991F830101C
:10B2E0000B4205D14F4950480978037001B91170DC
:10B2F0004D4B1B784BB1434A92F8302003EA0202CF
:10B300009A4202D1494B01221A703E4B93F83020E9
:10B3100012F0010F0AD093F8313013F0010F05D16C
:10B320003E4BDA78012A01D10132DA70354B93F8BD
:10B33000302012F0020F0AD093F8313013F0020FD0
:10B3400005D1364B1A79012A01D101321A712D4BE0
:10B3500093F8302012F0040F0AD093F8313013F034
:10B36000040F05D12D4B5A79012A01D101325A71AE
:10B37000244B93F8302012F0080F0AD093F83130A4
:10B3800013F0080F05D1254B9A79012A01D101321A
:10B390009A711C4B93F8302012F0100F0AD093F8DA
:10B3A000313013F0100F05D11C4BDA79012A01D18D
:10B3B0000132DA71134B93F8302012F0200F0AD0CB
:10B3C00093F8313013F0200F05D1144B1A7A012A6B
:10B3D00001D101321A720B4B032293F828000DF1B0
:10B3E000100CB0FBF2F2624412F9042C93F8301006
:10B3F000002A83F8311076DA022819D8410119E0C1
:10B40000D80F002018050020DC0D0020980E002029
:10B410002C0E0020A40E0020900E0020F40F00201F
:10B42000280E0020D80D0020220E0020231000201E
:10B43000C11E490141F01601022894BF00200120DD
:10B44000C9B202AA00F026FF9DF80A3013F0400F9F
:10B450000AD0674A674992F8282052001B32885C5C
:10B46000012801D10130885413F0800F0BD06049BE
:10B47000604A91F828100E3112F81100012802D10B
:10B48000013002F8110013F0100F0AD0584A594940
:10B4900092F8282052001B32885C012801D101302B
:10B4A000885413F0200F0BD0514A524B92F82820A9
:10B4B0000E3213F81210012902D1013103F81210D3
:10B4C0004B4B93F82800022801D8410101E0C11E2E
:10B4D000490141F01601C9B2022894BF00200120A1
:10B4E00002AA01F0BDF894B9414B93F82800022854
:10B4F00001D8410101E0C11E490141F00801C9B272
:10B50000022894BF0020012000F0ACFE28B1384D85
:10B51000394B95F828609B5D5BB3354B374A93F800
:10B52000283002EB4312D28912B9334AD35C2BB3D1
:10B53000FEF760FA2E4D314995F828304FF00A0C8D
:10B540009A0001EBC201C9895219526B0CFB01F13F
:10B55000821A002AB8BF52428A420FDD284EF25C9E
:10B5600062B91846FFF74CF995F828300122F254D9
:10B5700004E0FEF73FFA05EB860568631C4E214D9B
:10B5800096F82800002C55F83030B8BF64429C4231
:10B590000BD2FEF791FE96F8283005EBC3056A79C9
:10B5A00082420ED11846002109E0FEF785FE96F88A
:10B5B000283005EBC3056979884202D01846FFF7A9
:10B5C00017F80B4C94F8280000F034F894F8283061
:10B5D0000133DBB2052B84F8283002D9002384F82C
:10B5E0002830FEF707FA024BD86205B0F0BD00BF65
:10B5F00018050020F40F0020E40F0020A40E002006
:10B60000EC0F0020E40D0020024B1A5C0AB9013255
:10B610001A54704764050020024B1A5C0AB10F22CD
:10B620001A54704764050020014B185C704700BF36
:10B630006405002002282DE9F74F044694BF002539
:10B64000012501D8410101E0C11E490141F07C0101
:10B65000C9B2284601AA00F01DFEA54B274603EB00
:10B6600044131E7A16F0400F31D0022C05D8630027
:10B670004FF0020B0BFA03FB06E0A4F1030B4FEAB9
:10B680004B0B022303FA0BFB022C5FFA8BFB9DF89A
:10B69000063005D862004FF0010909FA02F906E008
:10B6A000A4F103094FEA4909012202FA09F9904A73
:10B6B00061018818895842685FFA89F909EA030923
:10B6C0000BEA030BC1F1000AC2F100082EE0022CC4
:10B6D00005D863004FF0020909FA03F906E0A4F166
:10B6E00003094FEA4909022303FA09F9022C5FFA18
:10B6F00089F99DF8063005D862004FF0010B0BFA6E
:10B7000002FB06E0A4F1030B4FEA4B0B012202FA05
:10B710000BFB774A610188185FFA8BFB51F802A096
:10B72000D0F804800BEA030B09EA0309022C06F0A7
:10B730003F0601D8601C00E0A01CC0B2F8F79CFFD7
:10B740006B4B03EB441393F90830002B03DAD0F171
:10B75000010038BF0020731E072B00F2E683DFE8EC
:10B7600013F00800080008000800D101D101D10140
:10B77000D101604B1B5D013B0E2B00F2D683DFE84D
:10B7800013F00F002D025D006D0274007D00960025
:10B79000BD0011016E017401D4039D01AD01AD0323
:10B7A000022C01D8610101E0E11E490141F01401C0
:10B7B00001AAC9B2284600F06DFD4E4B9DF8052048
:10B7C00003EB8403022C9A6001D8610101E0E11EC1
:10B7D000490141F00601C9B2284600F043FD454B3E
:10B7E000022C03EB8403186201D8214601E0E11E1C
:10B7F000C9B20222284600F0CDFC022C01D861011A
:10B8000001E0E11E490141F00601C9B2284640F2BB
:10B81000FF7200F04FFE022C01D9033CE4B2023E5D
:10B82000032228462146F6B200F086FC012E314B59
:10B8300001D8022200E00422DA5576E3BBF1000FC2
:10B8400000F07383022C01D8610101E0E11E49017F
:10B8500041F00201C9B2284600F0CAFC254B04227F
:10B860001A55254B43F824005FE3B9F1000F00F0AF
:10B870005C83204600F050FE062247E3022C01D8EC
:10B88000214601E0E11EC9B20322284600F054FC23
:10B89000022C01D8610101E0E11E490141F00801DB
:10B8A000C9B22846424600F005FE07222EE3B9F150
:10B8B000000F40F03A83022C01D8610101E0E11E43
:10B8C000490141F008010022C9B2284600F0F2FD0A
:10B8D000022C01D8610101E0E11E490141F008019B
:10B8E000C8F10002C9B2284600F0E4FD08220DE3C9
:10B8F000A40E002064050020C00D0020B9F1000F47
:10B9000000F01383022C01D8610101E0E11E49011E
:10B9100041F00201C9B2284600F06AFC022C06463A
:10B9200001D8610101E0E11E490141F00801002256
:10B93000C9B2284600F0BEFDA44B53F82420921B48
:10B94000022C43F8242001D8214601E0E11EC9B2AF
:10B950000322284600F0F0FB022C01D8610101E02F
:10B96000E11E490141F0060188EAE872C9B2A2EB82
:10B97000E872284600F09EFD022C01D8610101E02A
:10B98000E11E4901C9B23246284600F0F9FC022CFA
:10B9900001D9033CE4B200222846214600F0FAFB1C
:10B9A000092243E2284600F0F5FA022C01D8630090
:10B9B00001E0E31E5B00012212FA03F3034200F0F0
:10B9C000B482022C01D8610101E0E11E490141F07D
:10B9D0000201C9B2284600F00BFC7D4B022C43F853
:10B9E000240001D8610101E0E11E490141F0080194
:10B9F0000022C9B2284600F05DFD022C01D8214684
:10BA000001E0E11EC9B20222284600F0C3FB022C6D
:10BA100001D8610101E0E11E490141F0020100226B
:10BA2000C9B2284600F0ACFC022C01D8610101E04B
:10BA3000E11E4901033E0022C9B22846F6B200F0D9
:10BA40009FFC012E00F26182022C01D8214601E008
:10BA5000E11EC9B22846022200F09CFB7EE1B9F14A
:10BA6000000F00F062820B2250E2B9F1000F40F0AB
:10BA70005C82022C01D8610101E0E11E490141F024
:10BA80000201C9B2284600F0B3FB022C064601D8D9
:10BA9000610101E0E11E490141F008010022C9B243
:10BAA000284600F007FD022C01D8610101E0E11EEB
:10BAB00049010222C9B296FBF2F2AAE1284600F03F
:10BAC00069FA022C01D8630001E0E31E5B00012249
:10BAD00012FA03F3034200F0288216E2022C01D886
:10BAE000610101E0E11E49013A4B41F0060103EB1F
:10BAF0008403C9B21A6A284600F0DCFC022C00F26A
:10BB0000088208E2334B1B5D013B0E2B00F20D82D5
:10BB100001A252F823F000BF55BB0008D9BB0008B2
:10BB200037BC000859BC0008B9BC00082BBF00088E
:10BB3000DDBC00082BBF00082BBF00087DBD00083E
:10BB4000A9BD000829BD000831BE0008FDBA0008E3
:10BB5000DDBE0008022C01D8610101E0E11E4901AF
:10BB600041F0140101AAC9B2284600F093FB194B19
:10BB70009DF8052003EB8403022C9A6001D821462E
:10BB800001E0E11EC9B20222284600F003FB022CAC
:10BB900001D8610101E0E11E490141F00601C9B28D
:10BBA000284640F2FF7200F085FC022C01D9033CCC
:10BBB000E4B203222846214600F0BEFA062E01D048
:10BBC000082E01D1022231E104222FE1C00D002014
:10BBD000680F002064050020062E11D1022C01D828
:10BBE000214601E0E11EC9B2954B284603EB8403D0
:10BBF0009A6802F00402002A14BF0522012209E01B
:10BC0000082E09D1022C01D8214601E0E11EC9B25B
:10BC10002846032200F090FA022C01D8610101E0CD
:10BC2000E11E490141F008015246C9B2284600F020
:10BC300041FC03226AE1731FDBB2012B07D8BBF181
:10BC4000000F04D0062E7E4B42D104225FE1002873
:10BC500000F06B810C2259E1052E11D1022C01D884
:10BC6000214601E0E11EC9B2754B284603EB84036F
:10BC70009A6802F00402002A14BF0622022209E098
:10BC8000072E09D1022C01D8214601E0E11EC9B2DC
:10BC90002846032200F050FA022C01D8610101E08D
:10BCA000E11E490141F00801CAF10002C9B228466B
:10BCB00000F000FC052229E1731FDBB2012B09D83B
:10BCC000B9F1000F06D0052E5D4B01D102221EE115
:10BCD0000F221CE1002800F02881E6E5002840F052
:10BCE0002481073EF6B2012E12D9022C01D821463A
:10BCF00001E0E11EC9B2524B284603EB84039A6867
:10BD000002F00402002A14BF0522012200F014FAF6
:10BD1000022C01D8610101E0E11E490141F0080156
:10BD2000C9B22846424625E0002840F0FE80073E82
:10BD3000F6B2012E12D9022C01D8214601E0E11EF3
:10BD4000C9B23F4B284603EB84039A6802F0040211
:10BD5000002A14BF0622022200F0EEF9022C01D8BC
:10BD6000610101E0E11E490141F00801C9B2284624
:10BD7000C8F1000200F09EFB0A22C7E0002800F094
:10BD8000D480022C01D8610101E0E11E490141F09B
:10BD90000201C9B2284600F02BFA294B0B2103EB14
:10BDA000840219559063C0E0002840F0BE80022C48
:10BDB00001D8610101E0E11E490141F00201C9B26F
:10BDC000284600F015FA1F4B002203EB44130833FA
:10BDD000022C06465A7101D8610101E0E11E4901B9
:10BDE00041F0060188EAE872C9B2A2EBE87228467F
:10BDF00000F0C6FA022C01D8610101E0E11E490100
:10BE00000F4BC9B203EB84039B6BF618022396FB1E
:10BE1000F3F2284600F0B4FA022C01D9033CE4B254
:10BE200000222846214600F0B5F90D22044B03E517
:10BE3000284600F0AFF8022C06D8630006E000BFE9
:10BE400064050020A40E0020E31E5B00012212FA0C
:10BE500003F3034269D0364B0E22022C1A5501D847
:10BE6000610101E0E11E490141F00201C9B2284629
:10BE700000F0BEF92F4B022C43F8240001D86101D9
:10BE800001E0E11E490141F008010022C9B2284643
:10BE900000F010FB022C01D8214601E0E11EC9B2DE
:10BEA0000222284600F076F9022C01D8610101E057
:10BEB000E11E490141F002010022C9B2284600F00A
:10BEC0005FFA022C02D86401E1B202E0E11E4901EE
:10BED000C9B22846002200F053FA26E0022C01D80D
:10BEE000214601E0E11EC9B20222284600F052F9C3
:10BEF000022C01D8610101E0E11E490141F0080175
:10BF0000C9B22846002200F0D5FA0E22084B1A5575
:10BF10000BE0033CE4B2064E284606EB87031A7A90
:10BF2000214600F009F90023F355BDE8FE8F00BF5C
:10BF300064050020680F0020154B10B503EB0012BC
:10BF4000926891420EDD8A1AC2F18074A2424FEAD1
:10BF5000001C03DC63445C6812190EE063445A68F9
:10BF6000141B0FE00FDA521AC2F18074A2424FEA9A
:10BF7000001C04DC63445C68A21A5A6003E063445A
:10BF80005A68A4185C60024B03EB0010816010BD7E
:10BF9000FC11002008B5014618B1012804D000208A
:10BFA00006E00121072000E008200A46F8F7A0FC7F
:10BFB00008BD00BF2DE9F041137814460E46C3F3C7
:10BFC0004117054610B10337062F34D0554A02EB0E
:10BFD0004712127B7ABB13F0010F2CD15F2B2AD8AA
:10BFE000514AD25D3ABB13F09F0301D0082B22D1F6
:10BFF000DFF83C8118F8073093B94A4B03EB47123E
:10C00000D17F21B13846F8F793FB032306E003EB19
:10C010004713597A3846F8F78BFB022308F80730A4
:10C02000DFF8108118F807302BB13846FEF7D8FB3F
:10C03000002308F8073015B1012D2ED115E0217825
:10C040002A460720F8F754FC307061782A4607200A
:10C05000F8F74EFC7070A1782A460720F8F748FCE4
:10C06000B070E1780720012214E021780022082036
:10C07000F8F73EFC3070617800220820F8F738FCB1
:10C080007070A17800220820F8F732FCB070E178D7
:10C0900008202A46F8F72CFCF070237813F0010FE3
:10C0A0003ED15F2B3CD803F01E02082A04D0142A8C
:10C0B0002CD0062A34D11BE0242169435B090C20D3
:10C0C00000FB0313A57894F803C0184A4CEA052531
:10C0D0009D50A37813F0080F22D025786D0900FB3E
:10C0E0000515AB586FEA03536FEA1353AB5017E0D3
:10C0F000242255435B090C22A17802FB0353E2780A
:10C1000042EA012209495B185A6009E0242255439A
:10C110005B090C2202FB03530449E2785B181A7294
:10C12000BDE8F081A40E0020E40F0020480E00209E
:10C13000D80F0020EC0F0020022973B50C460546ED
:10C14000164601D84B0101E0CB1E5B0143F01503FD
:10C15000DBB22846694601AA8DF80430FFF72AFFB2
:10C16000022C88BF033C64019DF801C09DF8033098
:10C1700044F01404E4B22846694601AA8DF804404C
:10C180008DF805C08DF806608DF80730FFF712FFB7
:10C190007CBD00BF022973B50C460546164601D882
:10C1A0004B0101E0CB1E5B0143F01503DBB22846D7
:10C1B000694601AA8DF80430FFF7FCFE022C88BF07
:10C1C000033C64019DF801C09DF8023044F0140462
:10C1D000E4B22846694601AA8DF804408DF805C0EE
:10C1E0008DF806308DF80760FFF7E4FE7CBD00BFD8
:10C1F00037B541F001030C466A4601A98DF80030BD
:10C200000546FFF7D7FE9DF806009DF805200002C1
:10C210009DF8073040EA0240184310F4000F18BFA1
:10C2200040F07F405F2C1AD8C4F3411314F01E0471
:10C2300002D0022C13D106E0032202FB0535084A86
:10C240002D01A8580BE0032202FB053520F07F41A9
:10C25000E8B2FFF771FE024B03EB051568683EBDBF
:10C26000FC11002007B541F001036A4601A98DF8D1
:10C270000030FFF79FFE9DF806009DF8073043EA67
:10C28000002010F4006F1CBF6FEA00506FEA1050DE
:10C290000EBD00BF13B541F00103144601A96A4663
:10C2A0008DF80030FFF786FE9DF805109DF80630EA
:10C2B0009DF807202170A27063709DF804001CBDDA
:10C2C000022807B501D8410101E0C11E490141F032
:10C2D0001601C9B2022894BF0020012001AAFFF76D
:10C2E000D9FF9DF80530D80913F0200F18BF40F092
:10C2F00002000EBD022807B501D8410101E0C11EB0
:10C30000490141F01601C9B2022894BF0020012062
:10C3100001AAFFF7BFFF9DF80530C3F3801013F0AB
:10C32000100F18BF40F002000EBD00BF022837B545
:10C3300004460D4601D8410101E0C11E4901C9B2C0
:10C34000294301AA022C94BF00200120FFF7A2FF7D
:10C35000B4235C436D08032304F5807403FB054597
:10C360009DF804102846FCF773FC681C9DF8051026
:10C37000FCF76EFCA81C9DF80610FCF769FC3EBD9E
:10C380005F292DE9F3410D460646144667D8C1F3EF
:10C39000411C11F01E0102D0022960D11EE00322CF
:10C3A00002FB00CC374A4FEA0C1083185B688450BC
:10C3B000E01A0028B8BF4042B0F5000F0ADB9C42EB
:10C3C000CCBF314C314C2F4A1C1902EB0C1201230B
:10C3D000137344E002EB0C12117340E0032707FBD8
:10C3E00000C7284B3801C1587A00C4EB010E013256
:10C3F000BEF1000FB8BFCEF1000E00EB0308BEF592
:10C40000000F24F07F40C8F8044043F8320022DBDC
:10C41000A142CCBF1C4B1D4B3046E318BCF1030FAF
:10C420000CBF4FF0000C4FEA4C1C4FEA23484FEA78
:10C43000232E694601AA8DF807308DF804C08DF8C7
:10C4400005808DF806E0FFF7B5FD0E4B03EB0717EF
:10C4500001233B7303E003EBC20300221A714FEA8E
:10C46000244C23123046694601AA8DF804508DF8F9
:10C4700005C08DF806308DF80740FFF79BFDBDE83D
:10C48000FC8100BFFC110020FFFF7F00010080FF46
:10C4900038B50D4668210446FFF7AAFE15B140F0F5
:10C4A000010201E020F0010220466821FFF768FF49
:10C4B00038BD00BF07B513464FEA222C8DF8041093
:10C4C0004FF0000E694601AA8DF805E08DF806C010
:10C4D0008DF80730FFF76EFD0EBD00BF07B50B46A8
:10C4E00011F01E01024601D0022905D1104619465D
:10C4F0000022FFF745FF0DE04FF0000C694601AA4E
:10C500008DF804308DF807C08DF805C08DF806C091
:10C51000FFF750FD0EBD00BF022838B5044694BF9A
:10C520000025012501D8C1B201E0C11EC9B2022215
:10C530002846FFF72FFE022C01D8610101E0E11E21
:10C54000490141F00801C9B22846FFF7C7FF022C94
:10C5500001D8610101E0E11E490141F00A01C9B2BF
:10C560002846FFF7BBFF38BD07B59DF810C08DF812
:10C5700004108DF80520694601AA8DF806308DF863
:10C5800007C0FFF717FD0EBD30B5022885B0044681
:10C5900001D8430101E0C31E5B0143F00303022CF9
:10C5A00094BF00250125DBB2284603A902AA8DF815
:10C5B0000830FFF7FFFC9DF80E109DF80D209DF848
:10C5C0000F30090241EA024119432046FFF7B4FC4B
:10C5D0001F4B03EB04131B7B002B37D0022C1D4A8F
:10C5E00094BF2346E31E0C2101FB0323022C8CBFC6
:10C5F000242200229B181B7A43BB154822011118E4
:10C6000049681258C1EB020CBCF1000FB8BFCCF165
:10C61000000CBCF5000F05DB8A42CCBF0E4A0F4A66
:10C620008A1802E000EB04100373022C02D86401A4
:10C63000E1B202E0E11E4901C9B2D4B2C2F307235C
:10C640002846C2F307420094FFF78EFF05B030BDC5
:10C65000FC110020480E0020FFFF7F00010080FF3A
:10C6600007B5937892F800E092F801C08DF80410B5
:10C6700001AA69468DF805E08DF806C08DF80730EF
:10C68000FFF798FC0EBD00BF022873B504460E46A6
:10C6900094BF0025012501D8410101E0C11E4901D7
:10C6A00041F01601C9B2284601AAFFF7F3FD9DF833
:10C6B000053016F0010F1ABF6FEA43636FEA536348
:10C6C00003F07F038DF805309DF8053016F0020F5A
:10C6D00014BF43F0200323F02003022C8DF8053013
:10C6E00001D8610101E0E11E490141F0160100237A
:10C6F000C9B2284601AA8DF80630FFF7B1FF7CBD0C
:10C70000022873B504460E4694BF0025012501D8C2
:10C71000410101E0C11E490141F01601C9B228469C
:10C7200001AAFFF7B7FD9DF8053016F0010F14BF01
:10C7300043F0400323F040038DF805309DF80530A9
:10C7400016F0020F14BF43F0100323F01003022C65
:10C750008DF8053001D8610101E0E11E490141F089
:10C7600016010023C9B2284601AA8DF80630FFF74A
:10C7700077FF7CBD73B5B42545434B08032205F50F
:10C78000807502FB0355044628460E46FCF7CAF99D
:10C790008DF80400681CFCF7C5F98DF80500A81C8D
:10C7A000FCF7C0F9022C034601D8610101E0E11E4B
:10C7B0004901C9B23143022C94BF0020012001AAD3
:10C7C0008DF80630FFF74CFF7CBD00BF2DE9FF4719
:10C7D0004D05022804464FEA555594BF4FF0000816
:10C7E0004FF0010801D8410101E0C11E490141F0AB
:10C7F0001801C9B2404603AAFFF74CFD9DF80D9001
:10C8000009F00F0A4FEA1919CA4510DB284604F04F
:10C8100023FFC9EB0A0A0646012000FA0AF00F4678
:10C8200004F02AFF00223C4B04F08CFF11E0284664
:10C8300004F012FFCAEB090A0646012000FA0AF0CA
:10C840000F4604F019FF02460B460020324905F05E
:10C85000A3F802460B463046394605F09DF805F030
:10C86000ABF904F01BFF2AA3D3E9002304F06AFF0D
:10C8700005F0A2F904F012FF0022284B04F062FF39
:10C88000CDE900014FF0FF37BA4600260120B04045
:10C8900004F0F2FE02460B46DDE9000104F052FF0F
:10C8A00005F062F9A0F180027F2A98BF374603465F
:10C8B00006F1010688BF53460E2E01D09A46E5E7E1
:10C8C000022C01D8610101E0E11E490141F0120191
:10C8D0004FF0000CC9B2404603AA8DF80CC08DF889
:10C8E0000D308DF80E70FFF7BBFE022C01D86101F0
:10C8F00001E0E11E490141F00C014046C9B22A465F
:10C90000FFF7D8FD002004B0BDE8F087AFF300804A
:10C9100004560E2DB29DEF3F000060400000204005
:10C92000F7B5304B587E10F0010004D0002068218C
:10C9300040F2231202E068214FF49172FFF720FDCC
:10C9400000207E210346022402460094FFF70CFEDD
:10C95000244B5B7E13F0020F04D00120682140F2CB
:10C96000231203E0012068214FF49172FFF708FDC4
:10C970000022022401207E2113460094FD25FFF7AA
:10C98000F3FD00242BE0E7B2F1B238460136FFF7A1
:10C99000F1FE1D2EF7D1022C94BF0026012601D8EE
:10C9A000790100E0690141F00C01C9B23046FFF79E
:10C9B0001FFC01463846FFF709FF022C01D8790118
:10C9C00000E0690141F01601C9B2304643F2FF129E
:10C9D00001340135FFF76EFD062CEDB201D00026C3
:10C9E000D1E7FEBD04000020084B1868034605E0AF
:10C9F0002C2A02D100221A7003E001331A78002A8F
:10CA0000F6D1024A01331360704700BFB40500201D
:10CA100010B50E4B02461B78ABB10D4B1C7994B18F
:10CA20009C68601CE4180D2A2273986002D03F288D
:10CA300000D851B9064C014604F10C00FDF7E0F9AD
:10CA40000023A36001E0FCF703FB10BDBC0D002038
:10CA5000B405002030B50121044687B02020FFF73F
:10CA6000D7FF002C04DA2D200121FFF7D1FF64420B
:10CA700000230A2194FBF1F201FB124101AD303198
:10CA8000E954591C141E01DD0B46F2E7ED181C4653
:10CA90000121013C15F80109FFF7BAFFB4F1FF3F8E
:10CAA000F6D107B030BD00BF38B50C4D0446A878AC
:10CAB00001214030C0B2FFF7ABFF68780121403060
:10CAC000C0B2FFF7A5FF2078FFF7C4FF6068FFF74B
:10CAD000C1FF0D200121FFF79BFF38BD040000209E
:10CAE00070B5124B06461B78EBB1FCF77FFA104C81
:10CAF000054618B100232371012016E0E36C226D76
:10CB0000934208D21A1992F854200133012032704E
:10CB1000E364207109E004F15400FDF73FF9E56496
:10CB20002065284601E0FCF761FA70BDBC0D0020CD
:10CB3000B40500202DE9F34104460DF10700FFF78D
:10CB4000CFFF002800F0CB808B4B8C4A93F89410D9
:10CB500019BB51789DF80700403188420DD1D3F8B8
:10CB60009810002940F0BB801179012231F00101B9
:10CB700083F8942040F0B380AFE00D2801D01B284B
:10CB800002D100227C4B05E0D3F898207E2A00F2E7
:10CB9000A6800132C3F89820A1E0117931F001019B
:10CBA00003D19DF80700FFF733FF9DF807301F2BD7
:10CBB0000BD9714AD2F898107E297FD8481C891861
:10CBC00081F89C30C2F8980078E0082B08D16A4BB5
:10CBD000D3F89820002A71D0013AC3F898206DE06C
:10CBE0000D2B6BD1644BD3F89830002B66D0634B80
:10CBF0001A79112A15D1587801214030C0B2FFF7B7
:10CC000007FF002503E0585DFFF702FF01355A4B8F
:10CC10000121D3F898209C339542F4D30D20FFF7DF
:10CC2000F7FE554A00231568D2F8987019461A463F
:10CC300033E001290FD002D302292DD122E04E4E3C
:10CC400006F19C00805C202826D09E1986F81C01E5
:10CC50000133012120E0484800F19C0C1CF802C07F
:10CC6000BCF1200F0AD1012B04D91818002180F83B
:10CC70001C110133424D0221ED180DE0181880F807
:10CC80001CC108E03C4E06F19C00805C202803D0CB
:10CC90009E1986F81C0101330132BA42C9D3364AC3
:10CCA0000021981880F81C110120C2F89810156016
:10CCB00082F8A001C2F89C3182F894109DF80730E8
:10CCC0001B2B0CD12D4A2C4B12790021012A83F801
:10CCD0009410C3F8981002D10D20FFF799FE264B4F
:10CCE00093F8A001002878D00022164683F8A021EE
:10CCF0001546DFF8A880072707FB05872048394637
:10CD0000013504F03BF930B9BE797B7916F0010F9B
:10CD1000237049D007E018F806300736002B5ED0A4
:10CD2000FF2DE6D15BE0FFF75FFE23780546042B7D
:10CD30000CD1144904F022F90346D8B1284612490F
:10CD400004F01CF970B1284610490FE00D2B28D1D2
:10CD50000F4904F013F9034660B128460D4904F069
:10CD60000DF908B9012305E00B49284604F006F93E
:10CD7000B0B90223637017E0B4050020040000205E
:10CD8000D0060020592501085D250108612501080C
:10CD9000672501086D250108722501085023010847
:10CDA000284604F0E5F8607016F0020F04D0FFF793
:10CDB0001BFE04F0DDF8A07016F0040F0CD0FFF796
:10CDC00013FE04F0D5F8010EC0F30722C0F30743A9
:10CDD000A17122716371E0700120BDE8FC81002324
:10CDE0002370F9E7704700BFFEE700BFFEE700BF12
:10CDF000FEE700BFFEE700BF704700BF704700BFFF
:10CE0000704700BF704700BF704700BF704700BF4A
:10CE1000704700BF704700BF704700BF704700BF3A
:10CE2000704700BF704700BF704700BF704700BF2A
:10CE3000704700BF704700BF704700BF704700BF1A
:10CE4000704700BF704700BF704700BF704700BF0A
:10CE500008B5024B1B68984708BD00BF240E002090
:10CE600008B5024B1B68984708BD00BFE00F0020C3
:10CE700008B5024B1B68984708BD00BFA00E0020F4
:10CE800008B5024B1B68984708BD00BF640F00201F
:10CE9000704700BF704700BF704700BF704700BFBA
:10CEA000704700BF704700BF704700BF704700BFAA
:10CEB000704700BF704700BF704700BF704700BF9A
:10CEC000704700BF704700BF704700BF704700BF8A
:10CED000704700BF704700BF704700BF704700BF7A
:10CEE000704700BF704700BF704700BF704700BF6A
:10CEF000704700BF704700BF704700BF704700BF5A
:10CF0000704700BF704700BF704700BF704700BF49
:10CF1000704700BF704700BF704700BF704700BF39
:10CF2000704700BF436830B523F470230C680A795A
:10CF300023F48073234343EA0223436082688D68AD
:10CF4000CC680A4B45EA040C02EA03034A794CEA2E
:10CF5000030343EA420383600B7CC26A013B22F471
:10CF60007002DBB242EA0353C36230BDFDF7F1FF4A
:10CF7000002301220274C360036003714371836064
:10CF8000704700BF19B1836843F0010302E0836872
:10CF900023F001038360704719B1836843F4807301
:10CFA00002E0836823F4807383607047C9B212B1D2
:10CFB0004368194302E0436823EA01014160704776
:10CFC000836843F008038360704700BF8068C0F344
:10CFD000C0007047836843F004038360704700BF5C
:10CFE0008068C0F38000704719B1836843F4A003E0
:10CFF00002E0836823F4A003836070478068C0F375
:10D00000805070474368013923F4604343EA413359
:10D010004360704719B1436843F4006302E043681A
:10D0200023F4006343607047092930B511D94FF0EC
:10D03000030C0CFB01FC0725ACF11E0C05FA0CF5EA
:10D0400003FA0CFCC46824EA050343EA0C03C3603A
:10D050000EE04FF0030C0CFB01FC072505FA0CF564
:10D0600003FA0CFC046924EA050343EA0C03036198
:10D07000062A0DD80523013A5A434FF01F0C0CFA2B
:10D0800002FC9140436B23EA0C020A4342631CE01A
:10D090000C2A0DD805235A434FF01F0C233A0CFAE3
:10D0A00002FC9140036B23EA0C020A4302630CE08A
:10D0B00005235A434FF01F0C413A0CFA02FC9140F1
:10D0C000C36A23EA0C020A43C26230BD19B1836805
:10D0D00043F4801302E0836823F480138360704775
:10D0E000C06C80B2704700BF014B1868704700BF2A
:10D0F0004C24014019B1436843F4806302E0436863
:10D1000023F480634360704719B1436843F480534C
:10D1100002E0436823F4805343607047836823F43C
:10D12000E04341EA03038360704700BF19B183689D
:10D1300043F4004302E0836823F4004383607047B4
:10D1400019B1836843F4021302E0836823F40213E5
:10D15000836070478068C0F340507047092930B53C
:10D1600011D94FF0030C0CFB01FC0725ACF11E0C90
:10D1700005FA0CF503FA0CFCC46824EA050343EA3B
:10D180000C03C3600EE04FF0030C0CFB01FC072501
:10D1900005FA0CF503FA0CFC046924EA050343EADA
:10D1A0000C030361836BC3F3015CCCEB020202321C
:10D1B0004FF0050CD2B20CFB02F20CF11A0C0CFA77
:10D1C00002FC914023EA0C030B43836330BD00BF94
:10D1D000836B013923F4401343EA0153836370479F
:10D1E0000A5070472830405880B27047436823F493
:10D1F000400323F4007341EA03034360704700BF18
:10D2000041628262704700BF436823F01F0341EA16
:10D2100003034360704700BF20B1054B9A6842F496
:10D22000000203E0024B9A6822F400029A60704701
:10D2300000240140036819420CBF00200120704700
:10D24000C9430160704700BF4368006810EA1120BD
:10D2500004D0C9B219420CBF00200120704700BFA2
:10D260006FEA11210160704708B5134B98420FD047
:10D2700003F5A053984213D0A3F5C053984219D197
:10D280004FF40070012101F00BFB4FF400700EE031
:10D290004FF48060012101F003FB4FF4806006E051
:10D2A0004FF40040012101F0FBFA4FF4004000214F
:10D2B00001F0F6FA08BD00BF00280140374B0122FB
:10D2C0001A605A6812F0010201D1104664E0027837
:10D2D000012A0BBF1A681A6842F0800222F080020D
:10D2E0001A604378012B04D12C4B1A6842F040029B
:10D2F00003E02A4B1A6822F040021A608378012B5F
:10D3000004D1264B1A6842F0200203E0234B1A682E
:10D3100022F020021A60C378012B04D11F4B1A6837
:10D3200042F0100203E01D4B1A6822F010021A604E
:10D330000379012B04D1194B1A6842F0080203E06B
:10D34000164B1A6822F008021A604379012B04D1A7
:10D35000124B1A6842F0040203E0104B1A6822F0E4
:10D3600004021A608279C37990F808C0920742EAF1
:10D3700003624189437A42EA0C4242EA035201398C
:10D38000064B0A43DA611A6822F001021A605868F3
:10D3900080F0010000F00100704700BF0064004011
:10D3A00090F800C0012202FA0CF23B4B2DE9F04547
:10D3B000D3F8004292B244F00104C3F80042D3F81B
:10D3C0001C42D14301EA0404C3F81C428478A4B986
:10D3D0000CF1480CD3F80C72B0F80AA0C688B0F86B
:10D3E000088085884FEACC0404F1804446EA0A4666
:10D3F00045EA084501EA070715E0012C1AD10CF1AE
:10D40000480CD3F80C72B0F804A0C688B0F80880B5
:10D4100045894FEACC0404F1804446EA0A4645EACD
:10D42000084542EA070704F5C844C3F80C7243F8FC
:10D430003C60656043782BB9174BD3F8044201EA8E
:10D44000040404E0144BD3F8044242EA0404C3F891
:10D450000442838923B9104BD3F81442214006E0DB
:10D46000012B06D10C4BD3F8141242EA0101C3F888
:10D470001412837B012B05D1074BD3F81C120A43EE
:10D48000C3F81C22044BD3F8002222F00102C3F897
:10D490000022BDE8F08500BF006400400322027254
:10D4A000013A002342724FF00102C37142810370BE
:10D4B00043708370C370037143718371704700BF01
:10D4C00019B1054B5A69104303E0034B5A6922EA2C
:10D4D00000005861704700BF00640040364B70B5D3
:10D4E0009968024611F0806F01D000200CE0996825
:10D4F00011F0006F01D0012006E09B6813F0805FFF
:10D5000001D1042056E002202B4B00F11801090143
:10D51000CC5804F00104CC50157A92F809C035B902
:10D52000146864051460CD584CEA050C07E0546893
:10D5300045EA0C0CE4005460CE584CEA060C4CEA68
:10D540000404CC50947A00F1180C4FEA0C1C04F03F
:10D550000F040CF18043947203F5C8435D68010128
:10D5600025F00F055D605D6801F180412C435C6032
:10D57000537B947BD57A1B0443EA0463147B2B43CF
:10D5800043EA042301F5C841C1F88831557C937CF6
:10D59000D47B2D0445EA0365137C45EA040242EA84
:10D5A0000322054BC1F88C215CF8032042F00102F4
:10D5B0004CF8032070BD00BF00640040012810D06B
:10D5C00002D302282CD11AE0164A91689368926817
:10D5D00001F0010103F0020343EA8103C2F3806218
:10D5E0001AE0104A9368916803F48073926801F41A
:10D5F00000719B0943EA1123C2F3C0620CE0094A9F
:10D600009368916803F48033926801F400319B0BB6
:10D6100043EA1143C2F300721343034AD05C7047DC
:10D620000023FAE70064004030240108012808D0F4
:10D6300002D302280FD109E0074B9A6842F080021A
:10D6400008E0054B9A6842F4004203E0024B9A68F6
:10D6500042F400029A6070470064004018B9044B1D
:10D660002022DA6002E0024B20221A61704700BFDC
:10D670000064004010B9064BD86805E0012801D0CD
:10D68000002003E0024B186900F00300704700BF60
:10D6900000640040254B00F11B02120110B5D45864
:10D6A00004F004040C721CB9D3585B0D0B6002E04B
:10D6B000D358DB084B6000F11B021C4B1201D358FE
:10D6C00002F1804203F002034B7202F5C842546833
:10D6D000030104F00F0C81F80AC0526803F1804383
:10D6E000120ACA7403F5C843D3F8B821CA72D3F832
:10D6F000B821120A0A73D3F8B821120C4A73D3F86E
:10D70000B821120E8A73D3F8BC21CA73D3F8BC2196
:10D71000120A0A74D3F8BC21120C4A74D3F8BC3133
:10D720001B0E8B74FFF79AFF10BD00BF0064004012
:10D73000044B1A6842F002021A601868C0F34000F5
:10D74000704700BF00640040054B1A6822F00202D7
:10D750001A60186880F00200C0F34000704700BFF4
:10D7600000640040034B9B6918420CBF002001205D
:10D77000704700BF00640040024B9A6922EA000231
:10D780009A61704700640040202831D00CD80628E8
:10D7900020D004D8042825D0052844D118E0072833
:10D7A0001DD008283FD11FE0B0F5007F2BD005D851
:10D7B00040281FD0B0F5807F35D11FE0B0F5803F05
:10D7C0002CD0B0F5003F2BD0B0F5806F2BD11FE0EF
:10D7D000012201E04FF48072134B9A6023E04FF472
:10D7E0008032F9E7082200E010220F4BDA601AE0DD
:10D7F000082200E010220C4B1A6114E00A4B9A69CF
:10D8000022F0010208E0084B9A6922F0020203E0CC
:10D81000054B9A6922F004029A6104E0082200E0B4
:10D820001022014B5A6070470064004001420CBF57
:10D8300000200120704700BF202808B532D00CD846
:10D84000062821D004D8042826D0052818D119E0AC
:10D8500007281ED0082813D120E0B0F5007F29D07A
:10D8600005D8402820D0B0F5807F09D120E0B0F560
:10D87000803F27D0B0F5003F22D0B0F5806F1BD09D
:10D88000002024E0012101E04FF48071104B9868E2
:10D890001BE04FF48031F9E7082100E010210C4B28
:10D8A000D86812E0082100E01021094B18690CE04B
:10D8B000012102E0022100E00421054B986904E007
:10D8C000102100E00821024B5868FFF7AFFF08BDA8
:10D8D00000640040012108B54FF0007000F0EEFF39
:10D8E0004FF00070002100F0E9FF08BD026800233E
:10D8F00022F001020260036043608360C3602D4B2D
:10D90000984233D011D83C3B984229D006D8283BC6
:10D91000984221D0143398424BD11FE0264B9842B5
:10D9200020D01433984244D11EE0244B98422CD08E
:10D9300008D8A3F5677398421DD003F56273984227
:10D9400037D11DE01E4B984229D0143398422BD07A
:10D95000283B98422DD11DE01A4B12E0194B15E0DF
:10D96000184B18E0174B1BE0164B1EE0154B5A687E
:10D9700042F470021CE0134B5A6842F0706217E0E8
:10D98000114B5A6842F00F0212E00F4B5A6842F0F6
:10D99000F0020DE00C4B5A6842F4706208E00A4B4A
:10D9A0005A6842F4704203E0074B5A6842F470220E
:10D9B0005A6070476C000240440002401C04024060
:10D9C0004404024000000240000402408A6870B52E
:10D9D0000C6A0B6944EA02024C691A438B692243C0
:10D9E000CC6905684E6A42EA030323438C6A3343D9
:10D9F00025F4FE4C23432CF0F00C43EA0C030360A7
:10DA0000CB6843600B6883604B68C36070BD00BF28
:10DA100000238362036043608360C36003614361EA
:10DA20008361C36103624362704700BF19B1036839
:10DA300043F0010302E0036823F001030360704731
:10DA400012B10368194302E0036823EA010101608F
:10DA5000704700BF406880B2704700BF10F0805F21
:10DA600014BF044B044B1B6803420CBF0020012071
:10DA7000704700BF000402400000024010F0805FC9
:10DA800014BF024B024B5860704700BF00040240B5
:10DA90000000024010F0805F14BF044B044B1B6871
:10DAA00003420CBF00200120704700BF0004024069
:10DAB0000000024010F0805F14BF024B024B586020
:10DAC000704700BF0004024000000240044B0022E7
:10DAD0001A605A609A60DA60024A5A61704700BF61
:10DAE00000040140FFFF0700837930B50168027927
:10DAF0004BB3184BCC431D6890F805C004EA0505EC
:10DB00001D605D682C405C60D45844EA0101D1502E
:10DB100002689868D14301EA00009860D868014023
:10DB2000BCF1100FD96007D1996811439960D96889
:10DB300041EA0202DA600BE05CF8031041EA0202FB
:10DB40004CF8032004E0034BD05820EA0101D150E7
:10DB500030BD00BF0004014000230C2283714271DC
:10DB600003600371704700BF024B1A6940EA02026A
:10DB70001A61704700040140034B5B6918420CBFF7
:10DB800000200120704700BF00040140014B586194
:10DB9000704700BF00040140054B1A685B690340F1
:10DBA00001D1184603E010420CBF0020012070474D
:10DBB00000040140014B5861704700BF0004014060
:10DBC000044B1A6802F038021A601A6840EA02022E
:10DBD0001A60704700200240044B1A6822F00802C5
:10DBE0001A601A6840EA02021A6070470020024078
:10DBF000044B1A6822F010021A601A6840EA020206
:10DC00001A60704700200240034B044A5A6002F138
:10DC100088325A60704700BF0020024023016745E8
:10DC2000024B1A6942F080021A61704700200240DC
:10DC3000014BD8698008704700200240014B186AE8
:10DC4000704700BF00200240024BD869C0F340007B
:10DC5000704700BF00200240024B1868C0F340101C
:10DC6000704700BF0020024019B1054B1A691043EC
:10DC700003E0034B1A6922EA00001861704700BFF5
:10DC800000200240012804D1054BD86900F00100B2
:10DC900005E0034BDB6818420CBF002001207047F1
:10DCA00000200240014BD860704700BF00200240B6
:10DCB000094BDA6812F0010F01D001200BE0DA689D
:10DCC00012F0040F01D0022005E0DB6813F0100F02
:10DCD00014BF0320042070470020024013B50446FF
:10DCE0000AE000230193FF3301E0019B013B019314
:10DCF000019B002BF9D1013CFFF7DAFF012802D18B
:10DD0000002CEED100E004B905201CBDF8B5124C82
:10DD1000124B0546A36003F188330F20A3600E4623
:10DD20001746FFF7DBFF042814D1236945F0F805F7
:10DD300043F0100323612E43094B37430B305F80C0
:10DD4000FFF7CCFF012805D0226941F6EF7302EA04
:10DD500003032361F8BD00BF002002402301674593
:10DD600000F8FF1F38B5054640F6FF70FFF7B6FF15
:10DD700004283CD11E4C1F4B40F6FF70A36003F1FA
:10DD80008833A360236943F020032361236943F0B0
:10DD900040032361FFF7A2FF042820D1226941F646
:10DDA000DF7302EA03032361236943F01003236155
:10DDB0001DB1114B4FF0000202E00F4B4FF0A502D6
:10DDC0001A8040F6FF70FFF789FF01280FD0084A3C
:10DDD00041F6EF73116901EA0303136107E00128BB
:10DDE00005D0226941F6DF7302EA0303236138BDDF
:10DDF000002002402301674500F8FF1F10B50446CC
:10DE00000F20FFF76BFF04283DD11F4A1F4BE4434F
:10DE1000936003F1883393601169E3B241F010011C
:10DE2000FF2B116106D01A4A0B301381FFF756FF02
:10DE300004281FD1C4F30723FF2B06D0144A0F2058
:10DE40005381FFF74BFF042814D1C4F30743FF2B82
:10DE500006D00F4A0F209381FFF740FF042809D115
:10DE6000240EFF2C01D1042006E0094B0F20DC8199
:10DE7000FFF734FF012806D0034A41F6EF7311691A
:10DE800001EA0303136110BD00200240230167452E
:10DE900000F8FF1F70B504460F200E46FFF71EFF67
:10DEA000042815D10B4D0C4B0B30AB6003F18833BC
:10DEB000AB602B6943F010032B612680FFF70EFF48
:10DEC000012805D02A6941F6EF7302EA03032B61AA
:10DED00070BD00BF002002402301674570B50446B5
:10DEE0000F200E46FFF7FAFE042810D1084D0B3024
:10DEF0002B6943F001032B612680FFF7EFFE012819
:10DF000005D02A6941F6FE7302EA03032B6170BD56
:10DF10000020024070B504460F200E46FFF7DEFEDB
:10DF2000042818D10C4DB3B22A690B3042F001021B
:10DF30002A612380FFF7D2FE042804D1360C6680C4
:10DF40000B30FFF7CBFE012805D02A6941F6FE739E
:10DF500002EA03032B6170BD0020024010B540F6B9
:10DF6000FF70FFF7BBFE04282CD1174C174B40F66F
:10DF7000FF70A36003F18833A360236943F020039B
:10DF80002361236943F040032361FFF7A7FE0428C0
:10DF900010D1226941F6DF7302EA0303236123698A
:10DFA0004FF0A50243F010032361094B0B301A8098
:10DFB000FFF794FE012805D0226941F6EF7302EACB
:10DFC0000303236110BD00BF002002402301674509
:10DFD00000F8FF1F10B540F6FF70FFF77FFE042822
:10DFE00014D10B4C40F6FF70236943F00403236106
:10DFF000236943F040032361FFF770FE012805D039
:10E00000226941F6FB7302EA0303236110BD00BFDE
:10E010000020024038B5054640F6FF70FFF75EFE6F
:10E02000042815D10B4C40F6FF70236943F002031E
:10E0300023616561236943F040032361FFF74EFECE
:10E04000012805D0226941F6FD7302EA030323612A
:10E0500038BD00BF00200240CB78F0B513F0100FA0
:10E0600018BF8A78098803F00F0C18BF4CEA020C1D
:10E0700011F0FF0F1AD0046800220126964006EA2C
:10E080000105B5420ED196000F27B7400CFA06F6EF
:10E0900024EA07043443282B01D1456102E0482BD0
:10E0A00008BF05610132082AE7D10460FF291CD9A5
:10E0B0004468002202F108050126AE4006EA010587
:10E0C000B5420ED196000F27B7400CFA06F624EAA7
:10E0D00007043443282B01D1456102E0482B08BFD7
:10E0E00005610132082AE5D14460F0BD0423C37004
:10E0F000022383704FF0FF33038070478368194217
:10E100000CBF002001207047806880B2704700BFBC
:10E11000C36819420CBF002001207047C06880B25C
:10E12000704700BF01617047416170470AB10161EA
:10E1300000E04161704700BFC160704741F4803327
:10E14000836181618361836983697047064A10B581
:10E1500014684FF6807341EA001104EA030341EAB0
:10E160000303136010BD00BF00000140014B1860A5
:10E17000704700BF1C0020420304154A00F4401CF5
:10E180001B0CBCF5401F30B5546806D1556824F00F
:10E19000706425F07065556011E010F4801F06D0A2
:10E1A000C0F303424FF0030C0CFA02F203E0420DFD
:10E1B000120113FA02F224EA020444F0706419B165
:10E1C000400D000183401C43014B5C6030BD00BF2B
:10E1D0000000014001F003039B000F229A4010FA57
:10E1E00003F310B58908074C023154F8210020EAE6
:10E1F000020244F8212054F82120134344F821302E
:10E2000010BD00BF000001400120014608B500F02C
:10E2100047FB0120002100F043FB08BD08B5264B59
:10E2200098422BD00CD8A3F5006398421AD003F57E
:10E23000806398421CD0A3F5006398423AD10BE06A
:10E240001E4B984226D003F58063984228D0A3F550
:10E25000006398422ED117E00420012100F020FB3A
:10E26000042024E00820012100F01AFB08201EE011
:10E270001020012100F014FB102018E020200121C3
:10E2800000F00EFB202012E04020012100F008FBEE
:10E2900040200CE08020012100F002FB802006E0FD
:10E2A0004FF48070012100F0FBFA4FF480700021E0
:10E2B00000F0F6FA08BD00BF00140140001C014048
:10E2C0000B4B4FF0FF316FF07042C3F88010C3F872
:10E2D0008420C3F88011C3F88421002303F1C00116
:10E2E000034A013300200F2B42F82100F6D170477A
:10E2F00000E100E0094B4FF0206058600848002220
:10E300004FF0FF319A60D8601A615A619A61DA6100
:10E310001A625A629962D9621963704700ED00E08F
:10E320000000FA0540F0BE60024B40F42020D860A7
:10E33000704700BF00ED00E030B5C27803787AB3D3
:10E340001C4A4178D2684FF00F0CD243C2F302222C
:10E350002CFA02FCC2F104029140807803F003021F
:10E360000CEA000C4CEA010CD2004FEA0C1CFF2016
:10E3700090400CFA02FC012403F01F02944099081B
:10E380000D4AC03152F821500CEA000C25EA000079
:10E390004CEA00005B0942F8210042F8234008E003
:10E3A00003F01F02012191405B09034A203342F828
:10E3B000231030BD00ED00E000E100E00023C37059
:10E3C0000370437083707047024B5868C0F3093084
:10E3D000704700BF00ED00E0012200F01F0312FAB9
:10E3E00003F34009044A403052F820001840984294
:10E3F00014BF00200120704700E100E0014B1860CD
:10E40000704700BF00EF00E000F01F0301229A40B8
:10E410004009024B603043F82020704700E100E0E3
:10E42000024B58688005800D704700BF00ED00E08A
:10E43000012200F01F0312FA03F34009044A80305E
:10E4400052F820001840984214BF00200120704765
:10E4500000E100E0014B1868704700BF00ED00E0EC
:10E4600021F0604121F07F01014B01439960704729
:10E4700000ED00E0014A024BDA6070470400FA0543
:10E4800000ED00E0014A024BDA6070470100FA0536
:10E4900000ED00E019B1054B1A69104303E0034B8E
:10E4A0001A6922EA00001861704700BF00ED00E021
:10E4B00000F01F00012313FA00F019B1044B5A6A4F
:10E4C000104303E0024B5A6A22EA00005862704788
:10E4D00000ED00E0144B70B5DC684FF0FF0CE44336
:10E4E000C4F302242CFA04F5C4F1040411FA04F470
:10E4F000C0F30126F6000CFA06FC02EA050545EA1F
:10E500000404240114FA06F6C0F38110063053F80F
:10E51000202022EA0C0243F8202053F82020164342
:10E5200043F8206070BD00BF00ED00E0C0F3832021
:10E5300001238340044A506A03EA0000984214BF52
:10E5400000200120704700BF00ED00E000F01F0038
:10E5500001228240024B59680A435A60704700BF4B
:10E5600000ED00E000F01F020123013A13FA02F26D
:10E57000024B59680A435A60704700BF00ED00E043
:10E58000C0F3833001238340044A506A03EA000049
:10E59000984214BF00200120704700BF00ED00E04A
:10E5A000C0F3814313B90A4BD86A10E0012B0CD198
:10E5B000074AC0F30153906ADA00D040022B14BF1F
:10E5C00000F00F0000F0FF0001E0014B186B7047F6
:10E5D00000ED00E010F4800F0BBF024B014B586BB5
:10E5E000986B704700ED00E008B5F5F7C1FD08BD78
:10E5F00008B50001F5F7B9FD08BD00BF08B5F5F78E
:10E60000B2FD08BD08B5F5F7ACFD08BD08B5F5F7D6
:10E61000A6FD08BD08B5F5F7A0FD08BD0D4B0E4AD7
:10E62000196841F001011960596801EA02025A6053
:10E630001A6822F0847222F480321A601A6822F476
:10E6400080221A605A6822F4FE025A6000229A6000
:10E65000704700BF001002400000FFF80C4BB0F5FF
:10E66000803F1A6822F480321A601A6822F48022ED
:10E670001A6003D0B0F5802F08D103E01A6842F485
:10E68000803202E01A6842F4A0221A60704700BF8C
:10E6900000100240034B1A6822F0F80242EAC0025E
:10E6A0001A60704700100240014B1860704700BFAD
:10E6B00000004242044B5A6822F47C1240EA0202F3
:10E6C0000A435A60704700BF00100240014B1860B7
:10E6D000704700BF60004242034B5A6822F00302B9
:10E6E00040EA02025A60704700100240024B58682C
:10E6F00000F00C00704700BF00100240034B5A6846
:10E7000022F0F00240EA02025A6070470010024014
:10E71000034B5A6822F4E06240EA02025A607047F2
:10E7200000100240034B5A6822F4605242EAC002D1
:10E730005A6070470010024019B1054B1A78104317
:10E7400003E0034B1A7822EA00001870704700BFFC
:10E7500009100240014B1860704700BFD8004242C8
:10E76000034B5A6822F4404240EA02025A60704762
:10E7700000100240064B002201281A701A7002D0C5
:10E78000042804D101E0187001E005221A707047D6
:10E7900020100240014B1860704700BF80044242C5
:10E7A000024B1A6A40EA02021A62704700100240E5
:10E7B000014B1860704700BF3C0442421F4B10B52C
:10E7C0005A6802F00C02042A13D0082A11D15A68A0
:10E7D0005968C2F38342023211F4803F03D05B6870
:10E7E00013F4003F01D0164B00E0164B5A43026071
:10E7F00001E0144B0360114A134B51680468C1F3E4
:10E800000311595C34FA01F141605468C4F3022CDD
:10E8100013F80C4031FA04F484605468C4F3C22C39
:10E8200013F80CC021FA0CF1C1605268C2F38132B6
:10E830009B181B7CB1FBF3F1016110BD001002407D
:10E8400000093D0000127A003824010819B1054B77
:10E850005A69104303E0034B5A6922EA00005861E9
:10E86000704700BF0010024019B1054B9A69104370
:10E8700003E0034B9A6922EA00009861704700BFE9
:10E880000010024019B1054BDA69104303E0034B55
:10E89000DA6922EA0000D861704700BF0010024028
:10E8A00019B1054BDA68104303E0034BDA6822EA3A
:10E8B0000000D860704700BF0010024019B1054B3E
:10E8C0001A69104303E0034B1A6922EA0000186139
:10E8D000704700BF00100240014B1860704700BF36
:10E8E00040044242014B1860704700BF4C00424256
:10E8F000014B1870704700BF071002404309012BFD
:10E9000002D1084B1B6805E0022B0BBF054B054BE2
:10E910001B6A5B6A00F01F0033FA00F000F0010090
:10E92000704700BF0010024008B53120FFF7E6FF36
:10E93000094B18705A6801325A601A7822B95A681D
:10E9400040F2FF139A42F0D13120FFF7D7FF003891
:10E9500018BF012008BD00BF58070020024B5A6AAB
:10E9600042F080725A62704700100240034B9B686D
:10E9700018420CBF00200120704700BF0010024069
:10E98000014B1870704700BF0A1002400B884A887C
:10E99000B1F804C01A43CB8842EA0C02B1F808C0AF
:10E9A0001A434B8930B542EA0C028D89B0F800C099
:10E9B000CC891A432A4322430CF4415313439BB29C
:10E9C0000380838B23F400631B041B0C83830B8A5B
:10E9D000038230BD00234FF00702C381028203800F
:10E9E00043808380C380038143818381704700BF5C
:10E9F00000234381038043808380C3804FF0020360
:10EA00000381704721B103889BB243F0400304E0C7
:10EA1000038823F040031B041B0C0380704700BFD6
:10EA200021B1838B9BB243F4806304E0838B23F496
:10EA300080631B041B0C8383704700BF09090123FB
:10EA400013FA01F189B21AB183889BB2194303E02A
:10EA500083889BB223EA0101818070471AB18388C1
:10EA60009BB2194303E083889BB223EA01018180B2
:10EA7000704700BF81817047808980B2704700BFB6
:10EA80004FF6FF63994205D003889BB243F480732D
:10EA9000038002E0038819400180704721B1838818
:10EAA0009BB243F0040304E0838823F004031B04B7
:10EAB0001B0C8380704700BF038823F400631B0492
:10EAC0001B0C038003889BB241EA03030380704759
:10EAD00003889BB243F480530380704721B10388BD
:10EAE0009BB243F4005304E0038823F400531B0457
:10EAF0001B0C0380704700BF012914BF008B808A64
:10EB000080B27047008A80B2704700BFB1F5804F75
:10EB100004D103889BB243F4804304E0038823F4C8
:10EB200080431B041B0C0380704700BF03891942FC
:10EB30000CBF002001207047202906D103890388DB
:10EB40009BB243F04003038008E0402901D008292C
:10EB500001D1038902E0C94389B20181704700BF36
:10EB6000012301F00F0213FA02F2B0F804C0008989
:10EB70001FFA8CFC80B2104006D009098B401CEAB9
:10EB8000030F0CBF00200120704700BF552906D19C
:10EB9000038903889BB243F0400303800DE05629AC
:10EBA00001D0532901D1038907E001F00F010123AE
:10EBB00013FA01F1C94389B201817047838BF0B523
:10EBC00023F47A6323F01F031B041B0C83834FF091
:10EBD000020303840B89868B022B87B004460D4603
:10EBE000B6B201D1002225E001A88F88FFF7E6FD2B
:10EBF000EB88002F0CBF01270227B3F5007F29897E
:10EC0000019A06D1A3F5FB7353430902B3FBF1F359
:10EC100005E00A2349015A434F43B2FBF7F305339A
:10EC20000A229BB2B3FBF2F303F001021202C3F318
:10EC30004F0392B2991E89B2FE2928BF002228BF35
:10EC40000223E98842EA03030B439BB223842B8807
:10EC50006A8846EA0303A98843F4006313436A8978
:10EC60000B4313439BB2A38307B0F0BD08B5154B0C
:10EC700098421BD003F57443984204D0A3F578431F
:10EC800098421DD10AE001214FF48050FFF708FEA1
:10EC90004FF480500021FFF703FE11E04FF4804055
:10ECA0000121FFF70BFE4FF4804006E04FF40040D7
:10ECB0000121FFF703FE4FF400400021FFF7FEFDA6
:10ECC00008BD00BF003C0040042804D1054B1A6871
:10ECD00042F0040203E0034B1A6822F004021A60B7
:10ECE000704700BF10E000E0014B5860704700BF64
:10ECF00010E000E0012804D1084B1A6842F001023C
:10ED000006E010F1020F05D1044B1A6822F001024F
:10ED10001A6002E0014B00229A60704710E000E0A8
:10ED200020B1054B1A6842F0020203E0024B1A6858
:10ED300022F002021A60704710E000E0014B986870
:10ED4000704700BF10E000E0C308022B0BBF044B6C
:10ED5000034B1B68DB6833FA00F000F001007047DA
:10ED600010E000E0038803F08F0303800388B1F80C
:10ED700006C04A889BB243EA0C0313439BB203804C
:10ED80008B8883850B880385064B984203D003F557
:10ED90000063984201D10B7A03864FF0010383820E
:10EDA000704700BF002C0140038C2DE9F04123F097
:10EDB00001031B041B0C0384038C0A894C8823F079
:10EDC00002031C4E14431B048288B1F806C0058B55
:10EDD0001B0CA4B2B04244EA030392B20C88ADB259
:10EDE000A0F834C003D006F50066B04218D18E8971
:10EDF0004F89B1F80E804FF6F77C03EA0C0C4CEA11
:10EE0000070748EA06064FF6FB73898847F6FF4C6A
:10EE100002EA0C0C07EA0303B2B20B4342EA0C020B
:10EE20004FF68F7105EA010121438280018303843B
:10EE3000BDE8F081002C0140038C2DE9F04123F066
:10EE400010031B041B0C0384028CB1F808C022F0D1
:10EE5000200212048488120C4B8842EA0C1242EA07
:10EE60000313A2B21B4C068BB1F806C0A0420D885A
:10EE7000B6B29BB2A0F838C003D004F50064A0423B
:10EE80001BD1B1F80A804FF67F748F8903EA04041E
:10EE900047F2FF3C02EA0C0C44EA0814CA894FF618
:10EEA000BF73898804EA03034CEA870C43EA011321
:10EEB0004CEA82023C469BB292B248F6FF7106EAE7
:10EEC000010141EA052189B2828001830384BDE802
:10EED000F08100BF002C0140038C2DE9F04123F4A8
:10EEE00080731B041B0C0384028CB1F808C022F44D
:10EEF000007212048488120C4B8842EA0C2242EA07
:10EF00000323A2B21A4C868BB1F806C0A0420D882A
:10EF1000B6B29BB2A0F83CC003D004F50064A04296
:10EF20001BD1B1F80A804FF2FF748F8903EA040401
:10EF300044F6FF7C02EA0C0C44EA0824CA894FF626
:10EF4000FF33898804EA03034CEA071C43EA0123E0
:10EF50004CEA02123C469BB292B24FF68F7106EA1F
:10EF600001012943828081830384BDE8F08100BFD1
:10EF7000002C0140038CF0B523F480531B041B0CC0
:10EF80000384B1F806C0078C0C8882880D89868BB3
:10EF90004B88A0F840C0DFF848C0BFB2604592B2CD
:10EFA000B6B203D00CF5006C604505D19204898996
:10EFB000920C42EA811292B24DF6FF7C07EA0C0CE9
:10EFC00048F6FF7106EA01014CEA053C41EA0421DA
:10EFD0004CEA033389B29BB2828081830384F0BD03
:10EFE000002C0140B1F802C00B888A884CEA030368
:10EFF000B1F806C013430A8943EA0C03B1F80AC00A
:10F0000013438A8943EA0C0313439BB2A0F84430AC
:10F01000704700BF00234FF0FF32037243808280AD
:10F020000380C380704700BF0023C38103804380F7
:10F030008380C380038143818381704700234FF025
:10F0400001020381038043808280C380704700BF38
:10F0500000238381038043808380C38003814381B5
:10F06000704700BF21B103889BB243F0010304E065
:10F07000038823F001039B059B0D0380704700BFAD
:10F0800039B1B0F844306FEA43436FEA53439BB25F
:10F0900003E0B0F844305B045B0CA0F844307047E8
:10F0A0001AB183899BB2194303E083899BB223EA97
:10F0B00001018181704700BF818270470A43A0F837
:10F0C000482070471AB183899BB2194303E08389B2
:10F0D0009BB223EA01018181704700BF038923F0BD
:10F0E00007031B041B0C0381704700BFB0F808C066
:10F0F0005FFA8CFC41EA0C0C42EA0C0C4CEA032C43
:10F100001FFA8CFCA0F808C0704700BF10B5044679
:10F11000FFF7ECFF23899BB243F48043238110BDAA
:10F1200010B50446FFF7E2FF238923F077031B04A1
:10F130001B0C43F07703238110BD00BF0185828241
:10F14000704700BF038823F070039B059B0D41EAC5
:10F1500003030380704700BF038923F070031B047F
:10F160001B0C41EA03030381704700BF10B504463E
:10F17000FFF7F2FF23899BB243F00703238110BD01
:10F1800030B50489B0F818C0058C2CF4407CADB2C1
:10F190002CF0030C24F007044FEA0C4C25F0220558
:10F1A00042EA050524044FEA1C4C45EA0315240CE9
:10F1B0004CF4807C21434CF0010CADB20181A0F8ED
:10F1C00018C0058430BD00BF038B23F070031B04FF
:10F1D0001B0C41EA03030383704700BF038B23F436
:10F1E000E0431B041B0C43EA01239BB203837047DB
:10F1F000838B23F070031B041B0C41EA03038383FE
:10F20000704700BF838B23F4E0431B041B0C43EACD
:10F2100001239BB28383704721B103889BB243F0E3
:10F22000800304E0038823F080039B059B0D03808B
:10F23000704700BF21B183889BB243F0040304E010
:10F24000838823F004031B041B0C8380704700BFDA
:10F2500021B183889BB243F0080304E0838823F044
:10F2600008031B041B0C8380704700BF21B18388F7
:10F270009BB243F0010304E0838823F001031B04E5
:10F280001B0C8380704700BF038B23F008031B0413
:10F290001B0C41EA03030383704700BF038B23F475
:10F2A00000631B041B0C43EA01239BB203837047DA
:10F2B000838B23F008031B041B0C41EA03038383A5
:10F2C000704700BF838B23F400631B041B0C43EACD
:10F2D00001239BB283837047038B23F004031B0439
:10F2E0001B0C41EA03030383704700BF038B23F425
:10F2F00080631B041B0C43EA01239BB2038370470A
:10F30000838B23F004031B041B0C41EA0303838358
:10F31000704700BF838B23F480631B041B0C43EAFC
:10F3200001239BB283837047038B23F080031B046C
:10F330001B0C41EA03030383704700BF038B5B048C
:10F340005B0C43EA01239BB203837047838B23F05A
:10F3500080031B041B0C41EA03038383704700BF37
:10F36000838B5B045B0C43EA01239BB2838370476E
:10F37000038C23F002031B041B0C41EA03030384E8
:10F38000704700BF038C23F008031B041B0C41EAE9
:10F3900003030384704700BF038C23F020031B0486
:10F3A0001B0C43EA01139BB203847047038C23F0C8
:10F3B00080031B041B0C43EA01139BB203847047B8
:10F3C000038C23F400731B041B0C43EA01239BB240
:10F3D00003847047038C23F400631B041B0C43EA73
:10F3E00001239BB203847047038C23F400531B0456
:10F3F0001B0C43EA01339BB20384704701238B400B
:10F400008A40018C89B221EA03030384018C0A43F8
:10F4100092B20284704700BF04238B408A40018C63
:10F4200089B221EA03030384018C0A4392B2028465
:10F43000704700BF01238B40B0F820C010B51FFA01
:10F440008CFC2CEA0303038409B1082909D1183084
:10F45000490844584FF68F7304EA03034350435856
:10F460000CE004391830C1F34E01445848F6FF73DC
:10F4700004EA030343501202435892B243EA0202E1
:10F48000425010BD21B103889BB243F0020304E057
:10F49000038823F002039B059B0D0380704700BF88
:10F4A00021B103889BB243F0040304E0038823F0F6
:10F4B00004039B059B0D0380704700BF21B1838827
:10F4C0009BB243F0800304E0838823F080031B0495
:10F4D0001B0C8380704700BF038823F008039B0543
:10F4E0009B0D038003889BB241EA030303807047AE
:10F4F000838823F070031B041B0C838083889BB2DA
:10F5000041EA030383807047038923F007031B0448
:10F510001B0C038103899BB241EA030303817047FB
:10F52000038923F080031B041B0C038103899BB216
:10F5300041EA0303038170478184704781857047E6
:10F54000818670470187704781877047A0F8401017
:10F55000704700BF038B23F00C031B041B0C0383B9
:10F56000038B9BB241EA030303837047038B23F4AD
:10F5700040631B041B0C0383038B9BB243EA0123F0
:10F580009BB20383704700BF838B23F00C031B04E3
:10F590001B0C8383838B9BB241EA030383837047F5
:10F5A000838B23F440631B041B0C8383838B9BB2EC
:10F5B00043EA01239BB28383704700BF0388DBB219
:10F5C000038003889BB241EA03030380704700BFB6
:10F5D000808E80B2704700BF008F80B2704700BF3E
:10F5E000808F80B2704700BFB0F8400080B2704793
:10F5F000808C80B2704700BF008D80B2704700BF22
:10F60000038A19420CBF002001207047C94389B208
:10F6100001827047038A828911EA030092B203D003
:10F6200011420CBF00200120704700BFC94389B2BE
:10F6300001827047B0F820C010B52CF0010C4FEAE1
:10F640000C4C4FEA1C4CA0F820C0048BB0F820C032
:10F65000A4B21FFA8CFC24F0F30442EA04042CF058
:10F66000020C44EA03144CF0010C4CEA010CA4B265
:10F670000483A0F820C010BDB0F820C010B52CF055
:10F68000100C4FEA0C4C4FEA1C4CA0F820C0B0F80C
:10F6900018C0048C2CF4407CA4B24FEA0C5C4FEAF6
:10F6A0001C5C24F020044CEA022C44F010044CEAC8
:10F6B000033C44EA01141FFA8CFCA4B2A0F818C061
:10F6C000048410BD38B50D46602D1146044603D1A3
:10F6D0000122FFF7D1FF02E00122FFF7ABFF29462D
:10F6E0002046FFF739FD23899BB243F007032381AE
:10F6F00038BD00BFF8B50C46A2884988B4F800C0F0
:10F70000054600290CBF02270027012A0CBF02264C
:10F7100001262389BCF1000F10D1FFF78BFF28468B
:10F72000E188FFF717FF2846394632462389FFF75D
:10F73000A3FF2846E188FFF719FF0FE0FFF79CFFC2
:10F740002846E188FFF712FF2846394632462389CA
:10F75000FFF770FF2846E188FFF7FCFEF8BD00BF09
:10F7600038B50B880C4605464BB94988A2882389D1
:10F77000FFF760FF2846E188FFF7ECFE53E0042B1B
:10F7800009D14988A2882389FFF776FF2846E188B6
:10F79000FFF7ECFE47E0082BB1F802C0B1F804E037
:10F7A000098920D1028C22F480721204120C028486
:10F7B000838B028C9BB292B223F0F30322F400728B
:10F7C00043EA011142EA0C2C89B21FFA8CFC41EA8F
:10F7D0000E0E4CF4807CA0F81CE0A0F820C0E1885C
:10F7E000FFF7D2FE1FE0028C22F480521204120CAA
:10F7F0000284838B028C23F4407392B21B051B0D91
:10F8000022F4005243EA0E2342EA0C3C43EA01335D
:10F810001FFA8CFC9BB24CF4805C8383A0F820C060
:10F82000E188FFF7BDFE38BD08B52D4B984237D0B3
:10F830000BD8A3F50063984226D003F58063984265
:10F8400028D0B0F1804F4AD118E0264B984233D0EF
:10F8500004D8A3F58063984241D127E0224B984217
:10F8600004D003F50063984239D12EE04FF40060D4
:10F870000121FFF715F84FF400602DE0012001464B
:10F88000FFF71CF801201CE002200121FFF716F809
:10F89000022016E004200121FFF710F8042010E0F8
:10F8A00008200121FFF70AF808200AE010200121B2
:10F8B000FFF704F8102004E020200121FEF7FEFFEE
:10F8C00020200021FEF7FAFF09E04FF4005001214B
:10F8D000FEF7E6FF4FF400500021FEF7E1FF08BD00
:10F8E000000C004000140040002C014000238381E4
:10F8F0004FF416528380C38003814FF00C030260E3
:10F90000438170470A8810B54C88B1F804C0038A57
:10F91000C98844EA020242EA0C0223F470630A43F3
:10F920001B041B0C92B242EA0303038210BD00BF0A
:10F930000023C380038043808380704721B1838983
:10F940009BB243F4005304E0838923F400531B0467
:10F950001B0C8381704700BF01F01F034FF0010CA7
:10F96000C1F3421161450CFA03F301D10C3004E0FC
:10F97000022901D1103000E014301AB1026842EAC5
:10F98000030302E0026822EA03030360704700BF3A
:10F990001AB1838A9BB2194303E0838A9BB223EA9C
:10F9A00001018182704700BF038A23F00F031B040B
:10F9B0001B0C0382038A9BB241EA03030382704754
:10F9C000838923F400631B041B0C838183899BB20E
:10F9D00041EA03038381704721B183899BB243F0DD
:10F9E000020304E0838923F002031B041B0C8381C0
:10F9F000704700BF038A23F020031B041B0C038203
:10FA0000038A9BB241EA03030382704721B1038A50
:10FA10009BB243F4804304E0038A23F480431B0435
:10FA20001B0C0382704700BFC905C90D8180704758
:10FA30008088C005C00D704783899BB243F00103E5
:10FA400083817047038BDBB20383038B9BB243EA52
:10FA500001230383704700BF038B03F47F430383B9
:10FA6000038B9BB241EA03030383704721B1838A6E
:10FA70009BB243F0200304E0838A23F020031B049D
:10FA80001B0C8382704700BF21B1838A9BB243F075
:10FA9000100304E0838A23F010031B041B0C8382F1
:10FAA000704700BF21B1838A9BB243F0080304E092
:10FAB000838A23F008031B041B0C8382704700BF5A
:10FAC000838A23F004031B041B0C8382838A9BB26A
:10FAD00041EA03038382704721B1838A9BB243F0DA
:10FAE000020304E0838A23F002031B041B0C8382BD
:10FAF000704700BF038819420CBF002001207047E7
:10FB0000C94389B2018070474FF0010CC1F3421222
:10FB100001F01F0362450CFA03F301D1828903E06F
:10FB2000022A0CBF028A828A92B21340028892B2E1
:10FB30000BB9184607E0090A012313FA01F1114233
:10FB40000CBF002001207047090A01238B40DB43D2
:10FB50009BB20380704700BF038ACA8823F44053D6
:10FB60001B041B0C1343038283898A8830B5044627
:10FB700008890D4623F4B053498940EA020223F074
:10FB80000C030A431B041B0C92B242EA0303A38139
:10FB9000A38AAA8923F440731B041B0C134387B068
:10FBA000A38201A8FEF70AFE0E4B2A689C420CBFF6
:10FBB000049B039B1921594392006423B1FBF2F18A
:10FBC000B1FBF3F21201100903FB101109013231EC
:10FBD000B1FBF3F303F00F0343EA020292B2228176
:10FBE00007B030BD0038014008B5214B98422BD0FA
:10FBF00008D8A3F50063984216D003F580639842B5
:10FC000034D119E01B4B984226D003F56843984243
:10FC10002CD101214FF48040FEF742FE4FF480408A
:10FC20000021FEF73DFE21E04FF400300121FEF7F8
:10FC300045FE4FF4003016E04FF480200121FEF71E
:10FC40003DFE4FF480200EE04FF400200121FEF72E
:10FC500035FE4FF4002006E04FF480100121FEF73E
:10FC60002DFE4FF480100021FEF728FE08BD00BFD6
:10FC7000004C004000500040684620F007018D46CF
:10FC800001B5002303E00B495958995004330A4A3F
:10FC90000A4998188842F6D3094B02E0002243F83B
:10FCA000042B084A9342F9D3F4F79CFABDE80140CB
:10FCB00085467047802501080000002028020020AA
:10FCC000280200206412002010B5074C20B92268D9
:10FCD0004FF00103138205E0044B1B681B68984733
:10FCE00020680A3010BD00BFAC1100206811002050
:10FCF00010B50A4B0A4A1B685178DA7891420AD348
:10FD0000997841B99C8834B99A72064B1B685B6834
:10FD10009847204600E0022010BD00BFAC11002033
:10FD2000000100206811002010B5074C20B922689E
:10FD30004FF00103138205E0044B1B689B68984752
:10FD400020680C3010BD00BFAC11002068110020ED
:10FD500038B50E4C0E4B22681B68D1789B695079E0
:10FD6000984723689A7A7AB170B91A7962B99D78FE
:10FD700055B9084B1B68DB689847236828465979B2
:10FD8000DA78D9721A7300E0022038BDAC11002075
:10FD9000441100206811002008B50246244B20B908
:10FDA0001B684FF00201198240E0224A4FF0000127
:10FDB0001B681180197811F07F0113D15B7A13F061
:10FDC000200F03D0117841F00201117013F0400FA1
:10FDD000184B15BF1A781A7822F0010242F001027E
:10FDE0001A701EE0012921D0022901D000221DE055
:10FDF000597911F0800F01F00F0306D00E4951F828
:10FE0000233003F03003102B06E00B4951F8233068
:10FE100003F44053B3F5805F03D1137843F001033B
:10FE20001370064B1B681B699847024A104608BDB1
:10FE3000AC1100205C120020005C00406811002022
:10FE400010B51E4B19684A7912F0800F22F080031A
:10FE500005D01B4850F8230000F0300004E018489B
:10FE600050F8230000F44050164C94F800C063454D
:10FE700022D24C8804BBF8B1897AE9B112F0800F24
:10FE800009D00F4948F6BF7251F8230000EA020278
:10FE900082F0100208E00A494BF68F7251F82300F5
:10FEA00000EA020282F4805241F82320064B1B68CC
:10FEB0009B699847002000E0022010BDAC11002093
:10FEC000005C0040000100206811002008B5064BCE
:10FED0001B685A7A42F020025A72044B1B68DB6995
:10FEE0009847002008BD00BFAC1100206811002019
:10FEF000054B1A68538A18B98988CB1A138201E016
:10FF000008681818704700BFAC11002030B50E4BC0
:10FF10001C78002310E05FFA83FC4FEA8C0202F1A8
:10FF2000804202F5B842156848F68F7105EA010172
:10FF300041EA0C0111600133A342ECD3034B40F0C2
:10FF40008000186030BD00BF000100204C5C004004
:10FF5000704700BF08B50C4B002093F82C1000F040
:10FF60004FFE0A4B1B68187A082807D1084B4FF43C
:10FF700080521A80074B4FF010021A80092814BFD4
:10FF80000020012008BD00BF7C000020AC11002033
:10FF90005E1200206012002070B52D4B1C68237A81
:10FFA000032B01D0052B46D1A369228AABB1A2B1A4
:10FFB000A58A954228BF154628469847228A638A13
:10FFC000521BEB18064622826382002000F0E8FDF7
:10FFD0002A460146304600F0FBFB238A5BB11D4BED
:10FFE0004FF4405200201A80014600F0E7FD1A4B02
:10FFF0004FF030021A80A28A238A9A4203D8144B07
:020000040801F1
:1000000003221B6803E0124A1BB1136805221A720F
:100010000DE0126806211172104A1168104A89B267
:100020008A18520013600C4B4FF030021A80084BB4
:100030001B681B7A06E0072B03D10A4B1B68DB68A1
:1000400098470823024A12681372FFF783FF70BDB6
:10005000AC1100205E12002060120020505C0040B5
:100060000230002044110020F8B5244B1C68238A7C
:10007000267ABBB9042E15D1214822490278012ADB
:100080000BD1214C214A24680370A0B2821852007F
:1000900013604FF030020A802BE04FF010030B800A
:1000A000072626E0A68AA2699E4234BF35461D4631
:1000B0002846B34294BF04260226904707460020F4
:1000C00000F060FD2A460146384600F069FB2946EB
:1000D000002000F073FD638A228AEB186382094BCB
:1000E000551B4FF0300225821A80094B4FF44052C5
:1000F0001A80024B1B681E72F8BD00BFAC110020B5
:100100006007002060120020505C00400230002098
:100110005E12002008B5144B1B681A7A022A01D01F
:10012000042A05D1FFF7A0FF0F4B1B681B7A14E0D0
:10013000062A11D15A78052A0AD11A7812F07F0FAF
:1001400006D1D878FFF7E2FE084B1B681B6A984778
:10015000074B1B689B6898470823034A1268137271
:10016000FFF7F8FE08BD00BFAC11002068110020A9
:100170004411002038B5324B1B68187810F07F000E
:1001800004D15A7A22F020025A7258E0022855D13E
:100190005A88002A52D11A79002A4FD15A7912F07E
:1001A000800F22F0800405D0264951F8241001F078
:1001B000300104E0234951F8241001F44051224851
:1001C000007884423AD2002938D09B7A002B35D06F
:1001D00012F0800F0FD01B4B53F8243003F0300384
:1001E000102B25D1E4B2204600F082FC20463021BD
:1001F00000F05EFB1CE0134D55F8243003F440532F
:10020000B3F5805F14D134B9104B204693F82C100D
:1002100000F0F6FC02E0204600F056FC55F82420E1
:100220004BF68F7302EA030383F4405345F82430FE
:10023000074B1B685B699847002000E0022038BD2F
:10024000AC110020005C0040000100207C00002078
:1002500068110020F7B58D4B8D4E1A6835688D4BAF
:1002600092B2D3182A7A5B00092A1B681BD09BB272
:1002700003F1005303F540535B001C4614F8012BB7
:1002800003F10A072A705B786B70B4F8030000F082
:1002900063FE6880B4F80700346800F05DFEA0805B
:1002A00033687F88DF807A4C01212368DA881972ED
:1002B0005D78002A62D11A7812F07F022ED1092DC2
:1002C00002D1FFF715FD3BE0052D0DD193F9032079
:1002D000002A4EDB9A78002A4BD19A88002A48D10E
:1002E0009B7A002B37D044E0032D0BD1DA78012A1A
:1002F00027D19A882ABB5B7A13F0200F21D0FFF711
:10030000E5FD1DE0012D1CD1DA78012A19D19A886A
:10031000BAB95B7A13F0200F13D00AE0012A04D196
:100320000B2D0ED1FFF714FD0AE0022A09D1012D91
:1003300002D1FFF71FFF03E0032D02D1FFF780FD7D
:1003400048B1554B28461B685B699847032801D183
:1003500009230FE068B94D4A504B12684FF0300145
:1003600092B2D3185B0000221A604D4B198006230D
:1003700000E00823464A12681372E3E0062D18D104
:100380001A7812F07F0F40F097809B78012B03D1F1
:10039000414B1B68DB696EE0022B03D13E4B1B68AF
:1003A0001B6A68E0032B40F087803B4B1B685B6A4D
:1003B00061E0002D3CD1598800297DD15A6822F492
:1003C0007F42B2F5003F77D11A7812F07F0203D155
:1003D0009B88002B70D129E0012A0BD158792E4B34
:1003E0001B689B699847002866D123689B7A002B7D
:1003F00062D01BE0022A5FD15B7913F0800F03F01B
:100400000F0205D0274951F8221001F0300104E015
:10041000244951F8221001F44051234800788242C7
:100420004AD213F0700F47D1002945D01F4B23E06B
:10043000082D05D11B7813F07F0F3DD11C4B1BE01D
:100440000A2D39D11A7802F07F02012A34D19A7A22
:10045000002A31D0598800292ED15A6822F47F42CF
:10046000B2F5803F28D158790B4B1B689B699847A0
:1004700010BB104B00E0FBB1054A4FF000011268C1
:100480000020936151829847002020E0505C00409A
:10049000AC11002004300020441100200230002064
:1004A00060120020005C00400001002099FD00085F
:1004B000C9FC000829FD0008244C254B22681B6854
:1004C00050781B699847032801D1236806E01F4B29
:1004D0004FF6FF711B681A8A8A4201D1092203E094
:1004E000022800D012B908221A722BE093F90010EA
:1004F000002921DAD98801910198824202D9019A12
:100500001A8211E08A420FD21149096891F82C1021
:100510008A4201D2002105E092FBF1F001FB10229A
:1005200012B901210B4A1170094A126892F82C2065
:100530009A82FFF799FD05E003221A72064B4FF4E9
:1005400040521A80FFF706FDFEBD00BFAC1100202F
:1005500044110020600700205E120020074A02219B
:1005600008B5074811720749074B086007490A6038
:10057000074A13601B68984708BD00BF4C11002054
:1005800004010020681100207C000020AC11002034
:100590004411002008B529E047F6FF70086019886B
:1005A00001F00F018B0003F18043117003F5B84394
:1005B000196889B211F4004F09D0186840F68F719C
:1005C00000EA0101196012780E4B013A0BE011F0BC
:1005D000800F0BD0186848F60F7100EA010119600E
:1005E0001278094B013A53F8223098470749084BD3
:1005F0000868084A80B21880188800B20028CBDB4F
:1006000008BD00BFE4000020C8000020445C00409A
:100610004211002048110020F8B59AE047F6FF7615
:100620001E601688564F06F00F06B30003F1804394
:1006300003F5B8433E70002E64D12768266823680E
:1006400007F4405C03EA000080F400502060236857
:1006500006F0300003EA010181F0200121601388D7
:10066000484A13F0100F1080A5F800C004D023688A
:100670009BB213F0800F08D0226848F60F7302EA8D
:1006800003032360FFF746FD16E013F4006F08D064
:10069000226840F68F7302EA03032360FFF7DAFD56
:1006A0000AE013F4004F54D0226840F68F7302EA38
:1006B00003032360FFF770FC21682A884BF68F73D1
:1006C00001EA030312F4805F18BF83F4805312F42D
:1006D000005F2D4A18BF83F400531360294B116843
:1006E0001A8848F6BF7301EA030312F0100F18BF0F
:1006F00083F0100312F0200F234A18BF83F0200369
:1007000013603BE01C68A4B214F4004F0BD01968CE
:1007100040F68F7201EA02021A603A781B4B013AE6
:1007200053F82230984714F0800F12D0144948F63D
:100730000F720B789B0003F1804303F5B8431868F0
:1007400000EA02021A600A78114B013A53F822308B
:100750009847104B104A1D680B4C1FFA85FCA2F8F5
:1007600000C0B2F800C04BF68F700FFA8CFCBCF1E1
:10077000000F48F6BF71094DFFF650AFF8BD00BF3E
:100780004811002060120020005C0040E4000020BE
:10079000C8000020445C0040421100205E1200208E
:1007A00001F10051013201F5405110B549005208E4
:1007B000002308E010F803C06478013A4CEA042CE6
:1007C00021F813C00233C418002AF3D110BD00BFB2
:1007D00001F10051013201F5405110B549005208B4
:1007E000002304E031F81340013AC4520233002AD6
:1007F000F8D110BD014B1860704700BF405C00404D
:10080000014B186880B27047405C0040014B186093
:10081000704700BF445C0040014B186880B27047CD
:10082000445C0040014B186880B27047485C00404F
:10083000014B1860704700BF4C5C0040014B1868CA
:1008400080B270474C5C00404FF6F873024A00EAF1
:1008500003031360704700BF505C0040014B1868F1
:1008600080B27047505C0040014B43F82010704745
:10087000005C0040024B53F8200080B2704700BF7C
:10088000005C0040054B10B553F8204048F68F122D
:1008900004EA02020A4343F8202010BD005C004035
:1008A000024B53F8200000F4C0607047005C004029
:1008B0000A4B10B553F8202048F6BF7402EA04042E
:1008C00011F0100F18BF84F0100411F0200F18BFA2
:1008D00084F0200443F8204010BD00BF005C0040BD
:1008E0000A4B10B553F820204BF68F7402EA04042B
:1008F00011F4805F18BF84F4805411F4005F18BFB6
:1009000084F4005443F8204010BD00BF005C004058
:1009100038B50D460446FFF7ADFF012D02D120F496
:10092000805003E0022D04D120F01000014B43F869
:10093000240038BD005C0040024B53F8200000F05A
:1009400030007047005C0040024B53F8200000F478
:1009500040507047005C0040054B48F6BF7253F8AA
:10096000201001EA020282F0300243F82020704792
:10097000005C0040054B4BF68F7253F8201001EAE3
:10098000020282F4405243F820207047005C00408D
:10099000054B48F68F6253F8201001EA020242F438
:1009A000807243F820207047005C0040044B48F6FA
:1009B0008F6253F8201001EA020243F820207047AA
:1009C000005C0040044B48F68F6253F8201001EAA7
:1009D000020243F820207047005C0040054B48F6B7
:1009E0008F6253F8201001EA020242F4807243F849
:1009F00020207047005C0040054B48F68F6253F89A
:100A0000201001EA020242F4807243F8202070476D
:100A1000005C0040044B48F68F6253F8201001EA56
:100A2000020243F820207047005C0040044B53F85A
:100A3000200000F03000102814BF00200120704773
:100A4000005C0040054B53F8200000F44050B0F526
:100A5000805F14BF00200120704700BF005C004091
:100A6000044B40F68F7253F8201001EA020243F85B
:100A700020207047005C0040044B48F60F7253F88A
:100A8000201001EA020243F820207047005C004079
:100A9000054B48F68F7253F8201001EA020242F427
:100AA000804243F820207047005C0040054B48F628
:100AB0008F7253F8201001EA020242F0400243F81C
:100AC00020207047005C0040084B53F8202012F4AF
:100AD000804F09D053F8201048F68F7201EA0202C5
:100AE00042F4804243F82020704700BF005C004081
:100AF000084B53F8202012F0400F09D053F8201073
:100B000048F68F7201EA020242F0400243F82020C8
:100B1000704700BF005C0040054B10B553F8204003
:100B200048F68F7204EA02020A4343F8202010BDFF
:100B3000005C0040024B53F8200000F00F007047AB
:100B4000005C0040064B49081B6849009BB203EB60
:100B5000C00303F1005303F540535B001960704775
:100B6000505C0040054A064B1268490892B202EBFD
:100B7000C002D3185B00490019607047505C004008
:100B800004300020054B1B689BB203EBC00303F14C
:100B9000005303F540535B0018887047505C0040D9
:100BA000044A054B126892B202EBC002D3185B00F4
:100BB00018887047505C004004300020044A054B00
:100BC000126892B202EBC002D3185B001960704742
:100BD000505C0040023000203E2909D94B0911F039
:100BE0001F0F01D1013B9BB29B0243F4004305E080
:100BF0004B0811F0010F18BF01339B0203607047CF
:100C00000D4A0E4B126892B2D31803EBC0035B007F
:100C10003E2909D94A0911F01F0F01D1013A92B2B8
:100C2000920242F4004205E04A0811F0010F18BF99
:100C3000013292021A607047505C0040063000207A
:100C4000054A064B126892B202EBC002D3185B0051
:100C500018688005800D7047505C0040023000200D
:100C6000054A064B126892B202EBC002D3185B0031
:100C700018688005800D7047505C004006300020E9
:100C80000C4B30B51D681C68C0001FFA85FC8444FD
:100C9000A4B2094B00190CF1005CC3180CF5405CC0
:100CA000490852084FEA4C0049005B0052000160BD
:100CB0001A6030BD505C004004300020064B4908EB
:100CC0001B6849009BB203EBC00303F1005303F51B
:100CD00040535B0019607047505C0040054A064B6A
:100CE0001268490892B202EBC002D3185B004900B7
:100CF00019607047505C004004300020054B1B68B1
:100D00009BB203EBC00303F1005303F540535B00B8
:100D100018887047505C0040044A054B126892B234
:100D200002EBC002D3185B0018887047505C00408B
:100D300004300020012910B524D1254B25491B681A
:100D4000C0009BB2591809184B003E2A09D9510915
:100D500012F01F0F01D1013989B2890241F400411B
:100D600005E0510812F0010F18BF01318902196026
:100D70001749194B096889B2CB18181840003E2A48
:100D80001ED913E0022922D1114BC0001C681B6838
:100D9000A4B21FFA83FC0F490F4B84440019411879
:100DA000634449005B000A601A6010E0530912F0C6
:100DB0001F0F01D1013B9BB29B0243F4004305E0AE
:100DC000530812F0010F18BF01339B02036010BDDE
:100DD000505C0040023000200630002001291BD169
:100DE0001349144B096889B2CB1803EBC0004000CB
:100DF0003E2A09D9530912F01F0F01D1013B9BB2C2
:100E00009B0243F4004305E0530812F0010F18BFA2
:100E100001339B0203600AE0022908D10449054B13
:100E2000096889B201EBC000C3185B001A60704703
:100E3000505C00400230002001291BD11349144BA3
:100E4000096889B2CB1803EBC00040003E2A09D9DB
:100E5000530912F01F0F01D1013B9BB29B0243F4D7
:100E6000004305E0530812F0010F18BF01339B0245
:100E700003600AE0022908D10449054B096889B2D8
:100E800001EBC000C3185B001A607047505C004063
:100E900006300020054A064B126892B202EBC002EF
:100EA000D3185B0018688005800D7047505C0040C7
:100EB00002300020054A064B126892B202EBC002D3
:100EC000D3185B0018688005800D7047505C0040A7
:100ED000063000200D4BC00019680D4A89B2411838
:100EE0008A185200128812F47C4F01D001200CE0C5
:100EF0001A68084B92B28018C3185B0018888005E6
:100F0000800D002814BF022000207047505C004074
:100F10000630002002300020012909D10B4A48F692
:100F20008F7352F8201001EA030343F040030AE0F4
:100F300002290AD1054A48F68F7352F8201001EAB7
:100F4000030343F4804342F820307047005C0040C4
:100F500041EA0020704700BF030AC0B243EA002004
:100F6000704700BF08B500220A2300F045F808BD0D
:100F700008B500210A2200F0DFF808BDF0B40378BC
:100F8000002B2DD040F23012C2F20002156802E0B0
:100F900010F8013FEBB15A1903F12004527812F016
:100FA00001070A7808BF1C4601F10101561C94464E
:100FB000AE5D16F0010F18BF02F1200C6445E7D0BA
:100FC00007B1203316F0010F18BF2032981AF0BC79
:100FD00070470A786F78561C07F00107AE5DEFE79F
:100FE00040F230100A78C2F20000561C05686F7893
:100FF000AE5D07F00107E3E72DE9F04F40F2301551
:10100000C2F2000583B00C461F46D5F800800E469C
:101010000190009216F8015B08EB050393F801B00C
:101020001BF0080BF6D12D2D65D02B2D08BF16F81F
:10103000015BD7F1010338BF0023102F14BF1A46FC
:1010400043F0010232B1302D66D01BB1302D0CBF00
:1010500008270A27BBF1000F394614BF4FF000499B
:101060006FF00049484600F0A5F948468A463946DF
:1010700000F072F800218C4608EB0502A5F1300360
:10108000527812F0040F08D112F0030F20D012F0A2
:10109000010F14BF37235723EB1A9F4218DD8445F5
:1010A00094BF0022012252EAD1714FF0FF310CD1DE
:1010B000844514BF002201225345D4BF002202F010
:1010C000010212B907FB0C3C012116F8015BD3E7C2
:1010D000B1F1FF3F14D0BBF1000F09D16046009B76
:1010E0001BB101B1741E009A146003B0BDE8F08F0B
:1010F000CCF10000F3E716F8015B4FF0010B98E725
:10110000019ABBF1000F4FF0220314BF4FF00040D3
:101110006FF000401360E2E73278782A14BF0021B4
:101120000121582A14BF0A4641F00102002A8CD03E
:101130007578102702368DE710B540F23414C2F2EC
:1011400000048C461346014662462068FFF754FFB0
:1011500010BD00BF000000004A1E08BF7047C0F06D
:101160002481884240F21681114200F01781B0FAC2
:1011700080F3B1FA81F2A2EB0303C3F11F0304A2CF
:1011800002EB03134FF000029F4600BFAFF3008055
:10119000B0EBC17F00BF42EB020228BFA0EBC170E1
:1011A000B0EB817F00BF42EB020228BFA0EB817051
:1011B000B0EB417F00BF42EB020228BFA0EB4170C1
:1011C000B0EB017F00BF42EB020228BFA0EB017031
:1011D000B0EBC16F00BF42EB020228BFA0EBC160C1
:1011E000B0EB816F00BF42EB020228BFA0EB816031
:1011F000B0EB416F00BF42EB020228BFA0EB4160A1
:10120000B0EB016F00BF42EB020228BFA0EB016010
:10121000B0EBC15F00BF42EB020228BFA0EBC150A0
:10122000B0EB815F00BF42EB020228BFA0EB815010
:10123000B0EB415F00BF42EB020228BFA0EB415080
:10124000B0EB015F00BF42EB020228BFA0EB0150F0
:10125000B0EBC14F00BF42EB020228BFA0EBC14080
:10126000B0EB814F00BF42EB020228BFA0EB8140F0
:10127000B0EB414F00BF42EB020228BFA0EB414060
:10128000B0EB014F00BF42EB020228BFA0EB0140D0
:10129000B0EBC13F00BF42EB020228BFA0EBC13060
:1012A000B0EB813F00BF42EB020228BFA0EB8130D0
:1012B000B0EB413F00BF42EB020228BFA0EB413040
:1012C000B0EB013F00BF42EB020228BFA0EB0130B0
:1012D000B0EBC12F00BF42EB020228BFA0EBC12040
:1012E000B0EB812F00BF42EB020228BFA0EB8120B0
:1012F000B0EB412F00BF42EB020228BFA0EB412020
:10130000B0EB012F00BF42EB020228BFA0EB01208F
:10131000B0EBC11F00BF42EB020228BFA0EBC1101F
:10132000B0EB811F00BF42EB020228BFA0EB81108F
:10133000B0EB411F00BF42EB020228BFA0EB4110FF
:10134000B0EB011F00BF42EB020228BFA0EB01106F
:10135000B0EBC10F00BF42EB020228BFA0EBC100FF
:10136000B0EB810F00BF42EB020228BFA0EB81006F
:10137000B0EB410F00BF42EB020228BFA0EB4100DF
:10138000B0EB010F00BF42EB020228BFA0EB01004F
:10139000104670470CBF012000207047B1FA81F25F
:1013A000C2F11F0220FA02F0704708B14FF0FF307F
:1013B00000F00EB80029F8D02DE90340FFF7CCFE6D
:1013C000BDE8064002FB00F3A1EB0301704700BF3C
:1013D000704700BF81F0004102E000BF83F000438E
:1013E00030B54FEA41044FEA430594EA050F08BFC0
:1013F00090EA020F1FBF54EA000C55EA020C7FEA84
:10140000645C7FEA655C00F0E2804FEA5454D4EB00
:101410005555B8BF6D420CDD2C4480EA020281EACA
:10142000030382EA000083EA010180EA020281EA02
:101430000303362D88BF30BD11F0004F4FEA013154
:101440004FF4801C4CEA113102D0404261EB410163
:1014500013F0004F4FEA03334CEA133302D05242E9
:1014600063EB430394EA050F00F0A780A4F10104A5
:10147000D5F1200E0DDB02FA0EFC22FA05F28018DF
:1014800041F1000103FA0EF2801843FA05F35941C5
:101490000EE0A5F120050EF1200E012A03FA0EFC44
:1014A00028BF4CF0020C43FA05F3C01851EBE3716E
:1014B00001F0004507D54FF0000EDCF1000C7EEB8B
:1014C00000006EEB0101B1F5801F1BD3B1F5001FC9
:1014D0000CD349085FEA30004FEA3C0C04F10104E8
:1014E0004FEA445212F5800F80F09A80BCF1004F11
:1014F00008BF5FEA500C50F1000041EB045141EA93
:10150000050130BD5FEA4C0C404141EB010111F493
:10151000801FA4F10104E9D191F0000F04BF01463E
:101520000020B1FA81F308BF2033A3F10B03B3F11C
:1015300020020CDA0C3208DD02F1140CC2F10C02AC
:1015400001FA0CF021FA02F10CE002F11402D8BF0A
:10155000C2F1200C01FA02F120FA0CFCDCBF41EAD6
:101560000C019040E41AA2BF01EB0451294330BDA5
:101570006FEA04041F3C1CDA0C340EDC04F1140482
:10158000C4F1200220FA04F001FA02F340EA030059
:1015900021FA04F345EA030130BDC4F10C04C4F19F
:1015A000200220FA02F001FA04F340EA030029467F
:1015B00030BD21FA04F0294630BD94F0000F83F4C9
:1015C000801306BF81F480110134013D4EE77FEAAC
:1015D000645C18BF7FEA655C29D094EA050F08BFF8
:1015E00090EA020F05D054EA000C04BF19461046D9
:1015F00030BD91EA030F1EBF0021002030BD5FEA1D
:10160000545C05D14000494128BF41F0004130BD44
:1016100014F580043CBF01F5801130BD01F0004598
:1016200045F0FE4141F470014FF0000030BD7FEA0B
:10163000645C1ABF194610467FEA655C1CBF0B4606
:10164000024650EA013406BF52EA033591EA030F1D
:1016500041F4002130BD00BF90F0000F04BF002115
:10166000704730B54FF4806404F132044FF0000548
:101670004FF0000150E700BF90F0000F04BF0021C1
:10168000704730B54FF4806404F1320410F0004527
:1016900048BF40424FF000013EE700BF42004FEA22
:1016A000E2014FEA31014FEA02701FBF12F07F439F
:1016B00093F07F4F81F06051704792F0000F14BF9C
:1016C00093F07F4F704730B54FF4607401F00045E0
:1016D00021F0004120E700BF50EA010208BF704737
:1016E00030B54FF000050AE050EA010208BF70472C
:1016F00030B511F0004502D5404261EB41014FF495
:10170000806404F132045FEA915C3FF4DCAE4FF098
:1017100003025FEADC0C18BF03325FEADC0C18BF7F
:10172000033202EBDC02C2F1200300FA03FC20FAD0
:1017300002F001FA03FE40EA0E0021FA02F114441D
:10174000C1E600BF70B54FF0FF0C4CF4E06C1CEA32
:1017500011541DBF1CEA135594EA0C0F95EA0C0FA7
:1017600000F0DEF82C4481EA030621EA4C5123EA1A
:101770004C5350EA013518BF52EA033541F4801149
:1017800043F4801338D0A0FB02CE4FF00005E1FBFC
:1017900002E506F00042E0FB03E54FF00006E1FB46
:1017A00003569CF0000F18BF4EF0010EA4F1FF0489
:1017B000B6F5007F64F5407404D25FEA4E0E6D41C9
:1017C00046EB060642EAC62141EA55514FEAC520DA
:1017D00040EA5E504FEACE2EB4F1FD0C88BFBCF556
:1017E000E06F1ED8BEF1004F08BF5FEA500E50F107
:1017F000000041EB045170BD06F0004646EA0101CD
:1018000040EA020081EA0301B4EB5C04C2BFD4EBFE
:101810000C0541EA045170BD41F480114FF0000EF7
:10182000013C00F3AB8014F1360FDEBF002001F065
:10183000004170BDC4F10004203C35DA0C341BDCDF
:1018400004F11404C4F1200500FA05F320FA04F0B1
:1018500001FA05F240EA020001F0004221F00041E5
:1018600010EBD37021FA04F642EB06015EEA430E58
:1018700008BF20EAD37070BDC4F10C04C4F1200588
:1018800000FA04F320FA05F001FA04F240EA02003B
:1018900001F0004110EBD37041F100015EEA430E0C
:1018A00008BF20EAD37070BDC4F1200500FA05F22C
:1018B0004EEA020E20FA04F301FA05F243EA0203AB
:1018C00021FA04F001F0004121FA04F220EA0200BA
:1018D00000EBD3705EEA430E08BF20EAD37070BD00
:1018E00094F0000F0FD101F00046400041EB0101E0
:1018F00011F4801F08BF013CF7D041EA060195F0C2
:10190000000F18BF704703F00046520043EB03037B
:1019100013F4801F08BF013DF7D043EA0603704768
:1019200094EA0C0F0CEA135518BF95EA0C0F0CD073
:1019300050EA410618BF52EA4306D1D181EA0301B9
:1019400001F000414FF0000070BD50EA410606BFB3
:101950001046194652EA430619D094EA0C0F02D1F8
:1019600050EA013613D195EA0C0F05D152EA03363D
:101970001CBF104619460AD181EA030101F000415B
:1019800041F0FE4141F470014FF0000070BD41F0A4
:10199000FE4141F4780170BD70B54FF0FF0C4CF47E
:1019A000E06C1CEA11541DBF1CEA135594EA0C0F9D
:1019B00095EA0C0F00F0A7F8A4EB050481EA030EEA
:1019C00052EA03354FEA013100F088804FEA0333D1
:1019D0004FF0805545EA131343EA12634FEA02229F
:1019E00045EA111545EA10654FEA00260EF0004160
:1019F0009D4208BF964244F1FD0404F5407402D2B2
:101A00005B084FEA3202B61A65EB03055B084FEA42
:101A100032024FF480104FF4002CB6EB020E75EB3F
:101A2000030E22BFB61A754640EA0C005B084FEA67
:101A30003202B6EB020E75EB030E22BFB61A7546E4
:101A400040EA5C005B084FEA3202B6EB020E75EB2F
:101A5000030E22BFB61A754640EA9C005B084FEAA7
:101A60003202B6EB020E75EB030E22BFB61A7546B4
:101A700040EADC0055EA060E18D04FEA051545EAA3
:101A800016754FEA06164FEAC30343EA52734FEA4C
:101A9000C2025FEA1C1CC0D111F4801F0BD141EAC5
:101AA00000014FF000004FF0004CB6E711F4801F2A
:101AB00004BF01430020B4F1FD0C88BFBCF5E06F0A
:101AC0003FF6AFAEB5EB030C04BFB6EB020C5FEA1A
:101AD000500C50F1000041EB045170BD0EF0004E6F
:101AE0004EEA113114EB5C04C2BFD4EB0C0541EAA1
:101AF000045170BD41F480114FF0000E013C90E69E
:101B000045EA060E8DE60CEA135594EA0C0F08BF61
:101B100095EA0C0F3FF43BAF94EA0C0F0AD150EA60
:101B200001347FF434AF95EA0C0F7FF425AF1046F3
:101B300019462CE795EA0C0F06D152EA03353FF41B
:101B4000FDAE1046194622E750EA410618BF52EA98
:101B500043067FF4C5AE50EA41047FF40DAF52EA6C
:101B600043057FF4EBAE12E74FEA410212F5001293
:101B700015D211D56FF47873B3EB625212D94FEAD4
:101B8000C12343F0004343EA505311F0004F23FABE
:101B900002F018BF404270474FF00000704750EA13
:101BA000013005D111F0004008BF6FF000407047D0
:101BB0004FF00000704700BF4FEA4102B2F1E0432E
:101BC00024BFB3F5001CDCF1FE5C0DD901F0004C24
:101BD0004FEAC0024CEA5070B2F1004F40EB830074
:101BE00008BF20F00100704711F0804F21D113F1A0
:101BF0003872BCBF01F00040704741F480114FEAD9
:101C00005252C2F11802C2F1200C10FA0CF320FA61
:101C100002F018BF40F001004FEAC1234FEAD3237E
:101C200003FA0CFC40EA0C0023FA02F34FEA4303E8
:101C3000CCE77FEA625307D150EA01331EBF4FF071
:101C4000FE4040F44000704701F0004040F0FE408C
:101C500040F40000704700BF80F0004002E000BF89
:101C600081F0004142001FBF5FEA410392EA030F87
:101C70007FEA226C7FEA236C6AD04FEA1262D2EBD1
:101C80001363C1BFD218414048404140B8BF5B42D6
:101C9000192B88BF704710F0004F40F4000020F06F
:101CA0007F4018BF404211F0004F41F4000121F085
:101CB0007F4118BF494292EA030F3FD0A2F10102CF
:101CC00041FA03FC10EB0C00C3F1200301FA03F10D
:101CD00000F0004302D5494260EB4000B0F5000F30
:101CE00013D3B0F1807F06D340084FEA310102F1EF
:101CF0000102FE2A51D2B1F1004F40EBC25008BFA1
:101D000020F0010040EA03007047490040EB00006A
:101D100010F4000FA2F10102EDD1B0FA80FCACF199
:101D2000080CB2EB0C0200FA0CF0AABF00EBC25098
:101D300052421843BCBFD0401843704792F0000F86
:101D400081F4000106BF80F400000132013BB5E7D9
:101D50004FEA41037FEA226C18BF7FEA236C21D04F
:101D600092EA030F04D092F0000F08BF08467047B4
:101D700090EA010F1CBF0020704712F07F4F04D182
:101D8000400028BF40F00040704712F100723CBF95
:101D900000F50000704700F0004343F0FE4040F4BF
:101DA000000070477FEA226216BF08467FEA23637D
:101DB0000146420206BF5FEA412390EA010F40F468
:101DC000800070474FF0000304E000BF10F00043B4
:101DD00048BF40425FEA000C08BF704743F096439B
:101DE00001464FF000001CE050EA010208BF7047B6
:101DF0004FF000030AE000BF50EA010208BF70473D
:101E000011F0004302D5404261EB41015FEA010C51
:101E100002BF84460146002043F0B64308BFA3F149
:101E20008053A3F50003BCFA8CF2083AA3EBC2532B
:101E300010DB01FA02FC634400FA02FCC2F120024A
:101E4000BCF1004F20FA02F243EB020008BF20F081
:101E50000100704702F1200201FA02FCC2F12002E7
:101E600050EA4C0021FA02F243EB020008BF20EADC
:101E7000DC7070474FF0FF0C1CEAD0521EBF1CEA0A
:101E8000D15392EA0C0F93EA0C0F6FD01A4480EAF8
:101E9000010C400218BF5FEA41211ED04FF00063E1
:101EA00043EA501043EA5111A0FB01310CF000400D
:101EB000B1F5000F3EBF490041EAD3715B0040EA33
:101EC000010062F17F02FD2A1DD8B3F1004F40EB03
:101ED000C25008BF20F00100704790F0000F0CF0D6
:101EE000004C08BF49024CEA502040EA51207F3A9A
:101EF000C2BFD2F1FF0340EAC250704740F4000075
:101F00004FF00003013A5DDC12F1190FDCBF00F065
:101F100000407047C2F10002410021FA02F1C2F113
:101F2000200200FA02FC5FEA310040F1000053EAAF
:101F30004C0308BF20EADC70704792F0000F00F0FD
:101F4000004C02BF400010F4000F013AF9D040EA03
:101F50000C0093F0000F01F0004C02BF490011F497
:101F6000000F013BF9D041EA0C018FE70CEAD15395
:101F700092EA0C0F18BF93EA0C0F0AD030F0004C15
:101F800018BF31F0004CD8D180EA010000F00040C9
:101F9000704790F0000F17BF90F0004F084691F087
:101FA000000F91F0004F14D092EA0C0F01D14202C1
:101FB0000FD193EA0C0F03D14B0218BF084608D18A
:101FC00080EA010000F0004040F0FE4040F40000D4
:101FD000704740F0FE4040F4400070474FF0FF0C67
:101FE0001CEAD0521EBF1CEAD15392EA0C0F93EAAE
:101FF0000C0F69D0A2EB030280EA010C49024FEA00
:10200000402037D04FF0805343EA111143EA1013B8
:102010000CF000408B4238BF5B0042F17D024FF470
:10202000000C8B4224BF5B1A40EA0C00B3EB510F4B
:1020300024BFA3EB510340EA5C00B3EB910F24BF34
:10204000A3EB910340EA9C00B3EBD10F24BFA3EBB9
:10205000D10340EADC001B0118BF5FEA1C1CE0D181
:10206000FD2A3FF650AF8B4240EBC25008BF20F034
:10207000010070470CF0004C4CEA50207F32C2BF88
:10208000D2F1FF0340EAC250704740F400004FF025
:102090000003013A37E792F0000F00F0004C02BF56
:1020A000400010F4000F013AF9D040EA0C0093F020
:1020B000000F01F0004C02BF490011F4000F013B7A
:1020C000F9D041EA0C0195E70CEAD15392EA0C0FE2
:1020D00008D142027FF47DAF93EA0C0F7FF470AF1A
:1020E000084676E793EA0C0F04D14B023FF44CAF5D
:1020F00008466EE730F0004C18BF31F0004CCAD1F2
:1021000030F000427FF45CAF31F000437FF43CAF2D
:102110005FE700BF4FF0FF3C06E000BF4FF0010C4F
:1021200002E000BF4FF0010C4DF804CD4FEA400231
:102130004FEA41037FEA226C18BF7FEA236C11D07B
:1021400001B052EA530C18BF90EA010F58BFB2EB2E
:10215000030088BFC81738BF6FEAE17018BF40F0AE
:10216000010070477FEA226C02D15FEA402C05D162
:102170007FEA236CE4D15FEA412CE1D05DF8040BE7
:10218000704700BF844608466146FFE70FB5FFF77A
:10219000C9FF002848BF10F1000F0FBD4DF808ED32
:1021A000FFF7F4FF0CBF012000205DF808FB00BF23
:1021B0004DF808EDFFF7EAFF34BF012000205DF87D
:1021C00008FB00BF4DF808EDFFF7E0FF94BF0120CA
:1021D00000205DF808FB00BF4DF808EDFFF7D2FFC7
:1021E00094BF012000205DF808FB00BF4DF808ED0A
:1021F000FFF7C8FF34BF012000205DF808FB00BFD7
:1022000042000ED2B2F1FE4F0BD34FF09E03B3EB60
:10221000126209D44FEA002343F0004323FA02F08C
:1022200070474FF00000704712F1610F01D1420278
:1022300002D14FF0FF3070474FF00000704700BFF1
:102240000000000000000000010003E800000000A2
:1022500000000003E800000000000200FA0600038E
:102260000000000000370600000000000000000031
:10227000F401000064000000018008080000000074
:10228000000200000000000000000000C800000084
:102290001201100102000040D01650060118010280
:1022A0000301000009024300020100C032090400DA
:1022B00000010202010005240010010524010001B3
:1022C000042402020524060001070582030800FF1A
:1022D00009040100020A0000000705030240000093
:1022E000070581024000000004030904260354008E
:1022F000720069006E0061006D00690063004D00AE
:102300006F00740069006F006E00200043007400CD
:102310006C000000320354004D0043004D002D00BE
:1023200036003100310030002000280076006900BE
:1023300072007400750061006C00200043004F00C3
:102340004D002900200000000102030405060000E2
:10235000524F5200000106524F4C000002064D53EE
:1023600054000003024D5650000004075341500032
:102370000005074741500000060353544150000731
:1023800003525341500008035347500000090747C8
:10239000475000000A0353544750000B0352534761
:1023A00050000C0352465300000D0353494F0000E8
:1023B0000E0747494F00000F0353414300001D071C
:1023C00053434F00001E0747434F00001F03434382
:1023D0004F0000200341434F0000270355463000C3
:1023E0000040075546310000410755463200004283
:1023F000075546330000430755463400004407554F
:102400004635000045075546360000460755463715
:102410000000470752554E0000810553544F5000AD
:10242000800042494E00008B0000000000000000C8
:10243000020000000000000100000000010203048F
:1024400001020304060708090204060800202020F0
:102450002020202020202828282828202020202054
:102460002020202020202020202020202088101024
:102470001010101010101010101010101004040480
:10248000040404040404041010101010101041413E
:10249000414141410101010101010101010101012C
:1024A0000101010101010101101010101010424240
:1024B00042424242020202020202020202020202FC
:1024C000020202020202020210101010200000009C
:1024D00000000000000000000000000000000000FC
:1024E00000000000000000000000000000000000EC
:1024F00000000000000000000000000000000000DC
:1025000000000000000000000000000000000000CB
:1025100000000000000000000000000000000000BB
:1025200000000000000000000000000000000000AB
:10253000000000000000000000000000000000009B
:10254000000000000000000000000000000000008B
:102550003631313056313234004142530052454C0D
:1025600000434F4F52440053544152540053544F70
:1025700050005354415455530000000043000000E4
:1025800050250108000102000008000001000000C1
:102590000200000000000000000000000000000039
:1025A000000000000000000000000000000000002B
:1025B000000000000000000000000000000000001B
:1025C0000000000000C2010000000800E82201082D
:1025D00004000000EC22010826000000142301087A
:1025E00032000000AC0000201A000000A422010804
:1025F000430000009022010812000000A1A0000882
:10260000A99E0008B99C0008CD9C0008D19C000838
:10261000319D0008559D0008999E0008899E00087C
:10262000659E000800000000400000001A035400EE
:102630004D00430036003100310030000000000042
:102640000000000000000000B99B000851FF0008D6
:1026500051FF000851FF000851FF000851FF00081A
:1026600051FF000851FF000851FF0008F99F0008C2
:1026700051FF000851FF000851FF000851FF0008FA
:102680000401000051FF0008959C000851FF00085C
:1026900051FF000851FF000851FF000851FF0008DA
:1026A00051FF0008AD9C0008010000004D24010806
:1026B0004C24010838010020000000000000000048
:1026C000000000000000000000000000000000000A
:1026D00000000000000000007C2501080000000050
:1026E00000000000000000000000000000000000EA
:1026F00000000000000000000000000000000000DA
:1027000000000000000000000000000000000000C9
:1027100000000000000000000000000000000000B9
:1027200000000000000000000000000000000000A9
:102730000000000000000000000000000000000099
:102740000000000000000000000000000000000089
:102750000000000000000000000000000000000079
:102760000000000000000000000000000000000069
:102770000000000000000000000000000000000059
:102780000000000000000000000000000000000049
:102790000000000000000000000000000000000039
:0827A000000000000000000031
:04000005080041109E
:00000001FF
